:1000000055C7000084C7000082C7000080C70000F9
:100010007EC700007CC700007AC7000078C70000D8
:1000200076C7000074C7000072C7000070C70000E8
:100030006EC700000C94A5686AC7000068C700007E
:1000400066C7000064C7000062C7000060C7000008
:100050005EC700005CC700005AC700000C94828194
:1000600056C700000C945D850C94938550C7000022
:100070004EC700004CC700004AC7000048C7000038
:1000800046C7000044C7000042C7000040C7000048
:100090003EC700003CC700003AC700000C94F7615F
:1000A00036C7000034C7000032C7000030C7000068
:1000B0002EC700002CC700002AC7000028C7000078
:1000C00026C7000024C7000022C700000C94088641
:1000D0000C943E861CC700000C94B3860C94E986F1
:1000E00016C700007D455D45894589458945894597
:1000F0008945894589458945894589456E448044B6
:1001000087448E4495449C44A144AA44B144C844C5
:10011000CB448945CF44D244D444D744F144F3443A
:10012000FA44014514451B452245CF82D282C18243
:10013000C582CB820983D682DA82E082E482E882B9
:10014000EE82F282F6820983FC8200830483084AED
:10015000D73B3BCE016E84BCBFFDC12F3D6C7431DB
:100160009ABD56833DDA3D00C77F11BED9E4BB4C32
:100170003E916BAAAABE000000803F07634236B7DB
:100180009BD8A71A39685618AEBAAB558C1D3CB728
:10019000CC5763BD6DEDFD753EF6177231BF0000A3
:1001A00000803F08000000BE922449123EABAAAA7C
:1001B0002ABECDCCCC4C3E00000080BEABAAAAAA81
:1001C0003E00000000BF000000803F000000000073
:1001D000084178D3BB4387D1133D190E3CC3BD42C0
:1001E00082AD2B3E68EC8276BED98FE1A93E4C8071
:1001F000EFFFBE01C4FF7F3F0000000000003E4D46
:100200006F74696F6E20627920756C747261736FA0
:100210006E632073656E736F723A0A00696E707553
:10022000742044535463616C6962726174653A006E
:100230004E6F20445320546865726D6F6D65746510
:1002400072210050726573732061206B6579004CD8
:100250004344206F6E00234E6F2073656E736F7280
:1002600020666F7220504D21004E6F2073656E73B3
:100270006F722100504D313A322E353A3130004DF7
:100280006561737572696E672E2E004F3220436F61
:100290006E6300434F3220436F6E630070482076D8
:1002A000616C756500547572626964697479004E99
:1002B0006F2073656E736F72210049522054656D13
:1002C0007065726174757265004D656173757269F0
:1002D0006E672E2E004C6967687420496E74656ED7
:1002E0007369747900416E676C65732F006765747C
:1002F00053656C665465737442697428293A20000A
:100300006973496E74657272757074456E61626C62
:1003100065642831293A2000676574496E746572F6
:10032000727570744D617070696E672831293A205A
:1003300000676574496E74657272757074536F7579
:100340007263652831293A2000676574496E7465C7
:100350007272757074536F7572636528293A200044
:100360006765745261746528293A20332E3134311F
:1003700035393F00616363656C2E69734C6F77504C
:100380006F77657228293A2000616363656C2E6976
:100390007341736C65657028293A20006163636559
:1003A0006C2E6973546170536F757263654F6E5A2A
:1003B00028293A2000616363656C2E69735461706B
:1003C000536F757263654F6E5928293A2000616337
:1003D00063656C2E6973546170536F757263654FFA
:1003E0006E5828293A2000616363656C2E69734159
:1003F00063746976697479536F757263654F6E5A69
:1004000028293A2000616363656C2E697341637427
:100410006976697479536F757263654F6E592829CF
:100420003A200069734163746976697479536F7512
:100430007263654F6E5828293A20006973546170C1
:10044000446574656374696F6E4F6E5A28293B204A
:1004500066616C73653F2000697354617044657414
:10046000656374696F6E4F6E5A28293B20747275EC
:10047000653F2000697354617044657465637469F5
:100480006F6E4F6E5928293B2066616C73653F2063
:10049000006973546170446574656374696F6E4F6D
:1004A0006E5928293B20747275653F20006973548A
:1004B0006170446574656374696F6E4F6E58282966
:1004C0003B2066616C73653F200069735461704422
:1004D0006574656374696F6E4F6E5828293B20748C
:1004E0007275653F2000676574537570707265732F
:1004F0007342697428293B2066616C73653F200054
:1005000067657453757070726573734269742829D6
:100510003B20747275653F2000697341637469768E
:10052000697479416328293A20006973496E6163CF
:100530007469766974795A456E61626C65642829BC
:100540003A20006973496E616374697669747959F8
:10055000456E61626C656428293A20006973496EB2
:10056000616374697669747958456E61626C65641B
:1005700028293A2000697341637469766974795A4D
:10058000456E61626C656428293A20006973416395
:1005900074697669747959456E61626C656428295D
:1005A0003A20006973416374697669747958456EBD
:1005B00061626C656428293A20006765744672653B
:1005C0006546616C6C4475726174696F6E28293A76
:1005D00020006765744672656546616C6C5468728C
:1005E0006573686F6C6428293A20006765745469E4
:1005F0006D65496E616374697669747928293A205A
:1006000000676574496E61637469766974795468CA
:10061000726573686F6C6428292000676574416394
:100620007469766974795468726573686F6C64284C
:10063000292000676574446F75626C65546170575A
:10064000696E646F7728292000676574446F75624E
:100650006C655461704C6174656E637928293A2029
:10066000006765745461704475726174696F6E28B7
:10067000293A2000676574417869734F666673652F
:10068000742826782C2026792C20267A293A2000D6
:100690006765745461705468726573686F6C642820
:1006A000293A200058595A2047733A200058595A7D
:1006B00020434F554E54533A2000736574206761B0
:1006C000696E735B5D3A006761696E735F6F726933
:1006D000675B5D3A00466C616D65204952004F666C
:1006E00066206169722D636F6E64210049742773FF
:1006F00020746F6F20636F6F6C210054656D7020E4
:1007000069732066696E6521004973206169722DE5
:10071000636F6E64206F6E3F00497427732071759C
:1007200069746520686F74210049742773207665A9
:10073000727920686F74210054656D702048756D62
:10074000696469747900234E6F2073656E736F72EC
:1007500020666F722074656D7020262068756D6943
:100760006469747921004E6F2053656E736F722136
:100770000054656D702048756D6964697479004F27
:100780006666206169722D636F6E6421004974276B
:100790007320746F6F20636F6F6C210054656D70F0
:1007A0002069732066696E65210049732061697252
:1007B0002D636F6E64206F6E3F0049742773207144
:1007C0007569746520686F742100497427732076F9
:1007D00065727920686F74212000616E6F7468659E
:1007E0007220495220696E7075743D006B657932D4
:1007F0003D006B6579323D00496E76616C6964201D
:100800006B657921007265706C6965733D00233AF0
:1008100053686F772F48696465204C4344002A3A37
:10082000546869732048656C700044433A436C65B2
:100830006172204C43440044423A5265736574200F
:100840004C6F676765720044373A4D6F74696F6E1D
:100850000044363A44532054656D700044353A558F
:100860005620496E74656E736974790044343A4F4A
:100870003220636F6E632E0044333A434F3220635D
:100880006F6E632E0044323A504D28313A322E3585
:100890003A3130290044323A504D28313A322E351F
:1008A0003A3130292A0044313A54757262696469D8
:1008B00074790044303A566F6C7461676500393A58
:1008C0006F7220334420616363656C2E00393A49AE
:1008D0006E636C2E20616E672E00383A7048207669
:1008E000616C756500373A49522054656D70003768
:1008F0003A49522054656D702A00363A4D61676E50
:1009000065746963206669656C6400353A47617394
:10091000204C6576656C00343A495220466C616D16
:100920006500333A4C6967687420496E742E003252
:100930003A616E642048656967687400323A5465AC
:100940006D7020507265737375726500313A54652D
:100950006D702048756D696469747900303A536F21
:10096000756E64204C6576656C00303A536F756E19
:1009700064204C6576656C2A0020202020202020F1
:100980002020202020202020002020202020202087
:100990002020202020202020002020202020202077
:1009A0002020202020202020200020202020202067
:1009B0002020202020202020202000202020202057
:1009C0002020202020202020202020002020202047
:1009D000202020202020202020202020004C6F6775
:1009E00067657220446972656374696F6E002D2DAE
:1009F0002D2D2D2D2D2D2D2D2D2D2D2D2D2D2D2D27
:100A00002D2D2D2D2D2D2D2D2D2D2D2D2D2D2D2D16
:100A10002D2D005265736F6C7574696F6E3A2020CE
:100A200020004D696E2056616C75653A20202020AB
:100A3000004D61782056616C75653A2020202000B9
:100A4000556E697175652049443A20202020004484
:100A50007269766572205665723A202020005365CF
:100A60006E736F723A20202020202020002D2D2D23
:100A70002D204D61676E657469632053656E736FD9
:100A800072202D2D2D2D2D2D2D2D2D2D2D2D2D2D5E
:100A90002D2D2D2D2D2D006E6F20484D43353838CE
:100AA00033206D61676E657469632073656E736F63
:100AB00072202E2E2E20436865636B207769726941
:100AC0006E67210020766F6C746167653D00547518
:100AD00072626964697479205570706572204C691E
:100AE0006D69743A200020766F6C746167653D0013
:100AF000547572626964697479204C6F77657220ED
:100B00004C696D69743A2000547572626964697445
:100B100079204C6F776572204C696D697420566935
:100B20006E663A2000434F32204D415820766F6C5C
:100B300074202800434F32207A65726F20766F6CE4
:100B4000742028004F322063616C6962726174699D
:100B50006F6E3A2000547572626964697479204C32
:100B60006F776572204C696D69742056313A2000A8
:100B700023506172616D6574657273002343616C0B
:100B80006962726174696F6E2050726573737572F9
:100B9000653D0023536561206C6576656C205028A7
:100BA00063616C63293D00234572726F723A707203
:100BB00065737375726520424D503038352C206353
:100BC0006865636B20776972696E672100495220FE
:100BD00054656D702073656E736F7220666F756EED
:100BE0006400504D322E352073656E736F72206C29
:100BF000696B656C7920666F756E6400536F756EF6
:100C000064204C6576656C2073656E736F72206628
:100C10006F756E640053656E736F7220736C6F74C2
:100C200020616E6420747970653A00005EBCE261F8
:100C30003FDD83C29C7E20A3FD1F41009D23BE4655
:100C4000DB65F88C11AF32CA57E97400000A0B0259
:100C5000090C0D0E0807030401000000000000004D
:100C60000000000000000000000000000000000084
:100C70000000000000000012111000000000000041
:100C80000000000000000000000000000000000064
:100C9000000102102020080810204010204080028F
:100CA00001020108040201010204081020408080B2
:100CB0004020100804020180040201804020100836
:100CC000040201080402010102040810204080010E
:100CD00002040810204080050505050705080808DE
:100CE00008020202020A0A080804040404010101BD
:100CF00001010101010303030303030303040707C5
:100D0000070C0C0C0C0C0C0C0C0202020206060662
:100D100006060606060B0B0B0B0B0B0B0B0000203D
:100D2000002300260029002C002F003200000100C3
:100D30000003010601090100002200250028002B04
:100D4000002E003100340002010000050108010BF3
:100D50000100002100240027002A002D003000336C
:100D60000001010000040107010A014E414E494EF5
:100D7000495459494E46CDCCCC3D0AD7233C17B7F0
:100D8000D13877CC2B329595E6241FB14F0A00005D
:100D900020410000C84200401C4620BCBE4CCA1B7B
:100DA0000E5AAEC59D7400407A10F35A00A0724EE0
:100DB00018090010A5D4E80000E87648170000E400
:100DC0000B54020000CA9A3B000000E1F505000048
:100DD00080969800000040420F000000A0860100AD
:100DE0000000102700000000E8030000000064007D
:100DF000000000000A0000000000010000000000E8
:100E00002C76D888DC674F0823DFC1DFAE59E1B10B
:100E1000B796E5E3E453C63AE651997696E8E6C21A
:100E20008426EB898C9B62ED407C6FFCEFBC9C9F21
:100E300040F2BAA56FA5F490055A2AF75C936B6C43
:100E4000F9676DC11BFCE0E40D47FEF520E6B50037
:100E5000D0ED902E0300943577050080841E0800A5
:100E600000204E0A000000C80C333333330F986E55
:100E700012831141EF8D2114893BE65516CFFEE612
:100E8000DB18D1844B381BF77C1D901DA4BBE424D8
:100E9000203284725E228100C9F124ECA1E53D2755
:100EA000BF360E61C58570861B879D3711241FBE16
:100EB000CFEFD1E2DEBFCDBF00E00CBF1AE0A0E073
:100EC000B2E0ECEFF6E301E00BBF02C007900D9239
:100ED000AA37B107D9F720E1AAE7BAE001C01D920D
:100EE000AD37B207E1F71EE0CAEADEE000E006C077
:100EF00022970109FE010BBF0E94F093C03AD1076F
:100F000080E00807A9F70E941E8F0C946D9B78C89B
:100F1000CF92DF92EF92FF920F931F93E82FF92F5A
:100F200005C0015011092109310961F19081962311
:100F30009417B9F305C0015011092109310911F1C4
:100F4000908196239413F7CFC12CD12CE12CF12C56
:100F50000AC08FEFC81AD80AE80AF80A0C151D054E
:100F60002E053F0579F080818623841791F36C2D3F
:100F70007D2D8E2D9F2D1F910F91FF90EF90DF9073
:100F8000CF90089560E070E080E090E01F910F91B5
:100F9000FF90EF90DF90CF90089521EF39E0FC01B2
:100FA000318320830895089521EF39E0FC013183D6
:100FB00020830C942C8F2F923F924F925F926F92CE
:100FC0007F928F929F92AF92BF92CF92DF92EF92D9
:100FD000FF920F931F93CF93DF93CDB7DEB72E977A
:100FE0000FB6F894DEBF0FBECDBF8C017E876D8734
:100FF000DC014D915C91119712962D913C911397C4
:10100000421753072CF4942F852FA901292F382F2D
:10101000D801149660E070E0CB01E2E0F0E0ED84EE
:10102000FE84EE15FF0544F5CD90DD90C216D30683
:101030005CF44901AA2497FCA094BA2C680D791D90
:101040008A1D9B1D960116C04C155D055CF44A0176
:10105000AA2497FCA094BA2C680D791D8A1D9B1DAB
:10106000A60108C0EE24D7FCE094FE2C6C0D7D1D7B
:101070008E1D9F1D3196D3CF0E94C5906B017C01C0
:101080006D857E8562507109882777FD8095982F40
:101090000E94C5909B01AC01C701B6010E94F98F67
:1010A0006B017C012D853E85243131050CF4BFC0D8
:1010B0004801412C512C3201A12CB12CD4016D914D
:1010C0007D914D01882777FD8095982F0E94C590CE
:1010D000A70196010E942E8F9B01AC010E9459929C
:1010E0009B01AC01C301B2010E942F8F2B013C0177
:1010F000BFEFAB1ABB0AED85FE85AE16BF06F1F653
:10110000BF0161507109882777FD8095982F0E9453
:10111000C5909B01AC01C301B2010E94F98F0E94EE
:101120000C934B015C0120E030E040E85FE30E945B
:101130009A9118160CF07BC018870F83212C312C44
:101140001B821C821D821E821A821982AF81B88581
:101150008D919D91B887AF839C01442737FD4095C1
:10116000542F29873A874B875C87CA01B9010E94AF
:10117000C590A70196010E942E8F2B013C0120E013
:1011800030E0A9010E949A91181624F0C301B2011F
:10119000905802C0C301B201A50194010E94F58FCD
:1011A00087FF13C08B819C81AD81BE8129853A85E3
:1011B0004B855C85820F931FA41FB51F8B839C8377
:1011C000AD83BE833FEF231A330A49815A814F5FB3
:1011D0005F4F5A8349838D859E854817590709F0CB
:1011E000B5CF20E030E040EC5FE3C501B4010E94E0
:1011F00059924B015C0195E0291631040CF49CCF07
:101200006B817C818D819E810E94C5906B017C01E8
:10121000B101882777FD8095982F0E94C5909B018A
:10122000AC01C701B6010E94F98F6B017C01C701B7
:10123000B6012E960FB6F894DEBF0FBECDBFDF917C
:10124000CF911F910F91FF90EF90DF90CF90BF90C3
:10125000AF909F908F907F906F905F904F903F9056
:101260002F900895CF93DF93EC01FB01248135810A
:101270000E94698ECE01DF91CF91089526E00C94F3
:10128000D984DC01ED91FC910190F081E02D19945D
:10129000EF92FF920F931F93CF93DF931F92CDB7DF
:1012A000DEB77C01FC0100811181C80169830E94C5
:1012B0006C976981681719F0C8010E947497C7017B
:1012C0000F90DF91CF911F910F91FF90EF900895B4
:1012D000EF92FF920F931F93CF93DF931F921F9272
:1012E000CDB7DEB70DEB1AE08D5B9A407C01C701EC
:1012F000800F911FF80161918F019A838983CE013C
:101300000196C6DFFBE003331F0789F78DEB9AE0F8
:101310000F900F90DF91CF911F910F91FF90EF9061
:1013200008950F931F93CF93DF931F921F92CDB712
:10133000DEB704E01DE0F80160818EED93E09A8352
:101340008983CE010196A4DFF80161818FED93E0DE
:101350009A838983CE0101969BDFC8010F900F907D
:10136000DF91CF911F910F910895BF92CF92DF929D
:10137000EF92FF920F931F93CF93DF93CDB7DEB71A
:1013800062970FB6F894DEBF0FBECDBF6C017B0134
:101390008A0180919904882309F480C0809198047F
:1013A000882309F47BC077FF09C0E094F09440E003
:1013B0006E2D89EE9CE00E946E7F4CC040E060E0A4
:1013C00089EE9CE00E946E7F0E94CC8128EE33E083
:1013D00040E050E00E94BE93BA01A9012AE0CE018C
:1013E00001960E94788CBE016F5F7F4FCE010796F9
:1013F0000E94018C6BE378E0CE0107960E948C8DF1
:10140000BC01CE010D960E94018CCE0107960E9470
:10141000178BCE0101960E94178BBE01635F7F4F31
:1014200089EE9CE00E94BF87B98840E06B2D89EE71
:101430009CE00E946E7FE114F10411F4EB2C06C0D5
:1014400040E06E2D89EE9CE00E946E7FCE010D96ED
:101450000E94178BB60189EE9CE00E94BF876CEC5E
:1014600079E089EE9CE00E949C87F60164816E0D14
:1014700040E089EE9CE00E946E7F0E94CC816093E8
:10148000E50C7093E60C8093E70C9093E80CB801A0
:10149000882777FD8095982F0E94FB8162960FB672
:1014A000F894DEBF0FBECDBFDF91CF911F910F919A
:1014B000FF90EF90DF90CF90BF9008954F925F9292
:1014C0006F927F92AF92BF92CF92DF92EF92FF9294
:1014D0000F931F93CF93DF93CDB7DEB762970FB60D
:1014E000F894DEBF0FBECDBF6C017B015A01809125
:1014F0009904882309F498C080919804882309F4FA
:1015000093C00E94CC810091E50C1091E60C2091D3
:10151000E70C3091E80C40908C0450908D04609062
:101520008E0470908F04040D151D261D371D06179F
:1015300017072807390708F077C0F7FE0AC08701A8
:101540000095109540E0602F89EE9CE00E946E7F30
:1015500047C040E060E089EE9CE00E946E7F0E9400
:10156000CC8128EE33E040E050E00E94BE93BA0107
:10157000A9012AE0CE0101960E94788CBE016F5F1E
:101580007F4FCE0107960E94018C6BE378E0CE017D
:1015900007960E948C8DBC01CE010D960E94018C95
:1015A000CE0107960E94178BCE0101960E94178BE1
:1015B000BE01635F7F4F89EE9CE00E94BF8709896F
:1015C0001A89E114F10441F00E0D1F1D40E0602F57
:1015D00089EE9CE00E946E7FCE010D960E94178BD3
:1015E000B60189EE9CE00E94BF876BEB79E089EE43
:1015F0009CE00E949C87F6016481600F40E089EEC8
:101600009CE00E946E7F0E94CC816093E50C7093F9
:10161000E60C8093E70C9093E80CB501882777FDE2
:101620008095982F0E94FB8162960FB6F894DEBFDA
:101630000FBECDBFDF91CF911F910F91FF90EF9023
:10164000DF90CF90BF90AF907F906F905F904F9062
:1016500008958F929F92AF92BF92CF92DF92EF92B6
:10166000FF920F931F93CF93DF937C016B01EA01ED
:1016700080919904882309F474C080919804882388
:1016800009F46FC077FF1CC0C094D09441E06C2D6A
:1016900089EE9CE00E946E7FB70189EE9CE00E947B
:1016A000BF876AEA79E089EE9CE00E949C87F70197
:1016B00064816C0D41E089EE9CE00E946E7F3EC02B
:1016C0000E94CC8100918C0410918D0420918E0495
:1016D00030918F048090E10C9090E20CA090E30C8C
:1016E000B090E40C080D191D2A1D3B1D06171707A5
:1016F00028073907B0F541E06C2D89EE9CE00E9487
:101700006E7FB70189EE9CE00E94BF8769E979E0AE
:1017100089EE9CE00E949C87F70164816C0D41E09A
:1017200089EE9CE00E946E7F0E94CC816093E10C68
:101730007093E20C8093E30C9093E40CBE01882735
:1017400077FD8095982FDF91CF911F910F91FF909A
:10175000EF90DF90CF90BF90AF909F908F900C94C0
:10176000FB81DF91CF911F910F91FF90EF90DF9060
:10177000CF90BF90AF909F908F90089580919904E3
:10178000882379F080919804882359F0E091E90C3E
:10179000F091EA0C0190F081E02D60E089EE9CE090
:1017A0001994089580919904882379F08091980480
:1017B000882359F06FED89EE9CE00E94CE8761E3AB
:1017C00075E089EE9CE00C94CD870895CF93DF936C
:1017D000EC01809199048823A1F0809198048823DA
:1017E00081F06FED89EE9CE00E94CE878C819D8117
:1017F000892B39F0BE0189EE9CE0DF91CF910C94EA
:10180000BF87DF91CF91089580919904882301F1DA
:10181000809198048823E1F089EE9CE00E94697F22
:1018200040E060E089EE9CE00E946E7F69E879E02C
:1018300089EE9CE00E949C8741E060E089EE9CE09C
:101840000E946E7F69E779E089EE9CE00C949C87AA
:101850000895CF93DF93CDB7DEB72C970FB6F894EA
:10186000DEBF0FBECDBF66EA74E0CE0107960E94D0
:10187000828B6BED7CE0CE0107960E947B8DBC01D4
:10188000CE0101960E94018C48EC50E06FEF7FEF93
:10189000CE0101966ADDCE0101960E94178BCE0122
:1018A00007960E94178B6AEA74E0CE0107960E94A1
:1018B000828B65ED7CE0CE0107960E947B8DBC019A
:1018C000CE0101960E94018C40ED57E06FEF7FEF53
:1018D000CE010196BEDECE0101960E94178BCE018D
:1018E00007960E94178B8091020D9091030D01972E
:1018F00019F46AE679E002C06CE579E0CE01019660
:101900000E94208D48EC50E06FEF7FEFCE010196F2
:10191000D5DDCE0101960E94178B6CE479E0CE01F3
:1019200001960E94208D40ED57E06FEF7FEFCE01D2
:1019300001968FDECE0101960E94178B6CE379E051
:10194000CE0101960E94208D48EC50E06FEF7FEFB2
:10195000CE010196B3DDCE0101960E94178B6FE296
:1019600079E0CE0101960E94208D40ED57E06FEFA7
:101970007FEFCE0101966DDECE0101960E94178B9E
:1019800062E279E0CE0101960E94208D48EC50E0A1
:101990006FEF7FEFCE01019691DDCE0101960E949F
:1019A000178B67E179E0CE0101960E94208D40ED12
:1019B00057E06FEF7FEFCE0101964BDECE0101962F
:1019C0000E94178B6BE079E0CE0101960E94208D7A
:1019D00048EC50E06FEF7FEFCE0101966FDDCE0156
:1019E00001960E94178B6AEF78E0CE0101960E9463
:1019F000208D40ED57E06FEF7FEFCE01019629DE9D
:101A0000CE0101960E94178B8091020D9091030DDB
:101A1000039719F46FEE78E002C065EE78E0CE012E
:101A200001960E94208D48EC50E06FEF7FEFCE01D1
:101A3000019644DDCE0101960E94178B6AED78E095
:101A4000CE0101960E94208D40ED57E06FEF7FEFB1
:101A5000CE010196FEDDCE0101960E94178B6DEC42
:101A600078E0CE0101960E94208D48EC50E06FEFA7
:101A70007FEFCE01019622DDCE0101960E94178BE9
:101A80006EEB78E0CE0101960E94208D40ED57E08C
:101A90006FEF7FEFCE010196DCDDCE0101960E9453
:101AA000178B63EB78E0CE0101960E94208D48EC05
:101AB00050E06FEF7FEFCE01019600DDCE01019681
:101AC0000E94178B66EA78E0CE0101960E94208D75
:101AD00040ED57E06FEF7FEFCE010196BADDCE010A
:101AE00001960E94178B8091020D9091030D029731
:101AF00019F465E978E002C065E878E0CE01019666
:101B00000E94208D48EC50E06FEF7FEFCE010196F0
:101B1000D5DCCE0101960E94178B68E778E0CE01F4
:101B200001960E94208D40ED57E06FEF7FEFCE01D0
:101B300001968FDDCE0101960E94178B6CE678E04E
:101B4000CE0101960E94208D48EC50E06FEF7FEFB0
:101B5000CE010196B3DCCE0101960E94178B6CE595
:101B600078E0CE0101960E94208D40ED57E06FEFA6
:101B70007FEFCE0101966DDDCE0101960E94178B9D
:101B800061E578E0CE0101960E94208D48EC50E09E
:101B90006FEF7FEFCE01019691DCCE0101960E949E
:101BA000178B67E478E0CE0101960E94208D40ED0E
:101BB00057E06FEF7FEFCE0101964BDDCE0101962E
:101BC0000E94178B67E378E0CE0101960E94208D7A
:101BD00048EC50E06FEF7FEFCE0101966FDCCE0155
:101BE00001960E94178B6AE278E0CE0101960E946E
:101BF000208D40ED57E06FEF7FEFCE01019629DD9C
:101C0000CE0101960E94178B6EE178E0CE0101961D
:101C10000E94208D48EC50E06FEF7FEFCE010196DF
:101C20004DDCCE0101960E94178B6EE078E0CE016C
:101C300001960E94208D40ED57E06FEF7FEFCE01BF
:101C4000019607DDCE0101960E94178B2C960FB6E8
:101C5000F894DEBF0FBECDBFDF91CF9108954F92B4
:101C60005F926F927F928F929F92AF92BF92CF922C
:101C7000DF92EF92FF92CF93DF93CDB7DEB72C9731
:101C80000FB6F894DEBF0FBECDBFBEDD8BEF9BE07D
:101C90000E94157A2B013C018BEF9BE00E94A679F4
:101CA0004B015C01609138027091390280913A02D7
:101CB00090913B020E94C590AB01BC018BEF9BE071
:101CC0000E94B27B6B017C01C301B2010E94C590EE
:101CD00020E030E048EC52E40E94F98FAB01BC01F7
:101CE00022E0CE0101960E94A48CBE016F5F7F4F5F
:101CF00083ED9BE00E94098CCE0101960E94178B18
:101D00006FE878E083ED9BE00E94598D63ED7BE006
:101D100089ED9BE00E94EC8B6BE878E0CE010196A8
:101D20000E94828B63ED7BE0CE0101960E947B8D49
:101D3000BC0183ED9BE00E94EC8BCE0101960E94DA
:101D4000178B6FE476E08FED9BE00E941F8C21E003
:101D5000B501A401CE0101960E94A48CBE016F5F63
:101D60007F4F8FED9BE00E94538DCE0101960E9424
:101D7000178B6FEA74E08FED9BE00E94598D21E094
:101D8000B701A601CE0107960E94A48CBE01695F2F
:101D90007F4FCE0101960E94018C67EE75E0CE0167
:101DA00001960E948C8DBC018FED9BE00E94538DAB
:101DB000CE0101960E94178BCE0107960E94178BC9
:101DC00063ED7BE0CE0101960E94018C66EC74E02D
:101DD000CE0101960E948C8D6FED7BE00E947B8D81
:101DE000BC018FED9BE00E94EC8BCE0101960E941E
:101DF000178B69ED7BE0CE0101960E94018C4AE0D1
:101E000050E060E070E0CE010196AFDACE010196BD
:101E10000E94178B21E0B501A401CE0101960E941A
:101E2000A48CBE016F5F7F4F85EE9BE00E94098C02
:101E3000CE0101960E94178B65EE7BE0CE010196E4
:101E40000E94018C4AE050E06FEF7FEFCE010196D7
:101E500000DCCE0101960E94178B65EB74E0CE0189
:101E600001960E94828BCE010196B0DCCE010196D4
:101E70000E94178B21E0B701A601CE0107960E94B0
:101E8000A48CBE01695F7F4FCE0101960E94018C38
:101E900067EE75E0CE0101960E948C8DBC0185EE47
:101EA0009BE00E94EC8BCE0101960E94178BCE0125
:101EB00007960E94178B65EE7BE0CE0101960E948B
:101EC000018C4AE050E068EF7FEFCE010196C1DB64
:101ED000CE0101960E94178B8091D00B882331F0A0
:101EE00068E572E080E090E00E94FB812C960FB6DE
:101EF000F894DEBF0FBECDBFDF91CF91FF90EF9082
:101F0000DF90CF90BF90AF909F908F907F906F9019
:101F10005F904F900895CF93DF93EC018C819D816A
:101F2000892B61F0BE0180EA9EE00E94E887BE0135
:101F30008AED9FE0DF91CF910C94E887DF91CF91FC
:101F400008951F93CF93DF93CDB7DEB7A8970FB651
:101F5000F894DEBF0FBECDBF182F82E19CE00E9437
:101F6000617481110EC067E97AE0CE0101960E948A
:101F7000208DCE010196CFDFCE0101960E94178BF6
:101F8000A9C0BE016F5F7F4F82E19CE00E943F735A
:101F9000112309F499C06DE67AE080EA9EE00E9480
:101FA000D8876EE57AE080EA9EE00E949C87BE01B9
:101FB0006F5F7F4F80EA9EE00E94F8876FE47AE0CF
:101FC00080EA9EE00E949C874D855E856F857889BA
:101FD0002AE030E080EA9EE00E94D48860E47AE063
:101FE00080EA9EE00E949C8749895A896B897C8996
:101FF0002AE030E080EA9EE00E94D48861E37AE043
:1020000080EA9EE00E949C8720E030E040E251E4BC
:10201000698D7A8D8B8D9C8D0E945992AB01BC018C
:1020200022E030E080EA9EE00E94F08968EC74E0F3
:1020300080EA9EE00E94F88762E27AE080EA9EE011
:102040000E949C8720E030E040E251E46D8D7E8D5F
:102050008F8D98A10E945992AB01BC0122E030E023
:1020600080EA9EE00E94F08968EC74E080EA9EE0DD
:102070000E94F88763E17AE080EA9EE00E949C87F4
:1020800020E030E040E251E469A17AA18BA19CA15B
:102090000E945992AB01BC0122E030E080EA9EE050
:1020A0000E94F08968EC74E080EA9EE00E94F88764
:1020B0006EEE79E080EA9EE00E94D8876DE67AE0D5
:1020C00080EA9EE00E94F88764EF71E080E090E093
:1020D0000E94FB81A8960FB6F894DEBF0FBECDBF5D
:1020E000DF91CF911F9108954F925F926F927F92EF
:1020F0008F929F92AF92BF92CF92DF92EF92FF9218
:102100000F931F93CF93DF93CDB7DEB7CA54D10996
:102110000FB6F894DEBF0FBECDBF8C016DE67AE03E
:10212000CE01CD960E94828B6DE67AE0CE01C796F5
:102130000E94828BBE016F5F7F4F82E19CE00E9414
:10214000FF744D885E886F88788CC98CDA8CEB8C34
:10215000FC8C8D8D9E8DAF8DB8A12B968CAF9DAFD5
:10216000AEAFBFAF2B97C8010197039708F0E2C14C
:10217000A7019601C301B20190580E94A28F2BEDD6
:102180003FE049EC5FE30E942F8F209134023091B1
:10219000350240913602509137020E942F8F4B0139
:1021A0005C0120E030E0A9010E94F58F87FD09C0A5
:1021B0008092BF0B9092C00BA092C10BB092C20B49
:1021C00010C02BED3FE049EC50E4C501B4010E9482
:1021D0002F8F6093BF0B7093C00B8093C10B9093B4
:1021E000C20B8090BF0B9090C00BA090C10BB09021
:1021F000C20B2BED3FE049EC50E4C501B4010E9455
:102200009A91181684F42BED3FE049EC50E4C50197
:10221000B4010E942E8F6093BF0B7093C00B80930C
:10222000C10B9093C20B20E030E044E353E4609193
:10223000BF0B7091C00B8091C10B9091C20B0E949B
:1022400059922BED3FE049E450E40E94F98F6093EE
:10225000BB0B7093BC0B8093BD0B9093BE0B0E9485
:1022600092904AE0CE018B960E944D8C6CEC74E00B
:10227000CE0185960E94828BBE01655D7F4FCE01A7
:1022800085960E947B8D66ED74E00E948C8DBC016A
:1022900085EE9BE00E94EC8BCE0185960E94178B09
:1022A000CE018B960E94178B8090BB0B9090BC0B3D
:1022B000A090BD0BB090BE0B20E030E044EB52E4A8
:1022C000C501B4010E94F58F181694F020E030E0AB
:1022D00040E05FE3C501B4010E942F8F0E949290FD
:1022E0004AE0CE018B960E944D8C6DED74E023C0C8
:1022F00020E030E044E353E4C501B4010E94F58FCF
:102300001816A4F1A501940160E070E884E393E459
:102310000E942E8F6093BB0B7093BC0B8093BD0B00
:102320009093BE0B0E9492904AE0CE018B960E9441
:102330004D8C60EE74E0CE0185960E94828BBE01CA
:10234000655D7F4FCE0185960E947B8DBC01CE01DD
:10235000CD960E94EC8BCE0185960E94178BCE0104
:102360008B960E94178B6DED78E063C020E030E023
:1023700047E853E4C501B4010E94F58F181604F133
:1023800020E030E044E353E4C501B4010E942E8F05
:1023900020E030E040E05FE30E942F8F6093BB0BB2
:1023A0007093BC0B8093BD0B9093BE0B0E949290D8
:1023B0004AE0CE018B960E944D8C60EE74E01FC007
:1023C000A501940160E070E084EB93E40E942E8FFD
:1023D00020E030E040E05FE30E942F8F6093BB0B72
:1023E0007093BC0B8093BD0B9093BE0B0E94929098
:1023F0004AE0CE018B960E944D8C6DED74E0CE01CB
:1024000085960E94828BBE01655D7F4FCE018596C9
:102410000E947B8DBC01CE01CD960E94EC8BCE013B
:1024200085960E94178BCE018B960E94178B63EEC8
:1024300074E0CE01C7960E941F8CBE01635C7F4F83
:10244000CE0185960E94018C4AE050E060E070E089
:10245000CE0185960E94B509CE0185960E94178B04
:102460000E94CC8120918C0430918D0440918E0487
:1024700050918F048090E50C9090E60CA090E70CB2
:10248000B090E80C280D391D4A1D5B1D2617370733
:102490004807590708F441C20E94CC810E94C390AA
:1024A0004B015C0160918C0470918D0480918E04CD
:1024B00090918F040E94C59020E030E040E85EE3F8
:1024C0000E94599227966CAF7DAF8EAF9FAF279732
:1024D0006091E50C7091E60C8091E70C9091E80C0E
:1024E0000E94C5909B01AC0127966CAD7DAD8EAD71
:1024F0009FAD27970E942F8F9B01AC01C501B401AE
:102500000E94F58F87FD09C266EC74E0CE018596C6
:102510000E94828BBE01695C7F4FCE0185960E942E
:102520007B8DBC01CE01CD960E94538DCE01859648
:102530000E94178BC8010297029708F0C8C120E0DB
:1025400030E040E251E4C301B2010E9459924B01D4
:102550005C0120E030E040E251E4C701B6010E9496
:1025600059926B017C0120E030E040E251E42B966F
:102570006CAD7DAD8EAD9FAD2B970E9459922B0116
:102580003C010E94CC812091330B3091340B40915F
:10259000350B5091360B621B730B840B950B0E940D
:1025A000C39020E030E04AE754E40E94F98FAB0189
:1025B000BC0123E0CE018B960E94A48C69EF74E0ED
:1025C000CE0185960E94828BBE01655D7F4FCE0154
:1025D00085960E947B8D6BE378E00E948C8DBC0118
:1025E00083ED9BE00E94EC8BCE0185960E94178BB9
:1025F000CE018B960E94178B63ED7BE0CE01859612
:102600000E94018C65EE7BE0CE0185960E947B8D59
:10261000BE01635C7F4F0E947B8DBC01CE01CD96D5
:102620000E94EC8BCE0185960E94178B65EE74E0BC
:102630008FED9BE00E941F8C21E0B501A401CE012B
:1026400085960E94A48CBE016B5D7F4F8FED9BE051
:102650000E94538DCE0185960E94178B21E0B30115
:10266000A201CE0185960E94A48C21E0B701A601AB
:10267000CE01C1960E94A48C66EC74E0CE018B96CC
:102680000E94828BBE016F5C7F4FCE018B960E94B1
:102690007B8D66EC74E00E948C8DBE016B5D7F4F7C
:1026A0000E947B8D60EF74E00E948C8DBC018FEDE9
:1026B0009BE00E94538DCE018B960E94178BCE011A
:1026C000C1960E94178BCE0185960E94178BA5019B
:1026D0009401C501B4010E9459924B015C01A7010C
:1026E0009601C701B6010E9459929B01AC01C50138
:1026F000B4010E942F8F6B017C01A3019201C301E1
:10270000B2010E9459929B01AC01C701B6010E941F
:102710002F8F0E940C936093B70B7093B80B80932C
:10272000B90B9093BA0B64EF74E08FED9BE00E94BD
:10273000598D4091B70B5091B80B6091B90B7091C6
:10274000BA0B21E0CE018B960E94A48CBE01655D80
:102750007F4FCE0185960E94018C69EC74E0CE011A
:1027600085960E948C8DBC0185EE9BE00E94EC8BCF
:10277000CE0185960E94178BCE018B960E94178BF7
:1027800065EE7BE08FED9BE00E94538DC090B70B10
:10279000D090B80BE090B90BF090BA0B20E030E08D
:1027A0004AE754E4C701B6010E949A9187FD29C007
:1027B00020E030E04AE754E4C701B6010E94F98FF7
:1027C000AB01BC0123E0CE018B960E94D28CBE01EE
:1027D000655D7F4FCE0185960E94018C6AEC74E0A6
:1027E000CE0185960E948C8DBC0185EE9BE00E94F7
:1027F000EC8BCE0185960E94178BCE018B960E94A2
:10280000178B20E030E64AE656E46091B70B7091F2
:10281000B80B8091B90B9091BA0B0E94F58FBE0155
:10282000635C7F4F87FF4FC0CE0185960E94018C6D
:1028300068EF74E0CE0185960E948C8D6FED7BE091
:102840000E947B8DBC018FED9BE00E94EC8BCE0142
:1028500085960E94178B0330110599F46FED7BE08C
:10286000CE0185960E94018CCE01859654DBCE0167
:1028700085960E94178B6DE67AE08FED9BE00E94B3
:102880001F8C6BEF74E0CE018B960E94828B65EEFD
:102890007BE0CE018B960E947B8DBC01CE0185969C
:1028A0000E94018C4AE050E06FEF7FEFCE018596E9
:1028B0000E94290BCE0185960E94178BCE018B9624
:1028C0000E94178B04C08FED9BE00E94EC8B6AE0A6
:1028D00070E080E090E00E94FB81CE01C7960E94EC
:1028E000178BCE01CD960E94178BC65BDF4F0FB6BC
:1028F000F894DEBF0FBECDBFDF91CF911F910F9136
:10290000FF90EF90DF90CF90BF90AF909F908F900F
:102910007F906F905F904F9008956DE67AE0CE01C2
:1029200085960E94828BCE0185960E94E60BCE0191
:1029300085960E94178BBE01695C7F4F89EE9CE0F3
:102940000E94BF87E1CD8F929F92AF92BF92CF92AC
:10295000DF92EF92FF920F931F93CF93DF9300D0FC
:1029600000D0CDB7DEB78C01C0900A02D0900B0228
:10297000E0900C02F0900D0220E030E040E450E4E2
:10298000C701B6010E949A9118166CF420E030E05D
:102990004AE754E4C701B6010E9459920E949290FE
:1029A0006B017C0106C080E3C82E85E7D82EE12CA0
:1029B000F12C0E94040C40E060E089EE9CE00E9453
:1029C0006E7F64E075E089EE9CE00E94CD8741E077
:1029D00060E089EE9CE00E946E7F65E175E089EE23
:1029E0009CE00E94CD8764E670E080E090E00E9469
:1029F000FB810E94CC816093330B7093340B8093E6
:102A0000350B9093360B0E94CC818090330B9090C5
:102A1000340BA090350BB090360BDC01CB0188193C
:102A20009909AA09BB098C159D05AE05BF055CF483
:102A3000C8015ADB0E94CC8164E170E080E090E044
:102A40000E94FB81E0CF0130110509F041C06FED1C
:102A50007BE089ED9BE00E94EC8B0E94040C69ED09
:102A60007BE0CE0101960E94018C4AE050E060E0DC
:102A700070E0CE0101960E94B509CE0101960E9438
:102A8000178B6DED79E0CE0101960E94208D4AE012
:102A900050E06FEF7FEFCE0101960E94290BCE012F
:102AA00001960E94178B6DE175E0CE0101960E94A0
:102AB000828B6FED7BE0CE0101960E947B8DBC0185
:102AC0008FED9BE00E94EC8BCE0101960E94178B4C
:102AD00026960FB6F894DEBF0FBECDBFDF91CF9123
:102AE0001F910F91FF90EF90DF90CF90BF90AF902C
:102AF0009F908F900895CF92DF92EF92FF92CF93A5
:102B0000DF9300D000D0CDB7DEB70E94040C6EE199
:102B100070E080E090E00E94FB818BEF9BE00E94E0
:102B2000A6796B017C0164E670E080E090E00E9491
:102B3000FB816FE476E08FED9BE00E941F8C21E02B
:102B4000B701A601CE0101960E94A48CBE016F5F61
:102B50007F4F8FED9BE00E94538DCE0101960E9426
:102B6000178B6FED7BE0CE0101960E94018C4AE04D
:102B700050E060E070E0CE0101960E94B509CE0100
:102B800001960E94178B0E94D20B60E375E08FEDD7
:102B90009BE00E94598DC092C70BD092C80BE09267
:102BA000C90BF092CA0B20E030E040EF51E4C701BE
:102BB000B6010E949A9187FD03C06AEC77E054C089
:102BC00020E030E040ED51E4C701B6010E949A9147
:102BD00087FD1FC06AEB77E0CE0101960E94208D31
:102BE0004AE050E06FEF7FEFCE0101960E94290B83
:102BF000CE0101960E94178B80919C04882331F0AE
:102C00006CED75E080E090E00E94FB816AEA77E07D
:102C10002BC020E030E040EB51E4C701B6010E9438
:102C20009A9187FD03C06CE977E01EC06DE877E0FC
:102C3000CE0101960E94208D4AE050E06FEF7FEFB9
:102C4000CE0101960E94290BCE0101960E94178B9E
:102C500080919C04882331F06CED75E080E090E079
:102C60000E94FB816FE777E0CE0101960E94208DE4
:102C70004AE050E06FEF7FEFCE0101960E94290BF2
:102C8000CE0101960E94178B6CE271E080E090E02B
:102C90000E94FB8180919C04882331F068EE73E0F0
:102CA00080E090E00E94FB8126960FB6F894DEBF8C
:102CB0000FBECDBFDF91CF91FF90EF90DF90CF900F
:102CC0000895CF92DF92EF92FF92CF93DF93CDB72B
:102CD000DEB72C970FB6F894DEBF0FBECDBF61E70D
:102CE00077E0CE0101960E94208D4AE050E06FEF20
:102CF0007FEFCE0101960E94290BCE0101960E9422
:102D0000178B60916E0470916F0483E49CE00E94C5
:102D1000605BE12CF12C64E670E080E090E00E94C2
:102D2000FB8160916E0470916F0483E49CE00E94CB
:102D3000605B2FEFE21AF20A23E0E216F1045CF383
:102D40002AE0E216F1041CF4892B29F703C0892B31
:102D500009F0D4C06091450C7091460C882777FD2E
:102D60008095982F0E94C5906B017C016093C70BE2
:102D70007093C80B8093C90B9093CA0B6091430C5E
:102D80007091440C882777FD8095982F0E94C590FC
:102D90006093C30B7093C40B8093C50B9093C60BC9
:102DA00021E0B701A601CE0107960E94A48C6FE432
:102DB00076E0CE0101960E94828BBE01695F7F4F53
:102DC000CE0101960E947B8DBC018FED9BE00E949D
:102DD000EC8BCE0101960E94178BCE0107960E94C4
:102DE000178B4091C30B5091C40B6091C50B709130
:102DF000C60B21E0CE0107960E94A48C63E375E028
:102E0000CE0101960E94828BBE01695F7F4FCE0189
:102E100001960E947B8DBC018FED9BE00E94538D3B
:102E2000CE0101960E94178BCE0107960E94178B48
:102E300069E276E08FED9BE00E94598D6DE67AE0C5
:102E4000CE0101960E94828B44E150E060E070E088
:102E5000CE0101960E94B509CE0101960E94178B02
:102E60006091C70B7091C80B8091C90B9091CA0BF0
:102E70000E9492904AE0CE0101960E944D8CBE01C4
:102E80006F5F7F4F89ED9BE00E94098CCE01019618
:102E90000E94178B40E066E089EE9CE00E946E7F06
:102EA00069ED7BE089EE9CE00E94BF876FED89EEC3
:102EB0009CE00E94CE8765EB74E089EE9CE00E9466
:102EC000CD876091C30B7091C40B8091C50B90911D
:102ED000C60B0E9492904AE050E089EE9CE00E946E
:102EE000B78869E276E089EE9CE00E94CD8764E6CF
:102EF00070E080E090E00E94FB8118C066E677E019
:102F0000CE0101960E94208D4AE050E060E070E022
:102F1000CE0101960E94B509CE0101960E94178B41
:102F200066E477E08FED9BE00E94008D2C960FB653
:102F3000F894DEBF0FBECDBFDF91CF91FF90EF9031
:102F4000DF90CF900895CF92DF92EF92FF92CF93D0
:102F5000DF93CDB7DEB72C970FB6F894DEBF0FBE68
:102F6000CDBF68E377E0CE0101960E94208D4CE250
:102F700051E06FEF7FEFCE0101960E94290BCE0149
:102F800001960E94178B60916E0470916F0483E428
:102F90009CE00E94605BE12CF12C64E670E080E034
:102FA00090E00E94FB8160916E0470916F0483E455
:102FB0009CE00E94605B2FEFE21AF20A23E0E21627
:102FC000F1045CF32AE0E216F1041CF4892B29F7E2
:102FD00003C0892B09F057C16091450C7091460CD4
:102FE000882777FD8095982F0E94C5906B017C0102
:102FF0006093C70B7093C80B8093C90B9093CA0B57
:103000006091430C7091440C882777FD8095982F30
:103010000E94C5906093C30B7093C40B8093C50B43
:103020009093C60B21E0B701A601CE0107960E943E
:10303000A48C6FE476E0CE0101960E94828BBE01E3
:10304000695F7F4FCE0101960E947B8DBC018FEDA1
:103050009BE00E94EC8BCE0101960E94178BCE0163
:1030600007960E94178B4091C30B5091C40B60913F
:10307000C50B7091C60B21E0CE0107960E94A48C6F
:1030800063E375E0CE0101960E94828BBE01695F09
:103090007F4FCE0101960E947B8DBC018FED9BE09E
:1030A0000E94538DCE0101960E94178BCE01079688
:1030B0000E94178B69E276E08FED9BE00E94598DAC
:1030C0006DE67AE0CE0101960E94828B44E150E0E9
:1030D00060E070E0CE0101960E94B509CE01019634
:1030E0000E94178B6091C70B7091C80B8091C90B20
:1030F0009091CA0B0E9492904AE0CE0101960E94E4
:103100004D8CBE016F5F7F4F89ED9BE00E94098C63
:10311000CE0101960E94178B40E066E089EE9CE0AC
:103120000E946E7F69ED7BE089EE9CE00E94BF8784
:103130006FED89EE9CE00E94CE8765EB74E089EE2E
:103140009CE00E94CD876091C30B7091C40B80916D
:10315000C50B9091C60B0E9492904AE050E089EE18
:103160009CE00E94B78869E276E089EE9CE00E94CC
:10317000CD8764E670E080E090E00E94FB818BEEFA
:103180009BE00E94088FC090C70BD090C80BE090C6
:10319000C90BF090CA0B20E030E040EF51E4C701CA
:1031A000B6010E949A9187FD03C069E277E054C09E
:1031B00020E030E040ED51E4C701B6010E949A9151
:1031C00087FD1FC069E177E0CE0101960E94208D46
:1031D0004AE050E06FEF7FEFCE0101960E94290B8D
:1031E000CE0101960E94178B80919C04882331F0B8
:1031F0006CED75E080E090E00E94FB8169E077E093
:103200002BC020E030E040EB51E4C701B6010E9442
:103210009A9187FD03C06BEF76E01EC06CEE76E0FE
:10322000CE0101960E94208D4AE050E06FEF7FEFC3
:10323000CE0101960E94290BCE0101960E94178BA8
:1032400080919C04882331F06CED75E080E090E083
:103250000E94FB816EED76E0CE0101960E94208DEA
:103260004AE050E06FEF7FEFCE0101960E94290BFC
:10327000CE0101960E94178B62E370E080E090E03F
:103280000E94FB8101C037DC2C960FB6F894DEBF9C
:103290000FBECDBFDF91CF91FF90EF90DF90CF9029
:1032A0000895CF92DF92EF92FF921F93CF93DF9317
:1032B000CDB7DEB7AA970FB6F894DEBF0FBECDBF6D
:1032C000182F882331F06DE67AE080EA9EE00E94B4
:1032D000F88787E49CE00E94C263BE016F5F7F4F66
:1032E00087E49CE00E946263CE010D967C0111236D
:1032F00021F167EC76E080EA9EE00E94D887FE012B
:1033000031966F01F60141915191619171916F0177
:1033100026E030E080EA9EE00E94F08966EC74E0EE
:1033200080EA9EE00E94CD87CE14DF0459F76DE657
:103330007AE080EA9EE00E94F88723E938E144E8D9
:103340005FE369817A818B819C810E9459926D87AC
:103350007E878F87988B22E430E645E85FE36D81B6
:103360007E818F8198850E945992698B7A8B8B8B95
:103370009C8B25E83BEE41E95FE369857A858B8587
:103380009C850E9459926D8B7E8B8F8B988FB70195
:1033900087E49CE00E944263112309F48FC0B701C7
:1033A00087E49CE00E9462636AEB76E080EA9EE03C
:1033B0000E94D8876E01F9E1CF0ED11CF70141912F
:1033C0005191619171917F0122E030E080EA9EE0AD
:1033D0000E94F08966EC74E080EA9EE00E94CD874E
:1033E000EC14FD0459F76DE67AE080EA9EE00E9455
:1033F000F8876E01F5E2CF0ED11C9601AE01495D52
:103400005F4FBE01675D7F4F87E49CE00E94A5642B
:103410006DEA76E080EA9EE00E949C8769A57AA525
:103420004AE050E080EA9EE00E94B78866EC74E0D3
:1034300080EA9EE00E94CD876FA178A54AE050E027
:1034400080EA9EE00E94B78866EC74E080EA9EE025
:103450000E94CD876DA17EA14AE050E080EA9EE007
:103460000E94B7886DE67AE080EA9EE00E94F887C5
:10347000B70187E49CE00E94E36464EA76E080EAB6
:103480009EE00E949C87F701419151916191719159
:103490007F012AE030E080EA9EE00E94F08966EC3D
:1034A00074E080EA9EE00E94CD87EC14FD0459F799
:1034B0006DE67AE080EA9EE00E94F88761E070E0C5
:1034C00087E49CE00E94D663112389F060E976E0EE
:1034D00080EA9EE00E949C8787E49CE00E942D6524
:1034E0004AE050E0BC0180EA9EE00E94BE8824E0F1
:1034F00030E043E050E062E070E087E49CE00E944E
:10350000E3631123E9F164E776E080EA9EE00E943C
:103510009C879E012B5D3F4FAE01495D5F4FBE0111
:10352000675D7F4F87E49CE00E943F6569A57AA5AF
:103530004AE050E080EA9EE00E94B78866EC74E0C2
:1035400080EA9EE00E94CD876FA178A54AE050E016
:1035500080EA9EE00E94B78866EC74E080EA9EE014
:103560000E94CD876DA17EA14AE050E080EA9EE0F6
:103570000E94B7886DE67AE080EA9EE00E94F887B4
:1035800065E070E087E49CE00E940064112389F00C
:1035900061E676E080EA9EE00E949C8787E49CE0FA
:1035A0000E9482654AE050E0BC0180EA9EE00E94F1
:1035B000BE8866E070E087E49CE00E940D64112301
:1035C00089F069E476E080EA9EE00E949C8787E4C7
:1035D0009CE00E9494654AE050E0BC0180EA9EE0D5
:1035E0000E94BE8867E070E087E49CE00E9410645F
:1035F000112389F063E376E080EA9EE00E949C87D5
:1036000087E49CE00E94A6654AE050E0BC0180EAA5
:103610009EE00E94BE8868E070E087E49CE00E9423
:103620001D64112389F06BE176E080EA9EE00E9440
:103630009C8787E49CE00E94B8654AE050E0BC01AA
:1036400080EA9EE00E94BE8869E070E087E49CE02A
:103650000E942A64112389F061E076E080EA9EE00E
:103660000E949C8787E49CE00E94CA654AE050E083
:10367000BC0180EA9EE00E94BE886AE070E087E4B8
:103680009CE00E943764112389F06BEE75E080EABC
:103690009EE00E949C8787E49CE00E94DC654AE0F3
:1036A00050E0BC0180EA9EE00E94BE886BE070E0C2
:1036B00087E49CE00E944464112389F062ED75E088
:1036C00080EA9EE00E949C8787E49CE00E94EE6571
:1036D0004AE050E0BC0180EA9EE00E94BE886CE0B7
:1036E00070E087E49CE00E945164112309F48FC0CC
:1036F0006AEB75E080EA9EE00E949C8787E49CE08C
:103700000E9400664AE050E0BC0180EA9EE00E9410
:10371000BE8863EA75E080EA9EE00E949C8787E4A9
:103720009CE00E942567682F70E04AE050E080EA44
:103730009EE00E94BE886CE875E080EA9EE00E94F0
:103740009C8787E49CE00E942967682F70E04AE02C
:1037500050E080EA9EE00E94BE8865E775E080EA5E
:103760009EE00E949C8787E49CE00E942D67682F62
:1037700070E04AE050E080EA9EE00E94BE886CE57E
:1037800075E080EA9EE00E949C8787E49CE00E94AE
:103790003167682F70E04AE050E080EA9EE00E94C6
:1037A000BE8863E475E080EA9EE00E949C8787E41F
:1037B0009CE00E943567682F70E04AE050E080EAA4
:1037C0009EE00E94BE886AE275E080EA9EE00E9468
:1037D0009C8787E49CE00E943967682F70E04AE08C
:1037E00050E080EA9EE00E94BE8869E175E080EAD0
:1037F0009EE00E949C8787E49CE00E943D67682FC2
:1038000070E04AE050E080EA9EE00E94BE8861E0FD
:1038100087E49CE00E94DA6661E087E49CE00E9415
:10382000DF6661E087E49CE00E94E466112391F08A
:1038300060E075E080EA9EE00E949C8787E49CE05F
:103840000E944167682F70E04AE050E080EA9EE005
:103850000E94BE8860E087E49CE00E94E466112339
:1038600091F066EE74E080EA9EE00E949C8787E417
:103870009CE00E944167682F70E04AE050E080EAD7
:103880009EE00E94BE8861E087E49CE00E94E966B9
:10389000112391F06AEC74E080EA9EE00E949C871C
:1038A00087E49CE00E944567682F70E04AE050E0A2
:1038B00080EA9EE00E94BE8860E087E49CE00E946F
:1038C000E966112391F06DEA74E080EA9EE00E94BF
:1038D0009C8787E49CE00E944567682F70E04AE07F
:1038E00050E080EA9EE00E94BE8861E087E49CE0B0
:1038F0000E94EE66112391F061E974E080EA9EE097
:103900000E949C8787E49CE00E944967682F70E0D2
:103910004AE050E080EA9EE00E94BE8860E087E4D2
:103920009CE00E94EE66112391F064E774E080EA67
:103930009EE00E949C8787E49CE00E944967682F74
:1039400070E04AE050E080EA9EE00E94BE8861E0BC
:1039500087E49CE00E94F366112391F068E574E02F
:1039600080EA9EE00E949C8787E49CE00E944D676D
:10397000682F70E04AE050E080EA9EE00E94BE8836
:1039800060E087E49CE00E94F366112391F06BE312
:1039900074E080EA9EE00E949C8787E49CE00E949D
:1039A0004D67682F70E04AE050E080EA9EE00E9498
:1039B000BE8861E087E49CE00E94BC6661E087E429
:1039C0009CE00E94C16661E087E49CE00E94C666BC
:1039D00060E087E49CE00E94CB6660E087E49CE0C6
:1039E0000E94D06660E087E49CE00E94D5661123C7
:1039F00009F490C063E274E080EA9EE00E949C8734
:103A000087E49CE00E945167682F70E04AE050E034
:103A100080EA9EE00E94BE8865E074E080EA9EE055
:103A20000E949C8787E49CE00E945567682F70E0A5
:103A30004AE050E080EA9EE00E94BE8867EE73E0B4
:103A400080EA9EE00E949C8787E49CE00E94596780
:103A5000682F70E04AE050E080EA9EE00E94BE8855
:103A60006EEC73E080EA9EE00E949C8787E49CE015
:103A70000E945D67682F70E04AE050E080EA9EE0B7
:103A80000E94BE8865EB73E080EA9EE00E949C87FE
:103A900087E49CE00E946167682F70E04AE050E094
:103AA00080EA9EE00E94BE886CE973E080EA9EE0B6
:103AB0000E949C8787E49CE00E946567682F70E005
:103AC0004AE050E080EA9EE00E94BE8869E873E028
:103AD00080EA9EE00E949C8787E49CE00E946967E0
:103AE000682F70E04AE050E080EA9EE00E94BE88C5
:103AF00064E773E080EA9EE00E949C8787E49CE094
:103B00000E946D67682F70E04AE050E080EA9EE016
:103B10000E94BE8860E087E49CE00E94F86640ED69
:103B20005FE069E470E487E49CE00E943B66112357
:103B300009F449C060E673E080EA9EE00E949C8739
:103B400087E49CE00E941266AB01BC0122E030E0F9
:103B500080EA9EE00E94F18969E473E080EA9EE0D9
:103B60000E949C8787E49CE00E9476664AE050E0D1
:103B7000682F80EA9EE00E94F08861E373E080EAAB
:103B80009EE00E949C8761E087E49CE00E94716750
:103B9000682F70E04AE050E080EA9EE00E94BE8814
:103BA00068E173E080EA9EE00E949C8761E087E420
:103BB0009CE00E947567682F70E04AE050E080EA60
:103BC0009EE00E94BE8841E061E087E49CE00E94A4
:103BD000FD66112399F060E073E080EA9EE00E94A8
:103BE0009C8761E087E49CE00E947967682F70E021
:103BF0004AE050E080EA9EE00E94BE8841E061E039
:103C000087E49CE00E94026760E087E49CE00E94F9
:103C1000B7661123B1F06DEE72E080EA9EE00E947B
:103C20009C8787E49CE00E942167682F70E04AE04F
:103C300050E080EA9EE00E94BE8887E49CE00E94FB
:103C40007D67AA960FB6F894DEBF0FBECDBFDF9199
:103C5000CF911F91FF90EF90DF90CF9008952F921A
:103C60003F924F925F926F927F928F929F92AF920C
:103C7000BF92CF92DF92EF92FF920F931F93CF9359
:103C8000DF93CDB7DEB7C554D1090FB6F894DEBFC8
:103C90000FBECDBF2B013C012DA33EA34FA358A7C0
:103CA0000E94CC8122966CAF7DAF8EAF9FAF2297E2
:103CB00020E9421621E052066104710434F020E943
:103CC000422E55245394612C712C8DA19EA1AFA13D
:103CD000B8A580319742A105B1052CF030E127E26B
:103CE00090E080E004C03DA12EA19FA188A5409155
:103CF000D00B411104C03DA32EA39FA388A72296F9
:103D00006CAD7DAD8EAD9FAD229728EE33E040E0E7
:103D100050E00E94BE9326962CAF3DAF4EAF5FAFF2
:103D20002697F1E0FDAB19A61AA61BA61CA68E01CC
:103D3000035F1F4F22273327A9012419350946099C
:103D4000570929AB3AAB4BAB5CAB29A53AA54BA5C0
:103D50005CA58DA19EA1AFA1B8A5281739074A0778
:103D60005B070CF035C369A57AA58BA59CA50E94BD
:103D7000C59020E030E04AE754E40E94F98FAB019F
:103D8000BC0123E0C8010E94A48CB80189ED9BE02E
:103D90000E94098CC8010E94178B8DA19EA1AFA122
:103DA000B8A50A97A105B10594F42AE026964CAD72
:103DB0005DAD6EAD7FAD2697C8010E94788CB801CD
:103DC00089ED9BE00E94098CC8010E94178BBE01FF
:103DD0006F5F7F4F87E49CE00E94E36469E375E0D6
:103DE0008FED9BE00E941F8CDE0111961D01C12CFE
:103DF000D12C7601F10181909190A190B1901F0199
:103E0000A5019401C501B4010E9459929B01AC0126
:103E1000C701B6010E942F8F6B017C0123E0B50121
:103E2000A401CE0143960E94D28CBE016D5E7F4FED
:103E3000C8010E94018C66EC74E0C8010E948C8D60
:103E4000BC018FED9BE00E94538DC8010E94178B2F
:103E5000CE0143960E94178B2016310659F6C701F2
:103E6000B6010E940C936B017C01FDE24F16F1E05C
:103E70005F066104710444F00E94040C40E060E0BD
:103E800089EE9CE00E946E7F23E0B701A601C80185
:103E90000E94A48C68EF74E0CE0143960E94828B4E
:103EA00069ED7BE0CE0143960E947B8D66E475E070
:103EB0000E948C8DB8010E947B8D6BE475E00E949E
:103EC0008C8DBC018FED9BE00E94538DCE014396FB
:103ED0000E94178BC8010E94178B2DEC3CEC4CE420
:103EE0005FE3C701B6010E949A9129813A814B8113
:103EF0005C812DA73EA74FA758AB18160CF0ACC19C
:103F00002AE939E949E95FE3C701B6010E94F58F63
:103F100087FFA2C13DA9332309F49EC189849A84F5
:103F2000AB84BC8420E030E0A901C501B4010E944B
:103F3000F58FCD80DE80EF80F884882309F12DA5F0
:103F40003EA54FA558A9CA01B9010E9459926EAB6E
:103F50007FAB88AF99AFA7019601C701B6010E9458
:103F600059929B01AC016EA97FA988AD99AD0E94C1
:103F70002F8F0E940C93A50194010E94A28F04C070
:103F80006BED7FE089EC9FE320EE3EE245E652E4F4
:103F90000E9459926EAB7FAB88AF99AF20E030E0C2
:103FA000A901C701B6010E94F58F882309F12DA54B
:103FB0003EA54FA558A9CA01B9010E9459926AAFFE
:103FC0007BAF8CAF9DAFA5019401C501B4010E94E8
:103FD00059929B01AC016AAD7BAD8CAD9DAD0E9449
:103FE0002F8F0E940C93A70196010E94A28F04C0FC
:103FF0006BED7FE089EC9FE320EE3EE245E652E484
:104000000E9459926AAF7BAF8CAF9DAF20E030E049
:10401000A9016DA57EA58FA598A90E94F58F88237B
:10402000F9F0A5019401C501B4010E9459924B0118
:104030005C01A7019601C701B6010E9459929B013C
:10404000AC01C501B4010E942F8F0E940C932DA5D5
:104050003EA54FA558A90E94A28F6B017C0108C004
:104060009BEDC92E9FE0D92E99ECE92E9FE3F92E06
:1040700069EF74E0C8010E94828B69ED7BE0C801A2
:104080000E947B8D6EE475E00E948C8DBC018FEDEB
:104090009BE00E94EC8BC8010E94178B69EF74E0D3
:1040A000C8010E94828B69ED7BE0C8010E947B8D74
:1040B00068E675E00E948C8DBC0189ED9BE00E9452
:1040C000EC8BC8010E94178B21E04EA95FA968AD57
:1040D00079ADC8010E94A48C21E04AAD5BAD6CAD06
:1040E0007DADCE0143960E94A48C20EE3EE245E6D3
:1040F00052E4C701B6010E945992AB01BC0121E014
:10410000CE014F960E94A48CBE01615E7F4FCE010E
:1041100049960E94018C66EC74E0CE0149960E949B
:104120008C8DBE016D5E7F4F0E947B8D66EC74E0CE
:104130000E948C8DB8010E947B8DBC0183ED9BE0B9
:104140000E94EC8BCE0149960E94178BCE014F96B0
:104150000E94178BCE0143960E94178BC8010E94C4
:10416000178B4DE2441641E054066104710474F467
:1041700069A57AA58BA59CA525E030E040E050E03C
:104180000E94BE93672B682B692BC1F569ED7BE01C
:10419000C8010E94018C45E050E06FEF7FEFC8013D
:1041A0000E945E0AC8010E94178B61E775E0C80192
:1041B0000E94828B45E050E061EF7FEFC8010E94D2
:1041C000B509C8010E94178B6DE67AE0C8010E940C
:1041D000828BC8010E94E60BC8010E94178B63ED19
:1041E0007BE0C8010E94018C45E050E060E070E097
:1041F000C8010E94290BC8010E94178B63ED7BE068
:104200008FED9BE00E94538D5FE1451651046104E0
:10421000710434F489A59AA5ABA5BCA5B7FD11C05E
:104220006FED7BE0C8010E94018CC8010E948B0FDA
:10423000C8010E94178B6DE67AE08FED9BE00E942B
:104240001F8CB201C30177FE04C069A97AA98BA9AA
:104250009CA90E94FB81A9C023E04DA55EA56FA586
:1042600078A9C8010E94A48C69EF74E0CE0143963E
:104270000E94828B69ED7BE0CE0143960E947B8D8C
:1042800063E775E00E948C8DB8010E947B8D6CE421
:1042900075E00E948C8DBC0189ED9BE00E94EC8B47
:1042A000CE0143960E94178BC8010E94178B498547
:1042B0005A856B857C8523E0C8010E94D28C4D8194
:1042C0005E816F81788523E0CE0149960E94D28C71
:1042D000BE01675E7F4FCE0143960E94018C68E766
:1042E00075E0CE0143960E948C8DB8010E947B8DB3
:1042F0006CE475E00E948C8DBC0183ED9BE00E9414
:10430000EC8BCE0143960E94178BCE0149960E94FA
:10431000178BC8010E94178B9DE2491691E0590640
:104320006104710474F469A57AA58BA59CA525E0A8
:1043300030E040E050E00E94BE93672B682B692B71
:10434000F1F469ED7BE0C8010E94018C4AE050E085
:104350006FEF7FEFC8010E945E0AC8010E94178BB1
:1043600063ED7BE0C8010E94018C4AE050E060E010
:1043700070E0C8010E94290BC8010E94178B6FEDE5
:104380007BE0C8010E94018CC8010E948B0FC8010C
:104390000E94178B6DE67AE08FED9BE00E941F8CE8
:1043A000C301B2010E94FB811DAA0E94CC819B0126
:1043B000AC0122968CAD9DADAEADBFAD2297281B52
:1043C000390B4A0B5B0B29A73AA74BA75CA7BDCCBF
:1043D00069ED7BE0CE010D960E94018C4AE050E031
:1043E0006FEF7FEFCE010D960E94B509CE010D96BD
:1043F0000E94178B9DA99923B1F161E775E0CE0169
:104400000D960E94828B45E050E061EF7FEFCE0178
:104410000D960E94B509CE010D960E94178B8091D2
:10442000D00B882391F065EE72E0CE010D960E94CC
:10443000208D45E050E060E070E0CE010D960E94D6
:10444000B509CE010D960E94178B6DE67AE0CE017C
:104450000D960E94828BCE010D960E94E60BCE0136
:104460000D960E94178B63ED7BE0CE010D960E94A6
:10447000018C4AE050E06FEF7FEFCE010D960E9475
:10448000290BCE010D960E94178BCB5BDF4F0FB629
:10449000F894DEBF0FBECDBFDF91CF911F910F917A
:1044A000FF90EF90DF90CF90BF90AF909F908F9054
:1044B0007F906F905F904F903F902F900895CF9294
:1044C000DF92EF92FF920F931F93CF93DF93CDB7BD
:1044D000DEB72C970FB6F894DEBF0FBECDBF80912C
:1044E000D00B811102C00E94040C8DE39FE00E945A
:1044F0003B8564E670E080E090E00E94FB8169EC1F
:1045000072E089ED9BE00E94008D69ED7BE0CE01B9
:1045100001960E94018C44E150E060E070E0CE0121
:1045200001960E94B509CE0101960E94178B6AEB95
:1045300072E089ED9BE00E94008D69ED7BE0CE0189
:1045400001960E94018C44E150E06FEF7FEFCE01B5
:1045500001960E94290BCE0101960E94178B60E004
:1045600070E08AEC9CE00E94EC7C6B017C0104E032
:1045700010E0A7019601C701B6010E944D93882360
:1045800009F43DC00150110909F011C16FEA72E050
:1045900089ED9BE00E94008D69ED7BE0CE010196E4
:1045A0000E94018C4AE050E060E070E0CE0101968C
:1045B0000E94B509CE0101960E94178B6BE775E04A
:1045C000CE0101960E94828B69ED7BE0CE010196BF
:1045D0000E947B8DBC018FED9BE00E94EC8BCE0195
:1045E00001960E94178B8091020D9091030D039705
:1045F00009F0CCC01092030D1092020DC7C021E04B
:10460000B701A601CE0107960E94A48C6DE875E063
:10461000CE0101960E94828BBE01695F7F4FCE0161
:1046200001960E947B8DBC018FED9BE00E94EC8B7C
:10463000CE0101960E94178BCE0107960E94178B20
:104640006FED7BE0CE0101960E94018C42E350E0C9
:104650006FEF7FEFCE0101960E94290BCE010196EC
:104660000E94178B0E94D20B60E375E08FED9BE0F8
:104670000E94598D60E070E08AEC9CE00E94EA7C28
:104680006B017C0104E010E0A7019601C701B601AF
:104690000E944D93882359F00150110909F096C0EA
:1046A0006DE67AE085EE9BE00E941F8C50C021E011
:1046B000B701A601CE0107960E94A48C6FE476E0B4
:1046C000CE0101960E94828BBE01695F7F4FCE01B1
:1046D00001960E947B8DBC0185EE9BE00E94EC8BD5
:1046E000CE0101960E94178BCE0107960E94178B70
:1046F00066EC74E0CE0101960E94828B65EE7BE051
:10470000CE0101960E947B8DBC0189ED9BE00E9449
:10471000EC8BCE0101960E94178B69ED7BE0CE01F8
:1047200001960E94018C4AE050E060E070E0CE010A
:1047300001960E945E0ACE0101960E94178B0E948C
:10474000D20B60E375E085EE9BE00E94598D65EE2B
:104750007BE0CE0101960E94018C66EC74E0CE01F4
:1047600001960E948C8D6FED7BE00E947B8DBC01D9
:104770008FED9BE00E94EC8BCE0101960E94178B7F
:1047800083E090E09093030D8093020D64E670E067
:1047900080E090E00E94FB818091D00B882329F17A
:1047A00060E273E080E090E00E94FB811EC064E65E
:1047B00070E080E090E00E94FB8160E070E08AECB5
:1047C0009CE00E94EC7C6B017C01D3CE68EC70E035
:1047D00080E090E00E94FB8160E070E08AEC9CE069
:1047E0000E94EA7C6B017C014FCF2C960FB6F894A7
:1047F000DEBF0FBECDBFDF91CF911F910F91FF9014
:10480000EF90DF90CF9008951F93CF93DF93182FF1
:10481000C7E6DBE0812F0E949182899399936CE334
:1048200070E080E090E00E94FB818BE0C73BD807FE
:1048300089F768E270E087E69BE00E94DB0720E0F2
:1048400030E040EA50E40E94599220E030E040E835
:104850005AE30E945992DF91CF911F9108954F9290
:104860005F926F927F928F929F92AF92BF92CF9200
:10487000DF92EF92FF920F931F93CF93DF93CDB709
:10488000DEB764970FB6F894DEBF0FBECDBF7C01D4
:104890008B0165EA72E089ED9BE00E94008D0E9429
:1048A000040C69ED7BE0CE0101960E94018C4AE088
:1048B00050E06FEF7FEFCE0101960E94B509CE0167
:1048C00001960E94178BC7019FDF698B7A8B8B8BB8
:1048D0009C8B40901A0250901B0260901C027090BA
:1048E0001D02A3019201609116027091170280913E
:1048F0001802909119020E942E8F4B015C0120E05A
:1049000030E0A9010E94F58F882309F451C0C090BE
:104910002202D0902302E0902402F090250220E0B1
:1049200030E0A901C701B6010E94F58F18160CF0FE
:104930003FC080911E0290911F02A0912002B09171
:1049400021028D879E87AF87B88B9C01AD01C7017F
:10495000B6010E94F58F882359F1A70196016D8554
:104960007E858F8598890E94F98F0E94E6916D87D8
:104970007E878F87988BA301920169897A898B89B9
:104980009C890E942E8FA50194010E94F98F2D858C
:104990003E854F8558890E9459920E9466909B01DE
:1049A000AC01C701B6010E9459926B017C0103C0A2
:1049B000C12CD12C760169ED7BE0CE0101960E94DD
:1049C000018C4AE050E060E070E0CE0101960E9468
:1049D000B509CE0101960E94178B20E030E64AEE21
:1049E00056E4C701B6010E949A9118163CF466E994
:1049F00075E08FED9BE00E941F8C44C001151105EE
:104A0000B9F421E0B701A601CE0107960E94A48C5B
:104A100065EA75E0CE0101960E94828BBE01695F56
:104A20007F4FCE0101960E947B8D69EA75E01BC025
:104A30000230110539F522E049895A896B897C8950
:104A4000CE0107960E94A48C65EA75E0CE0101961E
:104A50000E94828BBE01695F7F4FCE0101960E944A
:104A60007B8D6DEA75E00E948C8DBC018FED9BE023
:104A70000E94EC8BCE0101960E94178BCE01079607
:104A80000E94178B6FED7BE0CE0101960E94018C96
:104A90004AE050E06FEF7FEFCE0101960E94290BB4
:104AA000CE0101960E94178B64E670E080E090E0F2
:104AB0000E94FB818091D00B882331F060E273E08B
:104AC00080E090E00E94FB8164960FB6F894DEBF10
:104AD0000FBECDBFDF91CF911F910F91FF90EF904F
:104AE000DF90CF90BF90AF909F908F907F906F900E
:104AF0005F904F9008954F925F926F927F928F9246
:104B00009F92AF92BF92CF92DF92EF92FF92CF939C
:104B1000C82F8091920A81110DC00E94CC816093B0
:104B2000860A7093870A8093880A9093890A81E0A5
:104B30008093920A80918A0A81110DC00E94CC81D3
:104B40006093820A7093830A8093840A9093850A03
:104B500081E080938A0A1092660B1092650BE090B8
:104B6000650BF090660B88E2E816F1040CF08AC041
:104B70008C2F0E949182F701EE0FFF1FE959F44F2D
:104B80009183808368E270E087E69BE00E94DB0708
:104B900020E030E040EA50E40E94599220E030E00A
:104BA00040E85AE30E9459926B017C0160937E0AAF
:104BB00070937F0A8093800A9093810A40902A0222
:104BC00050902B0260902C0270902D02A301920154
:104BD000609126027091270280912802909129020B
:104BE0000E942E8F9B01AC0160E070E080EC90E4AD
:104BF0000E942E8F4B015C0120E030E0A9010E9451
:104C0000F58F20E030E040E650E4811105C0C70197
:104C1000B6010E9459921EC0C701B6010E94599266
:104C2000A30192010E942F8F20E030E040E850E481
:104C30000E942E8FA50194010E94F98F20E030E0A0
:104C400040EC50E40E94599220E030E040E850E40B
:104C50000E942F8F60937A0A70937B0A80937C0A5C
:104C600090937D0A64E170E080E090E00E94FB8117
:104C70008091650B9091660B01969093660B8093E3
:104C8000650B6DCF60917A0A70917B0A80917C0AE6
:104C900090917D0ACF91FF90EF90DF90CF90BF90E1
:104CA000AF909F908F907F906F905F904F900895FE
:104CB000CF92DF92EF92FF92CF93DF93CDB7DEB723
:104CC0002C970FB6F894DEBF0FBECDBF6CE972E033
:104CD00089ED9BE00E94008D69ED7BE0CE0101969D
:104CE0000E94018C4AE050E060E070E0CE01019645
:104CF0000E94B509CE0101960E94178B8091810216
:104D000090918202F8DE6B017C0120E030E0A90185
:104D10000E949A9187FD22C022E0B701A601CE0130
:104D200007960E94A48C6FEA75E0CE0101960E945E
:104D3000828BBE01695F7F4FCE0101960E947B8D01
:104D4000BC018FED9BE00E94EC8BCE0101960E948E
:104D5000178BCE0107960E94178B06C063EB75E098
:104D60008FED9BE00E941F8C6FED7BE0CE010196E2
:104D70000E94018C4AE050E06FEF7FEFCE01019678
:104D80000E94290BCE0101960E94178B2C960FB61C
:104D9000F894DEBF0FBECDBFDF91CF91FF90EF90B3
:104DA000DF90CF9008952F923F924F925F926F9233
:104DB0007F928F929F92AF92BF92CF92DF92EF92AB
:104DC000FF920F931F93CF93DF9300D01F92CDB725
:104DD000DEB76B017C015A8349835901FA012081B6
:104DE0003181428153810E94F58F181614F0F5012C
:104DF00083C010E00150104C000F111F000F111F55
:104E0000E981FA81E00FF11F2081318142815381D4
:104E1000C701B6010E949A9187FF6BC011E0612E15
:104E2000712C4301880C991C880C991CE981FA812A
:104E3000E80DF91D2080318042805380A20191014C
:104E4000C701B6010E949A91181614F41F5FE7CFAC
:104E5000A2019101C701B6010E94F58F8501080DDD
:104E6000191D811102C0F80147C0C3018150904C47
:104E7000880F991F880F991FA981BA81A80FB91FA0
:104E80002D913D914D915C9129833A834B835C83B5
:104E9000F501E80FF91F80809180A280B380C701DF
:104EA000B6010E942E8F6B017C01A5019401F801CF
:104EB00060817181828193810E942E8F9B01AC0160
:104EC000C701B6010E9459926B017C0129813A8188
:104ED0004B815C81C201B1010E942E8F9B01AC010C
:104EE000C701B6010E94F98FA50194010E942F8F7E
:104EF00007C0F501E00FF11F60817181828193810C
:104F00000F900F900F900F90DF91CF911F910F9105
:104F1000FF90EF90DF90CF90BF90AF909F908F90D9
:104F20007F906F905F904F903F902F900895CF9219
:104F3000DF92EF92FF921F93CF93DF93182FCAE077
:104F4000D0E0C12CD12C7601812F0E949182BC012E
:104F5000882777FD8095982F0E94C5909B01AC0112
:104F6000C701B6010E942F8F6B017C0162E370E0E4
:104F700080E090E00E94FB81219731F720E030E053
:104F800040E251E4C701B6010E94F98F20E030E011
:104F900040EA50E40E94599220E030E040E85AE3B1
:104FA0000E945992DF91CF911F91FF90EF90DF9077
:104FB000CF9008952F923F924F925F926F927F927F
:104FC0008F929F92AF92BF92CF92DF92EF92FF9219
:104FD0000F931F93CF93DF93CDB7DEB73A0118013C
:104FE0002901A50194010E94F98F4B015C0120E089
:104FF00030E040EC5FE3C201B1010E9459929B0195
:10500000AC01C501B4010E949A91181694F120E0F8
:1050100030E040E05FE3C701B6010E9459929B0176
:10502000AC01C501B4010E94F58F87FD22C0F301D8
:105030002481358146815781C501B4010E942E8F9C
:10504000F30120853185428553850E94F98FF30154
:1050500020813181428153810E942F8F9B01AC01BD
:1050600060E070E080E291E40E94BC920E94929025
:1050700003C06FEF7FEFCB01DF91CF911F910F91B5
:10508000FF90EF90DF90CF90BF90AF909F908F9068
:105090007F906F905F904F903F902F9008954F9228
:1050A0005F926F927F928F929F92AF92BF92CF92B8
:1050B000DF92EF92FF920F931F93CF93DF93CDB7C1
:1050C000DEB7A0970FB6F894DEBF0FBECDBF2FDFBF
:1050D000698F7A8F8B8F9C8F40904502509046024B
:1050E0006090470270904802C0904102D090420206
:1050F000E0904302F09044028090490290904A026E
:10510000A0904B02B0904C0289829A82AB82BC8202
:105110004D825E826F827886A7019601C301B2013B
:105120000E942E8F6D8F7E8F8F8F98A320913D02CE
:1051300030913E0240913F0250914002C501B401BE
:105140000E942E8F9B01AC016D8D7E8D8F8D98A15D
:105150000E94F98F69877A878B879C87812C912C95
:1051600078E0A72E71E4B72E93018201AE014F5F64
:105170005F4F698D7A8D8B8D9C8D1CDF6B017C015F
:105180000E94040C63E972E089ED9BE00E94008DAF
:1051900069ED7BE0CE010D960E94018C42E350E068
:1051A00060E070E0CE010D960E94B509CE010D962B
:1051B0000E94178B2AE0B701A601CE0143960E94F8
:1051C000788C62EC75E0CE010D960E94828BBE0158
:1051D0006D5E7F4FCE010D960E947B8D67EC75E072
:1051E0000E948C8DBC018FED9BE00E94EC8BCE0168
:1051F0000D960E94178BCE0143960E94178B6FED80
:105200007BE0CE010D960E94018C42E350E06FEFEF
:105210007FEFCE010D960E94290BCE010D960E94C4
:10522000178B8091D00B882331F060E273E080E02F
:1052300090E00E94FB81A0960FB6F894DEBF0FBEEF
:10524000CDBFDF91CF911F910F91FF90EF90DF9035
:10525000CF90BF90AF909F908F907F906F905F9016
:105260004F900895FC0120E030E0772767FD7095AE
:10527000AB0142505109DF01A81BB90BA417B507B8
:1052800024F4A1912A0F311DF6CFA9014E5B5F4F87
:10529000860F971FFC013297208130E0322F2227A2
:1052A00031968081280F311D81E04217530709F0A4
:1052B00080E008952F923F924F925F926F927F927B
:1052C0008F929F92AF92BF92CF92DF92EF92FF9216
:1052D0000F931F93CF93DF93CDB7DEB763970FB6CE
:1052E000F894DEBF0FBECDBF8B8B60E00E940A83B7
:1052F0008091D00B811105C08FE090E0A0E0B0E07C
:1053000004C082E090E0A0E0B0E08F87988BA98B8A
:10531000BA8B67ED75E08FED9BE00E941F8C6FEDFF
:105320007BE0CE0101960E94018C4AE050E06FEFD5
:105330007FEFCE0101960E94B509CE0101960E9431
:10534000178BC12CD12C7601312C1D861E86212C69
:1053500002E310E0412C512C32018B890E94918292
:10536000AA2797FDA095BA2F480E591E6A1E7B1ECC
:1053700065E070E080E090E00E94FB81015011093F
:1053800061F78090120290901302A0901402B090E6
:105390001502C301B2010E94C59020E030E040EA4E
:1053A00050E40E94599220E030E040E85AE30E9425
:1053B000599220E030E048E452E40E94F98FA501C0
:1053C00094010E942E8F20E030E040E751E40E94DB
:1053D00059922B013C01A50194016AE979E989E31D
:1053E00090E40E942E8F9B01AC01C301B2010E9488
:1053F000F98F20E030E0A9010E942F8F20E030E0FB
:1054000040E251E40E9459925B018C01232D3D85BD
:105410004E85522D0E949A91181624F43A2CBD867E
:105420000E87212E20E030E0A901B501C8010E94BD
:10543000F58F87FF04C0A12CB12C00E010E022E022
:10544000A501B801CE0107960E94A48CBE01695F38
:105450007F4FCE0101960E94018C64EE75E0CE0173
:1054600001960E948C8DBC0189ED9BE00E94EC8B23
:10547000CE0101960E94178BCE0107960E94178BD2
:1054800069ED7BE0CE0101960E94018C4AE050E07C
:1054900060E070E0CE0101960E94290BCE010196DA
:1054A0000E94178B0E94CC8180908C0490908D0478
:1054B000A0908E04B0908F040091E10C1091E20C4A
:1054C0002091E30C3091E40C800E911EA21EB31EBD
:1054D00086169706A806B90608F4DEC00E94CC819D
:1054E0000E94C3904B015C0160918C0470918D040B
:1054F00080918E0490918F040E94C59020E030E04E
:1055000040E85EE30E9459922B013C016091E10C5E
:105510007091E20C8091E30C9091E40C0E94C59094
:105520009B01AC01C301B2010E942F8F9B01AC0112
:10553000C501B4010E94F58F87FDAEC06CE370E039
:1055400080E090E00E94FB819FEFC91AD90AE90A26
:10555000F90A8F859889A989BA898C159D05AE05A8
:10556000BF050CF0F5CE64E670E080E090E00E94AC
:10557000FB810E94040C64E670E080E090E00E94F1
:10558000FB8169EE75E089ED9BE00E941F8C69ED5F
:105590007BE0CE0101960E94018C44E150E060E086
:1055A00070E0CE0101960E94B509CE0101960E94DD
:1055B000178B22E0432D5D856E85722DCE010796F7
:1055C0000E94A48CBE01695F7F4FCE0101960E94AC
:1055D000018C64EE75E0CE0101960E948C8DBC01B9
:1055E00089ED9BE00E94EC8BCE0101960E94178B07
:1055F000CE0107960E94178B69ED7BE0CE010196E4
:105600000E94018C42E350E06FEF7FEFCE010196E4
:105610000E94290BCE0101960E94178B0E94BE0B9F
:1056200062E370E080E090E00E94FB8161EF75E052
:10563000CE0101960E94828B69ED7BE0CE0101963E
:105640000E947B8D65EF75E00E948C8D6FED7BE095
:105650000E947B8DBC018FED9BE00E94EC8BCE0104
:1056600001960E94178B63960FB6F894DEBF0FBEAB
:10567000CDBFDF91CF911F910F91FF90EF90DF9001
:10568000CF90BF90AF909F908F907F906F905F90E2
:105690004F903F902F9008950E94BE0B4FCFFF92E6
:1056A0000F931F93CF93DF93F82E0AE010E0C0E032
:1056B000D0E08F2D0E949182C80FD91F65E070E065
:1056C00080E090E00E94FB810150110991F7CE012A
:1056D0006AE070E00E947593CB01DF91CF911F913A
:1056E0000F91FF9008950F931F93CF93DF93CDB742
:1056F000DEB72E970FB6F894DEBF0FBECDBF8D87F5
:105700009E870E94040C8D859E85C9DF8C0162E313
:1057100070E080E090E00E94FB81B801882777FD6F
:105720008095982F0E94C59020E030E040EA50E438
:105730000E94599220E030EC4FE754E40E94F98F28
:10574000AB01BC0123E0CE0107960E94A48C62EF5E
:1057500075E0CE0101960E94828BBE01695F7F4F8A
:10576000CE0101960E947B8D6BEF75E00E948C8DBF
:10577000BC018FED9BE00E94EC8BCE0101960E9454
:10578000178BCE0107960E94178B6EEF75E089ED9F
:105790009BE00E941F8C69ED7BE0CE0101960E9488
:1057A000018C4AE050E068E070E0CE0101960E9472
:1057B000B509CE0101960E94178B6FED7BE0CE01FB
:1057C00001960E94018C4AE050E06FEF7FEFCE011E
:1057D00001960E94290BCE0101960E94178B69ED5C
:1057E0007BE08FED9BE00E94538D8091D00B88234E
:1057F00031F060E273E080E090E00E94FB812E9641
:105800000FB6F894DEBF0FBECDBFDF91CF911F91D1
:105810000F910895CF93DF93CDB7DEB72C970FB6D6
:10582000F894DEBF0FBECDBF3ADF9093CC0B8093D0
:10583000CB0B62E370E080E090E00E94FB8160911E
:10584000CB0B7091CC0B4AE0CE0101960E944D8C9F
:10585000BE016F5F7F4F8FED9BE00E94098CCE01F0
:1058600001960E94178B8091410C9091420C892BDC
:1058700009F45FC06DE37CE0CE0107960E94018CC5
:10588000BE01695F7F4FCE0101960E94018C44E109
:1058900050E060E070E0CE0101960E94B509CE01B3
:1058A00001960E94178B66E076E0CE0101960E9479
:1058B000828B6FED7BE0CE0101960E947B8DBC0157
:1058C00089ED9BE00E94EC8BCE0101960E94178B24
:1058D00069ED7BE0CE0101960E94018C44E150E02D
:1058E0006FEF7FEFCE0101960E94290BCE0101964A
:1058F0000E94178BBE01695F7F4FCE0101960E9407
:10590000018C66EC74E0CE0101960E948C8D69EDED
:105910007BE00E947B8DBC018FED9BE00E94EC8BB5
:10592000CE0101960E94178BCE0107960E94178B1D
:1059300054C061E176E089ED9BE00E941F8C69ED27
:105940007BE0CE0101960E94018C44E150E060E0D2
:1059500070E0CE0101960E94B509CE0101960E9429
:10596000178B65E176E0CE0101960E94828B6FED88
:105970007BE0CE0101960E947B8DBC0189ED9BE00E
:105980000E94EC8BCE0101960E94178B69ED7BE0A3
:10599000CE0101960E94018C44E150E06FEF7FEF51
:1059A000CE0101960E94290BCE0101960E94178B11
:1059B00066E076E0CE0101960E94828B6FED7BE07F
:1059C000CE0101960E947B8DBC018FED9BE00E9471
:1059D000EC8BCE0101960E94178B8091D00B88230F
:1059E00031F060E273E080E090E00E94FB812C9651
:1059F0000FB6F894DEBF0FBECDBFDF91CF910895F3
:105A00000F931F93CF93DF93CDB7DEB72C970FB6CD
:105A1000F894DEBF0FBECDBF8C0181E00E948E8264
:105A200064E670E080E090E00E94FB810E94040C3C
:105A3000C80135DE60E074E0681B790B4AE0CE01F6
:105A400007960E944D8C65E176E0CE0101960E949A
:105A5000828BBE01695F7F4FCE0101960E947B8DD4
:105A6000BC018FED9BE00E94EC8BCE0101960E9461
:105A7000178BCE0107960E94178B40E066E089EEF7
:105A80009CE00E946E7F65ED76E0CE0101960E945B
:105A9000208D42E350E068E070E0CE0101960E9464
:105AA000B509CE0101960E94178B6FED7BE0CE0108
:105AB00001960E94018C42E350E06FEF7FEFCE0130
:105AC00001960E94290BCE0101960E94178B6CE172
:105AD00076E0CE0101960E94828B6FED7BE0CE01D5
:105AE00001960E947B8DBC018FED9BE00E94EC8BA8
:105AF000CE0101960E94178B8091D00B882331F044
:105B000060E273E080E090E00E94FB812C960FB68B
:105B1000F894DEBF0FBECDBFDF91CF911F910F91E3
:105B200008950F9390E0BBDDBC01882777FD809539
:105B3000982F0E94C5902DE038E643E55BE30E9474
:105B4000599206E021E532E049E652E02CD920E006
:105B500030E048EC52E40E94599220E030E048EAFC
:105B600051E40E94599220914D0230914E02409191
:105B70004F02509150020E94F98F0F910895CF92D9
:105B8000DF92EF92FF92CF93DF93CDB7DEB72C97E2
:105B90000FB6F894DEBF0FBECDBFC3DF6B017C0133
:105BA0006BE872E089ED9BE00E94008D69ED7BE07F
:105BB000CE0101960E94018C42E350E060E070E06B
:105BC000CE0101960E94B509CE0101960E94178B65
:105BD00022E0B701A601CE0107960E94A48C63ECD7
:105BE00075E0CE0101960E94828BBE01695F7F4FF6
:105BF000CE0101960E947B8D66E276E00E948C8D3C
:105C0000BC018FED9BE00E94EC8BCE0101960E94BF
:105C1000178BCE0107960E94178B6FED7BE0CE01AC
:105C200001960E94018C42E350E06FEF7FEFCE01BE
:105C300001960E94290BCE0101960E94178B80913C
:105C4000D00B882331F060E273E080E090E00E94A6
:105C5000FB812C960FB6F894DEBF0FBECDBFDF914F
:105C6000CF91FF90EF90DF90CF900895CF92DF9289
:105C7000EF92FF920F9390E012DDBC01882777FD31
:105C80008095982F0E94C5902DE038E643E55BE3B0
:105C90000E94599206E021E532E049E652E083D8BD
:105CA00020E030E048EC52E40E9459926B017C0104
:105CB00020E030E0A9010E94F58F181634F0C12CC5
:105CC000D12C48EAE42E41E4F42EC0924D02D09249
:105CD0004E02E0924F02F09250020F91FF90EF902F
:105CE000DF90CF9008959F92AF92BF92CF92DF92B4
:105CF000EF92FF920F931F93CF93DF935C01C0E568
:105D0000D4E00EE314E057EFE52E5AE0F52ECC2454
:105D1000C394D12C75E1972E80913C0490913D0461
:105D20008C159D050CF49DC081E0A816B10429F4E2
:105D3000F70180819181F80108C0F2E0AF16B1044B
:105D400031F4F80180819181F70191838083F8011A
:105D500080819181009739F48881998190936104C1
:105D60008093600422C08130910539F48881998143
:105D700090936F0480936E0418C08230910539F4BB
:105D80008881998190936D0480936C040EC0039771
:105D900061F48881998190936304809362046DE635
:105DA0007AE08DE39CE00E941F8CF80121913191F3
:105DB0008F012430310539F48881998190938202D2
:105DC0008093810228C02530310539F4888199817A
:105DD00090936B0480936A041EC02630310539F419
:105DE0008881998190936704809366041EC0273050
:105DF000310539F488819981909365048093640416
:105E000028C02A30310539F488819981909369043A
:105E1000809368041EC02531310539F48881998149
:105E2000909371048093700414C02B3031058CF072
:105E3000888199819093630480936204929EB0015B
:105E4000939E700D11246D577D4F8DE39CE00E9451
:105E50001F8CFFEFCF1ADF0A229682E0E80EF11CBA
:105E60005BCFDF91CF911F910F91FF90EF90DF906B
:105E7000CF90BF90AF909F90089581E08093980459
:105E800089EE9CE00C94AA7F89EE9CE00E94A47F9E
:105E90001092980408954F925F926F927F92AF9202
:105EA000BF92CF92DF92EF92FF920F931F93CF9307
:105EB000DF93CDB7DEB7EA970FB6F894DEBF0FBE1B
:105EC000CDBF182F6DE67AE0CE01C5960E94828B79
:105ED000612FCE0145960E94187EBE016B5E7F4FFA
:105EE000CE0101960E94475CCE0101960E94A65DFC
:105EF000CE0101960E943A5F6CE0CE0101960E94AD
:105F0000965ECE0101960E94505C082F10E003308F
:105F1000110509F453C16BE276E0CE01C5960E94EB
:105F20001F8C6DE67AE08FED9BE00E941F8CBE0116
:105F30006B5C7F4FCE0183960E94018C4AE050E05B
:105F400060E070E0CE0183960E94B509CE01839691
:105F50000E94178B41E060E089EE9CE00E946E7F1A
:105F60006FE476E0CE01C5960E941F8CEBE3AE2E67
:105F7000EBE0BE2ECC24C394D12CE12CF12CE01606
:105F8000F1060CF0E1C06E2DCE0101960E94C75FB4
:105F9000F50121913191419151915F010E942F8F23
:105FA0002B013C0120E030E04CEF52EC0E94F58FD9
:105FB00087FF25C04AE0B601CE0189960E944D8C2C
:105FC0006CE677E0CE0183960E94828BBE01675D0E
:105FD0007F4FCE0183960E947B8D65E376E00E9421
:105FE0008C8DBC018FED9BE00E94538DCE0183967A
:105FF0000E94178BCE0189960E94178B49C022E020
:10600000B301A201CE0183960E94A48C4AE0B6019E
:10601000CE018F960E944D8C6CE677E0CE0189967A
:106020000E94828BBE01615D7F4FCE0189960E94E6
:106030007B8D64E178E00E948C8DBE016D5D7F4FA9
:106040000E947B8DBC0183ED9BE00E94EC8BCE0116
:1060500089960E94178BCE018F960E94178BCE01D6
:1060600083960E94178B63ED7BE0CE0183960E949E
:10607000018C66EC74E0CE0183960E948C8DBC018D
:106080008FED9BE00E94538DCE0183960E94178B6B
:106090000130110559F4E114F10409F04EC06FED1F
:1060A0007BE0CE01C5960E94EC8B47C00230110503
:1060B00011F522E0B301A201CE0189960E94A48CC1
:1060C000BE01675D7F4FCE0183960E94018C66EC16
:1060D00074E0CE0183960E948C8DBC01CE01C596E2
:1060E0000E94538DCE0183960E94178BCE01899614
:1060F0000E94178B22C063ED7BE0CE0183960E9445
:10610000018C44E150E06FEF7FEFCE0183960E9457
:10611000290BCE0183960E94178B0E94D20B80918F
:106120009904882351F080919804882331F060ED20
:1061300077E080E090E00E94FB81FFEFEF1AFF0A1A
:106140008FEFC81AD80A1BCFCE01C5960E94AC8E1D
:1061500001151105C9F460E372E08FED9BE00E9428
:10616000008D61E476E0CE0183960E94828B4AE046
:1061700050E06FEF7FEFCE0183960E94290BCE0196
:1061800083960E94178BD6C0043011050CF0EBC02B
:10619000BE016B5C7F4FCE0183960E94018C4AE06A
:1061A00050E06FEF7FEFCE0183960E94290BCE0166
:1061B00083960E94178B0E94D20BD5C06CE476E0C8
:1061C000CE01C5960E941F8CBE016B5C7F4FCE0135
:1061D00083960E94018C4AE050E060E070E0CE01BE
:1061E00083960E94B509CE0183960E94178B6DE6B7
:1061F0007AE08FED9BE00E941F8C6FED7BE0CE017B
:10620000C5960E94EC8B00E010E0602FCE01019655
:106210000E94C75F6B017C0122E0AB01BC01CE0193
:106220000115110569F483960E94A48CBE016D5D71
:106230007F4F89EE9CE00E94BF87CE0183961BC0F2
:1062400089960E94A48CBE01675D7F4FCE01839624
:106250000E94018C66EC74E0CE0183960E948C8DC6
:10626000BC01CE01C5960E94538DCE0183960E943B
:10627000178BCE0189960E94178B22E0B701A601E9
:10628000CE0189960E94A48CBE01675D7F4FCE012E
:1062900083960E94018C66EC74E0CE0183960E9486
:1062A0008C8DBC018FED9BE00E94538DCE018396B7
:1062B0000E94178BCE0189960E94178B0F5F1F4F8C
:1062C0000330110509F0A1CFCE01C5960E94AC8E16
:1062D000BE016B5C7F4FCE0183960E94018C4AE029
:1062E00050E06FEF7FEFCE0183960E94290BCE0125
:1062F00083960E94178B0E94D20B8FED9BE00E9429
:10630000AC8E62E576E0CE0183960E94828B6FEDC3
:106310007BE0CE0183960E947B8D6CE576E00E9447
:106320008C8DBC018FED9BE00E94EC8BCE0183969F
:106330000E94178BCE01C5960E94178BEA960FB666
:10634000F894DEBF0FBECDBFDF91CF911F910F91AB
:10635000FF90EF90DF90CF90BF90AF907F906F90C5
:106360005F904F9008956CE576E08FED9BE00E9482
:10637000598DE0CF8F929F92AF92BF92CF92DF92D2
:10638000EF92FF920F931F93CF93DF93CDB7DEB7BA
:10639000A2970FB6F894DEBF0FBECDBF5C016A01B5
:1063A0007B01122F6CE172E080EA9EE00E949C87E4
:1063B0004AE050E0B50180EA9EE00E94B78866ECB2
:1063C00074E080EA9EE00E94CD8722E030E0B701D1
:1063D000A60180EA9EE00E94F189612FCE014596D8
:1063E0000E94187EBE016B5E7F4FCE0101960E9417
:1063F000475CCE0101960E94A65DCE0101960E94E7
:106400003A5F6CE0CE0101960E94965ECE01019645
:106410000E94505C082F10E00B30110514F00AE0C8
:1064200010E08BE5A816B10408F44FC09BE3892E59
:106430009BE0992EC12CD12C7601A12CB12CA01659
:10644000B106BCF46A2DCE0101960E94C75F9B0184
:10645000AC01F40161937193819391934F01C70152
:10646000B6010E942F8F6B017C01FFEFAF1ABF0AAC
:10647000E6CFB801882777FD8095982F0E94C590B8
:106480009B01AC01C701B6010E94F98F6B017C0131
:106490008BE3882E8BE0982EA12CB12CA016B10690
:1064A0000CF052C0F4012081318142815381C70137
:1064B000B6010E942E8FF4016193719381939193A1
:1064C0004F01FFEFAF1ABF0AE9CFA114B10439F4AD
:1064D000BBE38B2EBBE09B2EA12CB12C1DC00A155B
:1064E0001B050CF0850101501109602FCE010196AA
:1064F0000E94C75F9B01AC01000F111F000F111F0D
:10650000055C144FC701B6010E942E8FF80160830D
:1065100071838283938318C0A016B106ACF46A2DF0
:10652000CE0101960E94C75F9B01AC01C701B60175
:106530000E942E8FF40161937193819391934F0187
:10654000FFEFAF1ABF0AE8CFA2960FB6F894DEBFEE
:106550000FBECDBFDF91CF911F910F91FF90EF90B4
:10656000DF90CF90BF90AF909F908F90089560E0A4
:106570008DE30E94438382E090E00E94218261E0EB
:106580008DE30E9443838AE090E00E94218260E0D4
:106590008DE30E94438320E432E44FE050E061E069
:1065A0008EE30E94A0830E94C39020E030E048EC7C
:1065B00052E40E94F98F2091D10C3091D20C40917D
:1065C000D30C5091D40C0E94599220E030E44CE15D
:1065D00056E40E94F98F20E030E040E05FE30C9445
:1065E00059920895CF92DF92EF92FF92C0DF6B0134
:1065F0007C0120E030E040E050E40E949A911816BF
:106600001CF4B5DF6B017C0120E030E040E050E499
:10661000C701B6010E949A9118161CF4A8DF6B01FD
:106620007C0120E030E040E050E4C701B6010E9468
:106630009A9118161CF49BDF6B017C0120E030E07E
:1066400040E050E4C701B6010E949A9118162CF45C
:10665000FF90EF90DF90CF908ACFC701B601FF90F7
:10666000EF90DF90CF9008954F925F926F927F925C
:106670008F929F92AF92BF92CF92DF92EF92FF9252
:10668000CF93DF9300D01F92CDB7DEB7ABDF9B0176
:10669000AC0169833A834B835C830E94D8812B01D0
:1066A0003C016EE170E080E090E00E94FB819ADFA7
:1066B0006B017C010E94D8814B015C018418950814
:1066C000A608B70829813A814B815C8181ED881643
:1066D00087E09806A104B1040CF43DC0C701B601DF
:1066E0000E942E8F6B017C0120E030E0A9010E9406
:1066F0009A9118165CF426EA3BE944EC5BE3C70187
:10670000B6010E94F58F87FF0BC025C026EA3BE942
:1067100044EC5BEBC701B6010E949A911816DCF0BD
:10672000C501B40128EE33E040E050E00E94BE9382
:10673000CA01B9010E94C5904B015C0120E030E024
:106740004AE754E4C701B6010E945992A501940199
:106750000E94F98F03C060E070E0CB010F900F90B2
:106760000F900F90DF91CF91FF90EF90DF90CF903F
:10677000BF90AF909F908F907F906F905F904F9061
:10678000089523E333E948E853E40E94F98F20E0B9
:1067900030E040E85FE30E942F8F0E940C9326E6D2
:1067A00036EA45EA53E40E9459926093D10C709303
:1067B000D20C8093D30C9093D40C08954F925F9297
:1067C0006F927F928F929F92AF92BF92CF92DF9201
:1067D000EF92FF92CF93DF93CDB7DEB76C970FB6F2
:1067E000F894DEBF0FBECDBF6B017C010E94CC814F
:1067F0006D8B7E8B8F8B988F61E08DE30E940A8377
:1068000060E08EE30E940A838BEF9BE00E94A679F2
:106810006093CD0C7093CE0C8093CF0C9093D00CE2
:10682000B0DFE0DE6D877E878F87988B0E94D881EE
:10683000698B7A8B8B8B9C8B6AE070E080E090E0B8
:106840000E94FB816EEF71E08FED9BE00E94008D56
:1068500020E030E04AE754E4C701B6010E945992B3
:10686000698F7A8F8B8F9C8F412C512C3201C12CD8
:10687000D12C7601C701B6010E94C590298D3A8DB1
:106880004B8D5C8D0E94F58F87FF87C10E94CC8164
:106890002D893E894F89588D621B730B840B950B94
:1068A0000E94C39020E030E04AE754E40E94F98F50
:1068B000AB01BC0123E0CE0101960E94A48CBE0175
:1068C0006F5F7F4F89ED9BE00E94098CCE0101969E
:1068D0000E94178B87DE6B017C010E94D8814B01DF
:1068E0005C0189899A89AB89BC89881A990AAA0AA4
:1068F000BB0A91ED891697E09906A104B1040CF446
:1069000041C020E030E0A901C701B6010E949A9180
:1069100018165CF426EA3BE944EC5BE3C701B601D8
:106920000E94F58F87FF0BC02DC026EA3BE944EC9F
:106930005BEBC701B6010E949A9118161CF1C501C4
:10694000B40128EE33E040E050E00E94BE93CA015B
:10695000B9010E94C5904B015C012D853E854F8594
:106960005889C701B6010E942E8F20E030E04AE727
:1069700054E40E945992A50194010E94F98F4B01A1
:106980005C0103C0812C912C540169ED7BE0CE01A8
:1069900001960E94018C67E776E0CE0101960E9485
:1069A0008C8DBC0189ED9BE00E94EC8BCE010196A1
:1069B0000E94178B23E0B701A601CE0107960E9423
:1069C000A48CBE01695F7F4FCE0101960E94018CAD
:1069D0006EE676E0CE0101960E948C8DBC0183EDBF
:1069E0009BE00E94EC8BCE0101960E94178BCE019A
:1069F00007960E94178B22E0B501A401CE010196F3
:106A00000E94A48C69EF74E0CE0107960E94828BED
:106A100069ED7BE0CE0107960E947B8D61E776E011
:106A20000E948C8D63ED7BE00E947B8D61E876E0B7
:106A30000E948C8DBE016F5F7F4F0E947B8D65E74A
:106A400076E00E948C8DBC018FED9BE00E94538DFF
:106A5000CE0107960E94178BCE0101960E94178BDC
:106A600020E030E0A901C501B4010E949A9187FDA0
:106A700006C066EC74E083ED9BE00E94598D22E035
:106A8000B501A401CE0107960E94A48CBE01695FE6
:106A90007F4FCE0101960E94018C65E776E0CE0122
:106AA00001960E948C8DBC0183ED9BE00E94538D6A
:106AB000CE0101960E94178BCE0107960E94178B7C
:106AC0006FED7BE0CE0101960E94018CCE01019614
:106AD0000E948B0FCE0101960E94178BC301B20159
:106AE00025E030E040E050E00E94BE93672B682B29
:106AF000692B21F569E776E0CE0101960E94828B31
:106B000045E050E060E070E0CE0101960E94B509DA
:106B1000CE0101960E94178B63ED7BE0CE010196BA
:106B20000E94018C45E050E06FEF7FEFCE010196AF
:106B30000E94290BCE0101960E94178B6DE67AE028
:106B40008FED9BE00E941F8C65E070E080E090E09C
:106B50000E94FB810E94CC816B017C012D893E89C2
:106B60004F89588DC21AD30AE40AF50A3BDD6D87B6
:106B70007E878F87988B0E94D881698B7A8B8B8BCD
:106B80009C8B6AE070E080E090E00E94FB813FEF28
:106B9000431A530A630A730A6DCE60E08DE30E94C4
:106BA0000A836C960FB6F894DEBF0FBECDBFDF919F
:106BB000CF91FF90EF90DF90CF90BF90AF909F90DC
:106BC0008F907F906F905F904F900895CF93DF9359
:106BD000CDB7DEB72C970FB6F894DEBF0FBECDBF92
:106BE00061E08DE30E940A8360E08EE30E940A83E5
:106BF0008BEF9BE00E94A6796093CD0C7093CE0C36
:106C00008093CF0C9093D00CBCDDECDCAB01BC01CD
:106C100023E0CE0107960E94A48CBE01695F7F4FDE
:106C2000CE0101960E94018C67EE75E0CE010196BF
:106C30000E948C8DBC0189ED9BE00E94EC8BCE0103
:106C400001960E94178BCE0107960E94178B62E770
:106C500076E0CE0101960E94828B69ED7BE0CE0149
:106C600001960E947B8DBC018FED9BE00E94EC8B16
:106C7000CE0101960E94178BF7DCAB01BC0122E02C
:106C8000CE0107960E94A48CBE01695F7F4FCE01A2
:106C900001960E94018C65E776E0CE0101960E9484
:106CA0008C8DBC0183ED9BE00E94EC8BCE010196A4
:106CB0000E94178BCE0107960E94178B60E876E042
:106CC000CE0101960E94828B63ED7BE0CE0101969E
:106CD0000E947B8DBC018FED9BE00E94538DCE0105
:106CE00001960E94178B66EC74E0CE0101960E941B
:106CF000828B63ED7BE0CE0101960E947B8DBC010F
:106D000089ED9BE00E94538DCE0101960E94178B66
:106D100069E776E0CE0101960E94828B4AE050E05E
:106D200060E070E0CE0101960E94B509CE010196A7
:106D30000E94178B69ED7BE0CE0101960E94018CC9
:106D400045E050E06FEF7FEFCE0101960E94290BE6
:106D5000CE0101960E94178B64E876E08FED9BE0F0
:106D60000E94598D60E08DE30E940A832C960FB635
:106D7000F894DEBF0FBECDBFDF91CF9108958F9203
:106D80009F92AF92BF92CF92DF92EF92FF920F93BA
:106D90001F921F9283E08F9327E0822E36E0A32E6E
:106DA00045E0C42E54E0E52E00E021E042E06FE330
:106DB00089EE9CE00E94E68067E976E08BED9CE03E
:106DC0000E94828B6EE976E085ED9CE00E94828BCA
:106DD00020E141E168E18AEC9CE00E94027C04E051
:106DE00022E734E046E754E06AE774E08BE59CE094
:106DF0000E948E7587E49CE00E9425636DE67AE030
:106E00008DE39CE00E94828B8091660490916704E0
:106E100090933C0C80933B0C8090450290904602EE
:106E2000A0904702B0904802209141023091420266
:106E30004091430250914402C501B4010E942E8F3B
:106E40006B017C016093370C7093380C8093390C84
:106E500090933A0C6091490270914A0280914B02E2
:106E600090914C0260932B0C70932C0C80932D0C02
:106E700090932E0C80922F0C9092300CA092310C9B
:106E8000B092320C20913D0230913E0240913F027F
:106E9000509140020E942E8F9B01AC01C701B601A8
:106EA0000E94F98F6093330C7093340C8093350CEF
:106EB0009093360C4FEF5FEFBA0182E19CE00E94A5
:106EC0008C738BEF9BE00E9487786DE67AE081EF10
:106ED0009BE00E94828B6DE67AE08BEE9BE00E9445
:106EE000828B6DE67AE085EE9BE00E94828B6DE6F8
:106EF0007AE08FED9BE00E94828B6DE67AE089ED6F
:106F00009BE00E94828B6DE67AE083ED9BE00E941D
:106F1000828B0F900F900F9060913202709133022C
:106F20008CEB9AE00F91FF90EF90DF90CF90BF90A5
:106F3000AF909F908F900C94516983ED9BE00E94DD
:106F4000178B89ED9BE00E94178B8FED9BE00E94D1
:106F5000178B85EE9BE00E94178B8BEE9BE00E94C7
:106F6000178B81EF9BE00E94178B81EF99E0909344
:106F7000130C8093120C8DE39CE00E94178B85ED1F
:106F80009CE00E94178B8BED9CE00C94178BCF93A9
:106F9000DF9300D000D0CDB7DEB780919904811186
:106FA0003BC061E080919A040E94438320E042E06C
:106FB00060E189EE9CE00E946A8140E954E060E073
:106FC00089EE9CE00E94228081E0809399046FE426
:106FD00072E0CE0101960E94208D4AE050E060E010
:106FE00070E0CE0101960E94B509CE0101960E9483
:106FF000178B63E472E0CE0101960E94208D4AE077
:1070000050E060E070E0CE0101960E94290BCE01B5
:1070100001960E94178B0EC080919804882351F02E
:107020000E94442F60E080919A040E944383109252
:10703000990402C00E943D2F26960FB6F894DEBF39
:107040000FBECDBFDF91CF9108956F927F928F9247
:107050009F92AF92BF92CF92DF92EF92FF920F93E7
:107060001F93CF93DF93CDB7DEB7E8970FB6F894B1
:10707000DEBF0FBECDBF4B015C018DE39FE00E94E0
:107080003B8564E670E080E090E00E94FB8140E890
:1070900055E260E070E08DE39FE00E943E0964E607
:1070A00070E080E090E00E94FB816FE772E089ED84
:1070B0009BE00E94008D69ED7BE0CE0101960E946D
:1070C000018C42E350E06FEF7FEFCE0101960E940A
:1070D000B509CE0101960E94178B64E772E089ED35
:1070E0009BE00E94008D69ED7BE0CE0101960E943D
:1070F000018C42E350E06FEF7FEFCE0101960E94DA
:10710000290BCE0101960E94178B8091020D909160
:10711000030D8D7F712CC12CD12CE12CF12C00E0C2
:1071200010E0019709F459C0F2E46F2E0E94CC815F
:10713000681979098A099B09683B7B40810591059B
:1071400008F04BC08DE39FE00E94CC83892BF1F1C6
:107150004CED55E060E070E08DE39FE00E942F8AE7
:1071600068AE41E050E0BE01685C7F4F8DE39FE078
:107170000E94168B882351F14FE150E0BE016F5FF2
:107180007F4F8DE39FE00E94358A89818D34F1F431
:107190006FE1CE0101960E9432298823B9F00C815B
:1071A00010E0102F00278D81080F111DEE80F12CAB
:1071B000FE2CEE248F81E80EF11CC884D12CDC2C2F
:1071C000CC248985C80ED11C7724739462E370E0C7
:1071D00080E090E00E94FB81A9CF0E94CC816819D9
:1071E00079098A099B09683B7B408105910510F468
:1071F0007110C3C00E94040C69ED7BE0CE01809643
:107200000E94018C42E350E066E070E0CE0180967F
:107210000E94B509CE0180960E94178B772009F451
:10722000D1C082E090E09093030D8093020D4AE07C
:10723000B601CE0180960E944D8C4AE0B701CE0186
:1072400086960E944D8C4AE0B801CE01C2960E94FB
:107250004D8CBE016E5C7F4FCE018C960E94018CDE
:1072600068E279E0CE018C960E948C8DBE016A5D49
:107270007F4F0E947B8D68E279E00E948C8DBE0179
:10728000605E7F4F0E947B8DBC018FED9BE00E9472
:10729000EC8BCE018C960E94178BCE01C2960E9479
:1072A000178BCE0186960E94178BCE0180960E9486
:1072B000178B6FED7BE0CE0180960E94018C4AE037
:1072C00050E06FEF7FEFCE0180960E94290BCE0138
:1072D00080960E94178B66EA76E089EE9CE00E9419
:1072E000CD876CEA76E08FED9BE00E941F8C4AE030
:1072F000B601CE0180960E944D8C4AE0B701CE01C6
:1073000086960E944D8C4AE0B801CE01C2960E943A
:107310004D8CBE016E5C7F4FCE018C960E94018C1D
:1073200066EC74E0CE018C960E948C8DBE016A5D85
:107330007F4F0E947B8D66EC74E00E948C8DBE01B5
:10734000605E7F4F0E947B8D66EA76E00E948C8DA6
:10735000BC018FED9BE00E94538DCE018C960E9464
:10736000178BCE01C2960E94178BCE0186960E9483
:10737000178BCE0180960E94178B62E370E080E04D
:1073800090E00E94FB818DE39FE00E943B8562E3D9
:1073900070E080E090E00E94FB81E8960FB6F894E0
:1073A000DEBF0FBECDBFDF91CF911F910F91FF9038
:1073B000EF90DF90CF90BF90AF909F908F907F9095
:1073C0006F90089569E672E08FED9BE00E94008D5A
:1073D0006FED7BE0CE0180960E94018C4AE050E088
:1073E00060E070E0CE0180960E94290BCE0180966D
:1073F0000E94178B66E572E08FED9BE00E94008D86
:107400008091020D9091030D029709F0B6CF109272
:10741000030D1092020DB1CF7F928F929F92AF9287
:10742000BF92CF92DF92EF92FF920F931F93CF9371
:10743000DF9300D000D0CDB7DEB74C018DE39FE0E5
:107440000E943B8540E052EC61E070E08DE39FE0FC
:107450000E943E094CED55E060E070E08DE39FE056
:107460000E942F8A64E670E080E090E00E94FB8139
:10747000A12CB12C712CA814B9040CF051C065E0FA
:1074800070E080E090E00E94FB8100E010E0C12C01
:10749000D12C760171100FC08DE39FE00E94CC8348
:1074A000892B31F485E1C816D104E104F1041CF400
:1074B0000330110554F08FEFA81AB80A64E670E0A3
:1074C00080E090E00E94FB81D6CF8DE39FE00E9498
:1074D000CC83892B69F08DE39FE00E94E583E1E096
:1074E000F0E0EC0FFD1FE00FF11F80830F5F1F4FD7
:1074F00065E070E080E090E00E94FB8102301105C1
:107500004CF089818B3B31F4772473948A818A3AD9
:1075100009F0712C8FEFC81AD80AE80AF80ABACF16
:10752000872D26960FB6F894DEBF0FBECDBFDF9134
:10753000CF911F910F91FF90EF90DF90CF90BF9070
:10754000AF909F908F907F9008958F929F92AF926F
:10755000BF92CF92DF92EF92FF920F931F93CF9340
:10756000DF93CDB7DEB72C970FB6F894DEBF0FBE12
:10757000CDBF61E080919A040E940A8361E080910E
:107580009A040E94438320E042E060E189EE9CE09F
:107590000E946A8140E954E060E089EE9CE00E942C
:1075A00022800E943D2F8EED93E09093640B809398
:1075B000630B0E946C978093040D8FED93E00E9403
:1075C0006C978093050D8091040D9091050D181610
:1075D000190654F410929C04019731F41092050D91
:1075E0001092040D0E9491096CEB76E089EE9CE00C
:1075F0000E94CD8740E855E260E070E080EA9EE0BE
:107600000E943E0940E855E260E070E08AED9FE0AC
:107610000E943E0964E670E080E090E00E94FB81F9
:1076200080919C04882331F068EE73E080E090E064
:107630000E94FB8180EA9EE00E94E583182F82373A
:1076400009F42DC11092640B1092630B9DEBC92EAF
:107650009AE0D92EE12CF12CC7010E946C97D6013B
:107660008D936D01BFEFEB1AFB0AE6E7EE16F1040E
:1076700099F78091BD0A9091BE0AA091BF0AB0917E
:10768000C00A85369105A105B1050CF408C18093A7
:10769000380290933902A0933A02B0933B02809152
:1076A000C10A9091C20AA091C30AB091C40A809302
:1076B000340290933502A0933602B0933702809142
:1076C000C50A9091C60AA091C70AB091C80A8093D2
:1076D0002E0290932F02A0933002B093310269EDF5
:1076E0007AE0CE0101960E94828BBE016F5F7F4FD0
:1076F0008BED9CE00E94098CCE0101960E94178BB5
:107700008091C90A9091CA0AA091CB0AB091CC0A83
:107710008093220290932302A0932402B093250227
:107720008091CD0A9091CE0AA091CF0AB091D00A53
:1077300080931E0290931F02A0932002B093210217
:107740008091D10A9091D20AA091D30AB091D40A23
:1077500080931A0290931B02A0931C02B0931D0207
:107760008091D50A9091D60AA091D70AB091D80AF3
:107770008093160290931702A0931802B0931902F7
:107780008091E10A9091E20AA091E30AB091E40AA3
:107790008093450290934602A0934702B09348021B
:1077A0008091E50A9091E60AA091E70AB091E80A73
:1077B0008093410290934202A0934302B09344020B
:1077C0008091E90A9091EA0AA091EB0AB091EC0A43
:1077D0008093490290934A02A0934B02B0934C02CB
:1077E0008091ED0A9091EE0AA091EF0AB091F00A13
:1077F00080933D0290933E02A0933F02B0934002DB
:107800008091F10A9091F20AA091F30AB091F40AE2
:1078100080934D0290934E02A0934F02B09350027A
:10782000C090070BD090080BE090090BF0900A0B6A
:10783000A7019601C701B6010E944D93811108C0AE
:10784000C0921202D0921302E0921402F09215023A
:107850000BE0A02E0BE0B02E8BE3882E8BE0982E51
:10786000D501CD90DD90ED90FD905D01A7019601D1
:10787000C701B6010E944D93811105C0F401C08279
:10788000D182E282F382F4E08F0E911C83E3A8168A
:107890008BE0B80629F781E090E00E94732E0EE895
:1078A000010F023070F08091BD0A9091BE0AA09144
:1078B000BF0AB091C00A85369105A105B1050CF04B
:1078C00032C18091380290913902A0913A02B09170
:1078D0003B028093BD0A9093BE0AA093BF0AB09367
:1078E000C00A8091340290913502A0913602B09185
:1078F00037028093C10A9093C20AA093C30AB0933F
:10790000C40A80912E0290912F02A0913002B09172
:1079100031028093C50A9093C60AA093C70AB09318
:10792000C80A123751F420E030E048E050E069ED39
:107930007AE08BED9CE00E94E88D8091220290918C
:107940002302A0912402B09125028093C90A90934A
:10795000CA0AA093CB0AB093CC0A80911E029091E0
:107960001F02A0912002B09121028093CD0A909332
:10797000CE0AA093CF0AB093D00A80911A029091B8
:107980001B02A0911C02B0911D028093D10A90931A
:10799000D20AA093D30AB093D40A80911602909190
:1079A0001702A0911802B09119028093D50A909302
:1079B000D60AA093D70AB093D80A80914502909135
:1079C0004602A0914702B09148028093E10A909349
:1079D000E20AA093E30AB093E40A809141029091F5
:1079E0004202A0914302B09144028093E50A909331
:1079F000E60AA093E70AB093E80A809149029091C1
:107A00004A02A0914B02B0914C028093E90A9093F4
:107A1000EA0AA093EB0AB093EC0A80913D029091A0
:107A20003E02A0913F02B09140028093ED0A9093F4
:107A3000EE0AA093EF0AB093F00A80914D02909164
:107A40004E02A0914F02B09150028093F10A9093A0
:107A5000F20AA093F30AB093F40A80911202909173
:107A60001302A0911402B09115028093070B90931A
:107A7000080BA093090BB0930A0BEBE3FBE02BE0A0
:107A80003BE04191519161917191D9014D935D9389
:107A90006D937D939D01BBE0E336FB0791F765E1B4
:107AA0007CE080EA9EE00E94D887A5EFAA2EAAE09B
:107AB000BA2EBCE3CB2EB4E0DB2EE12CF12C80916E
:107AC0003C0490913D048E159F051CF14601F60182
:107AD000819191916F01D5018D939D935D014AE054
:107AE00050E0B70180EA9EE00E94B7886DEC76E036
:107AF00080EA9EE00E94CD87F401608171814AE0B6
:107B000050E080EA9EE00E94BE88FFEFEF1AFF0A75
:107B1000D6CF023040F41092640B1092630B80E0D9
:107B200090E00E94680964E670E080E090E00E94C6
:107B3000FB818CEB9AE00E94566962ED76E0CE0103
:107B400001960E94828B4AE050E06FEF7FEFCE01FA
:107B500001960E94B509CE0101960E94178B66EA34
:107B600074E0CE0107960E94828B6BED7CE0CE0123
:107B700007960E947B8DBC01CE0101960E94018C6C
:107B80004AE050E06FEF7FEFCE0101960E94290B93
:107B9000CE0101960E94178BCE0107960E94178B8B
:107BA00060ED76E0CE0107960E94828B6BED7CE063
:107BB000CE0107960E947B8D62EE76E00E948C8D4E
:107BC000BC01CE0101960E94018CCE0101960E945B
:107BD0008B0FCE0101960E94178BCE0107960E9453
:107BE000178B64E670E080E090E00E94FB8186E005
:107BF0009DE00E94856064E670E080E090E00E9475
:107C0000FB8163E270E086E09DE00E94986061E0A5
:107C100070E086E09DE00E94410986E09DE00E94C0
:107C20000C6183E090E09093030D8093020D60E07F
:107C300070E08AEC9CE00E94EC7C6B017C0162E3CA
:107C400070E080E090E00E94FB81A7019601C701EF
:107C5000B6010E944D93882309F465C060E070E08E
:107C60008AEC9CE00E94EA7C6B017C0162E370E09C
:107C700080E090E00E94FB81A7019601C701B60158
:107C80000E944D93882309F44EC081E090E09093C8
:107C9000030D8093020D40E052EC61E070E08DE353
:107CA0009FE00E943E0964E670E080E090E00E9460
:107CB000FB8182E090E0B0DB882339F06CEF7BE061
:107CC00080EA9EE00E94D8872EC01092030D109289
:107CD000020D8DE39FE00E943B8564E670E080E04A
:107CE00090E00E94FB8140E855E260E070E08DE3A7
:107CF0009FE00E943E098DE39FE00E94CC83892B88
:107D000091F062EE7BE080EA9EE00E94D88782E0FC
:107D100090E09093030D8093020D64E670E080E0A4
:107D200090E00E94FB818091020D9091030D0397DA
:107D300031F46DEC7BE080EA9EE00E94D88763E03E
:107D40008BEF9BE00E944779811111C067EA7BE0CD
:107D5000CE0101960E94208DCE0101960E948B0FCC
:107D6000CE0101960E94178B10923C0293C063E9EA
:107D70007BE08FED9BE00E94008D40E050E0BA0177
:107D80008BEF9BE00E94687B0E94C59020E030E072
:107D900048EC52E40E94F98FAB01BC0122E0CE0115
:107DA00007960E94A48CBE01695F7F4FCE010196A9
:107DB0000E94018C6FE878E0CE0101960E948C8DC4
:107DC000BC018FED9BE00E94538DCE0101960E9475
:107DD000178BCE0107960E94178B6FED7BE080EA30
:107DE0009EE00E94E8876CE77BE08FED9BE00E94BD
:107DF000008D609138027091390280913A02909121
:107E00003B020E94C59020E030E048EC52E40E9422
:107E1000F98FAB01BC0122E0CE0107960E94A48C31
:107E2000BE01695F7F4FCE0101960E94018C6FE811
:107E300078E0CE0101960E948C8DBC018FED9BE015
:107E40000E94538DCE0101960E94178BCE0107969A
:107E50000E94178B6FED7BE080EA9EE00E94E8872E
:107E6000113629F481E00E94511981E011C080EAA5
:107E70009EE00E94E583182F64E670E080E090E0C9
:107E80000E94FB81113671F380E00E94511980E05D
:107E90000E94A10F64E670E080E090E00E94FB8108
:107EA00080919C04882331F068EE73E080E090E0DC
:107EB0000E94FB816EE477E08BEE9BE00E941F8CBA
:107EC00082E090E09093CE0B8093CD0B80919C0448
:107ED00081110E94A3172C960FB6F894DEBF0FBE37
:107EE000CDBFDF91CF911F910F91FF90EF90DF9069
:107EF000CF90BF90AF909F908F9008952F923F9218
:107F00004F925F926F927F928F929F92AF92BF92A9
:107F1000CF92DF92EF92FF920F931F93CF93DF9355
:107F2000CDB7DEB72B970FB6F894DEBF0FBECDBF2F
:107F30001C018BEB8F838AEA888781E0898784E63E
:107F4000829D9001839D300D11243B872A87E12C6F
:107F5000F12CC12CD12C812C912C5401C214D304AE
:107F600094F1C501B4010E94C59020E030E040E2E8
:107F700051E40E94F98F6B017C01B101882777FDE4
:107F80008095982F0E94C5909B01AC01C701B60156
:107F90000E94F98F2B960FB6F894DEBF0FBECDBFAF
:107FA000DF91CF911F910F91FF90EF90DF90CF90D5
:107FB000BF90AF909F908F907F906F905F904F9009
:107FC0003F902F9008952A853B85E216F3064CF6E4
:107FD000C7016AE070E00E948993892B79F4E091EF
:107FE0003D0FF0913E0F0280F381E02D43E050E021
:107FF000BE01695F7F4F8DE39FE0199565E070E0FA
:1080000080E090E00E94FB813FEFE31AF30A00E07A
:1080100010E0412C512C32018DE39FE00E94CC8373
:10802000892B39F424E042165104610471040CF0E8
:1080300095CF063011050CF091CF8DE39FE00E94A3
:10804000CC83892B69F08DE39FE00E94E583E1E01A
:10805000F0E0EC0FFD1FE00FF11F80830F5F1F4F5B
:1080600065E070E080E090E00E94FB810630110541
:1080700001F599818F8198131CC09A818885981386
:1080800018C09B818985981314C02C818D8190E044
:10809000A0E0B0E0BA2FA92F982F8827820F911D5A
:1080A000A11DB11D880E991EAA1EBB1E8FEFC81AF6
:1080B000D80A9FEF491A590A690A790AADCFCF92B7
:1080C000DF92EF92FF92CF93DF93CDB7DEB72C977D
:1080D0000FB6F894DEBF0FBECDBF8DE39FE00E94C8
:1080E0003B8540E052EC61E070E08DE39FE00E9450
:1080F0003E094CED55E060E070E08DE39FE00E94AA
:108100002F8A64E670E080E090E00E94FB8164E0EA
:1081100077E08FED9BE00E941F8C6FED7BE080EAA3
:108120009EE00E94E88762E370E080E090E00E94B9
:10813000FB816FED7BE0CE0101960E94018C42E352
:1081400050E06FEF7FEFCE0101960E94B509CE019E
:1081500001960E94178B60E177E089ED9BE00E9419
:108160001F8C69ED7BE0CE0101960E94018C44E1F9
:1081700050E06FEF7FEFCE0101960E94290BCE01F8
:1081800001960E94178B8091020D9091030D01972B
:1081900031F484E090E0B2DE6B017C0103C0C12CBD
:1081A000D12C76018091020D9091030D892B29F439
:1081B00081E090E0A3DE6B017C0120E030E040EA4A
:1081C00051E4C701B6010E949A91181664F521E0A6
:1081D000B701A601CE0107960E94A48C6FEC75E052
:1081E000CE0101960E94828BBE01695F7F4FCE0156
:1081F00001960E947B8D6CEC75E00E948C8DBC0119
:108200008FED9BE00E94EC8BCE0101960E94178BB4
:10821000CE0107960E94178B81E090E09093030DAA
:108220008093020D10C06CE177E08FED9BE00E941F
:108230001F8C8091020D9091030D019721F41092F3
:10824000030D1092020D6FED7BE0CE0101960E94AE
:10825000018C4AE050E060E070E0CE0101960E949F
:10826000B509CE0101960E94178B6FED7BE0CE0120
:1082700001960E94018C66EC74E0CE0101960E948A
:108280008C8D69ED7BE00E947B8DBC018FED9BE0C6
:108290000E94EC8BCE0101960E94178B8DE39FE02C
:1082A0000E943B858091D00B882331F060E273E01F
:1082B00080E090E00E94FB812C960FB6F894DEBF20
:1082C0000FBECDBFDF91CF91FF90EF90DF90CF90A9
:1082D0000895FF920F931F93CF93DF93CDB7DEB72F
:1082E0002C970FB6F894DEBF0FBECDBF1092D10B06
:1082F0006DE67AE081EF9BE00E941F8C11E080EA3E
:108300009EE00E94CC832091D10B1816190684F5AB
:1083100021112EC080EA9EE00E94E5838093D20B5B
:108320008A3041F08D3031F0682F81EF9BE00E9460
:10833000688D17C01093D10B68E277E0CE010196EB
:108340000E94828B61EF7BE0CE0101960E947B8DC3
:10835000BC0180EA9EE00E94E887CE0101960E945F
:10836000178B6AE070E080E090E00E94FB81C7CF4D
:10837000222361F02091D10B8091F50B9091F60BA7
:1083800021116CC0009709F069C0B0C000E010E096
:10839000FF24F3948AED9FE00E94CC8318161906FF
:1083A000A4F58AED9FE00E94E5838093D20B8A308A
:1083B00071F08D3061F09091D10B911108C0682F50
:1083C00081EF9BE00E94688D0F5F1F4F17C0809167
:1083D000F50B9091F60B892B89F0F092D10B8AED79
:1083E0009FE00E94CC831816190644F46DE67AE0EB
:1083F00081EF9BE00E941F8C1092D10B6FE070E028
:1084000080E090E00E94FB81C5CF62E370E080E0F5
:1084100090E00E94FB81012B09F4ACCF61E377E08F
:10842000CE0101960E94828B61EF7BE0CE01019626
:108430000E947B8DBC0180EA9EE00E94E887CE010D
:1084400001960E94178B8AED9FE00E94548464E697
:1084500070E080E090E00E94FB818CCF019709F0F2
:1084600069C067E776E0CE0107960E94828BBE0165
:10847000695F7F4F81EF9BE00E94C88D811115C01D
:1084800066E377E0CE0101960E94828BBE016F5FAA
:108490007F4F81EF9BE00E94C88D11E0811110E0B9
:1084A000CE0101960E94178B01C010E0CE01079605
:1084B0000E94178B112399F040E050E061EF7BE0C0
:1084C000CE0101960E943209BE016F5F7F4F8BEE95
:1084D0009BE00E94098CCE0101960E94178B64E1FB
:1084E00070E080E090E00E94FB8124C064E670E0D0
:1084F00080E090E00E94FB810E94CC81CB0168EE7D
:1085000073E00E948993CB0164E670E00E94899336
:10851000823691057CF08091D00B81110BC08BEEDF
:108520009BE00E94088F613071058105910511F46F
:108530000E94A3172C960FB6F894DEBF0FBECDBFD6
:10854000DF91CF911F910F91FF9008954F925F920D
:108550006F927F928F929F92AF92BF92CF92DF9253
:10856000EF92FF92CF93DF93CDB7DEB760970FB650
:10857000F894DEBF0FBECDBF8091D00B811105C036
:108580008EE190E0A0E0B0E004C082E090E0A0E0E6
:10859000B0E08D879E87AF87B88B65ED72E08FED79
:1085A0009BE00E94008D6FED7BE0CE0101960E9462
:1085B000018C4AE050E06FEF7FEFCE0101960E9400
:1085C000290BCE0101960E94178B812C912C54010E
:1085D000C12CD12C760163E270E086E09DE00E9420
:1085E000986067E070E086E09DE00E94410986E0C7
:1085F0009DE00E940C6166E970E080E090E00E94DE
:10860000FB8163E270E086E09DE00E94986060E29A
:1086100070E086E09DE00E94410986E09DE00E94B6
:108620000C6166E970E080E090E00E94FB8142E02E
:1086300050E063E270E086E09DE00E940A61412C18
:10864000512C320186E09DE00E94F05F1816190659
:108650006CF486E09DE00E94F85F762C652C542C2B
:108660004424480E511C611C711CECCFC301B201A3
:108670000E94C5902AE939E949E95FE30E94F98F30
:108680000E949290AB01BC01C416D506E606F7061F
:1086900014F46A017B012AE0CE0107960E94788CCF
:1086A000BE01695F7F4FCE0101960E94018C68E395
:1086B00077E0CE0101960E948C8DBC0189ED9BE094
:1086C0000E94EC8BCE0101960E94178BCE0107967B
:1086D0000E94178B69ED7BE0CE0101960E94018C10
:1086E0004EE150E060E070E0CE0101960E945E0A2B
:1086F000CE0101960E94178B9FEF891A990AA90A49
:10870000B90A8D859E85AF85B88988159905AA0512
:10871000BB050CF060CF2AE0B701A601CE01079699
:108720000E94788CBE01695F7F4FCE0101960E9446
:10873000018C68E377E0CE0101960E948C8DBC012C
:1087400089ED9BE00E94EC8BCE0101960E94178B75
:10875000CE0107960E94178B69ED7BE0CE01019652
:108760000E94018C4AE050E060E070E0CE0101968A
:108770000E94B509CE0101960E94178B2AE0B7012D
:10878000A601CE0107960E94788C6CE377E0CE01BB
:1087900001960E94828BBE01695F7F4FCE010196D8
:1087A0000E947B8D6FE377E00E948C8D6FED7BE004
:1087B0000E947B8DBC018FED9BE00E94EC8BCE0173
:1087C00001960E94178BCE0107960E94178B62E3D9
:1087D00070E080E090E00E94FB8160960FB6F89414
:1087E000DEBF0FBECDBFDF91CF91FF90EF90DF9046
:1087F000CF90BF90AF909F908F907F906F905F9041
:108800004F9008958F929F92AF92BF92CF92DF9236
:10881000EF92FF920F931F93CF93DF9300D000D07E
:10882000CDB7DEB78C01E090CD0BF090CE0B65E0BC
:1088300078E080EA9EE00E949C874AE050E0B80120
:1088400080EA9EE00E94BE88C8010596059718F14F
:108850008091CD0B9091CE0B8017910719F10E945A
:10886000040C1093CE0B0093CD0B89EE9CE00E947C
:10887000AA7F4AE0B801CE0101960E944D8CBE014C
:108880006F5F7F4F8BEE9BE00E94098CCE010196BB
:108890000E94178B07C00E3F8FEF1807A9F40E94A4
:1088A000C73798C166EC74E0CE0101960E94828BB6
:1088B0004AE050E06FEF7FEFCE0101960E945E0A22
:1088C000CE0101960E94178BF8017996E332F105EB
:1088D00008F01FC1EE58FF4F0C94DA938091D00B33
:1088E000882319F00E94E63542C160910A02709116
:1088F0000B0280910C0290910D020E94DE3337C171
:1089000080918A0490918B040E944B2F30C18091FA
:108910007004909171040E945A2929C180916404C5
:10892000909165040E94BF2D22C1809166049091B0
:1089300067040E944F281BC10E94CC810E942538E9
:1089400016C160E070E080916A0490916B040E940F
:108950002F240DC180916004909161040E94732BBB
:1089600006C18091CF0B91E089278093CF0B809136
:10897000D00B882331F06FED7BE08AED9FE00E9401
:10898000E88768EC70E080E090E00E94FB81EFC037
:108990001092D00BECC081E08093D00BE8C00E9415
:1089A000290CE5C08CDBE3C00E946116E0C0809119
:1089B0003C02882309F4DBC06DE67AE0CE01019623
:1089C0000E94828B4AE050E061E070E0CE010196A7
:1089D0000E94B509CE0101960E94178B0E942F0EAE
:1089E000C6C0B4DDC4C080916C0490916D040E9437
:1089F000002DBDC080916204909163040E940A2CF6
:108A0000B6C080913C02882309F4B1C08091D00B9C
:108A1000882329F082E090E00E947410A8C083E0CF
:108A200090E00E94A314A3C00E945F228AED9FE001
:108A30000E9454849CC080918102909182020E9485
:108A4000582695C080913C02882309F490C08091FB
:108A5000D00B811127C0C0900A02D0900B02E09089
:108A60000C02F0900D0220E030E04AE754E4C70128
:108A7000B6010E9459920E9492904B015C0120E045
:108A800030E040EA50E4C701B6010E94599220E06C
:108A900030E040EA50E40E942F8F0E949290A5019E
:108AA000940108C021E030E040E050E06AE070E06E
:108AB00080E090E00E942F1E5AC08091040D90919A
:108AC000050D892BA1F481E090E09093050D809332
:108AD000040D8EED93E09093640B8093630B0E94E2
:108AE000910968EC70E080E090E00E94FB81E091E9
:108AF0009A0AF0919B0A19953AC020E042E060E1A1
:108B000089EE9CE00E946A810E943D2F0E94040C25
:108B10002EC0F092CE0BE092CD0B68EF77E08FED98
:108B20009BE00E94008D6DE67AE0CE0101960E94E6
:108B3000828B4AE050E060E070E0CE0101960E9436
:108B4000B509CE0101960E94178B6FED7BE0CE0137
:108B500001960E94018C4AE050E06FEF7FEFCE015A
:108B600001960E94290BCE0101960E94178B8091DD
:108B7000E30B9091E40B009799F0419718F40230C1
:108B80001105ACF46FED7BE0CE0101960E94018CE3
:108B9000CE0101960E948B0FCE0101960E94178B89
:108BA00064E670E080E090E00E94FB8113C06FED0E
:108BB0007BE0CE0101960E94018C4AE050E06FEF0D
:108BC0007FEFCE0101960E94290BCE0101960E94F3
:108BD000178BD8CF26960FB6F894DEBF0FBECDBF49
:108BE000DF91CF911F910F91FF90EF90DF90CF9089
:108BF000BF90AF909F908F900895FF920F931F9317
:108C0000CF93DF9300D000D0CDB7DEB7823409F424
:108C100072C0D4F4803309F48EC07CF4833209F43A
:108C200081C08A3209F0A5C060E577E081EF9BE062
:108C30000E941F8C8FEF9FEFF8C0813309F48AC028
:108C4000813409F44DC095C0813609F449C034F42B
:108C5000833409F45BC0843449F08BC0833609F453
:108C600055C00CF448C0843609F083C08091EF0BE6
:108C70009091F00B892B09F4DAC08BEE9BE00E94F7
:108C8000088F97FDD4C062EF77E080EA9EE00E94F3
:108C90009C876BEE7BE080EA9EE00E94E8878BEE8B
:108CA0009BE00E94088FDC01CB014AEF5FEF6FEF82
:108CB0007FEF481B590B6A0B7B0B2AE0CE01019614
:108CC0000E94788CBE016F5F7F4F8BEE9BE00E940D
:108CD000098CCE0101960E94178B8BEE9BE0A2C0FF
:108CE00064E477E081EF9BE00E941F8C8091CD0BC4
:108CF0009091CE0B9AC067E477E081EF9BE00E94F1
:108D00001F8C1092D00B8CEF9FEF8FC06AE477E03E
:108D100081EF9BE00E941F8C81E08093D00B8DEF50
:108D20009FEF83C06DE477E081EF9BE00E941F8C92
:108D30008EEF9FEF7AC06EE577E08BEE9BE00E94AE
:108D40001F8C6EE577E081EF9BE00E941F8C80E036
:108D500090E06BC061E577E08BEE9BE00E941F8C9A
:108D600061E577E081EF9BE00E941F8C81E090E05D
:108D70005CC0682FCE0101960E94358CBE016F5FEA
:108D80007F4F8BEE9BE00E94098CCE0101960E94E2
:108D9000178B8BEE9BE00E94088FCB0133DD64E6DE
:108DA00070E080E090E00E94FB8149C00F5F1F4FA0
:108DB000093E83E0180769F06EE170E080E090E022
:108DC0000E94FB818BE59CE00E946778F82EFF20D3
:108DD00069F36AE270E06F197109F7FC73954AE074
:108DE000CE0101960E944D8CBE016F5F7F4F81EFD7
:108DF0009BE00E94098CCE0101960E94178B61EFC7
:108E00007BE08BEE9BE00E94EC8B6CEE77E080EADF
:108E10009EE00E949C876F2D80EA9EE00E94088859
:108E200081EF9BE00E94088FCB01ECDC08C08BE552
:108E30009CE00E946778F82E00E010E0C8CF2696EC
:108E40000FB6F894DEBF0FBECDBFDF91CF911F915B
:108E50000F91FF9008950F931F93CF93DF9300D04E
:108E600000D0CDB7DEB74091B00A5091B10A609101
:108E7000B20A7091B30A20E130E080EA9EE00E94DD
:108E800005898091B00A9091B10AA091B20AB0917F
:108E9000B30A883025E09207A105B10509F4F8C1AD
:108EA00008F08DC0893421E09207A105B10509F4CD
:108EB000F2C1E0F5843421E09207A105B10509F47F
:108EC000DBC1E8F4813421E09207A105B10509F482
:108ED000C4C138F480349140A105B10509F4AEC194
:108EE000DDC1823421E09207A105B10509F4BEC1BC
:108EF00083349140A105B10509F4BBC1CFC18634CB
:108F000021E09207A105B10509F4BCC108F4B7C17D
:108F1000873421E09207A105B10509F4B6C1883470
:108F20009140A105B10509F4B3C1B8C1823025E073
:108F30009207A105B10509F499C1E8F4843721E04D
:108F40009207A105B10509F444C138F48237914074
:108F5000A105B10509F448C1A1C1811525E0920719
:108F6000A105B10509F46AC181309540A105B1059B
:108F700009F473C193C1853025E09207A105B105BD
:108F800009F47DC170F4833025E09207A105B10595
:108F900009F46FC184309540A105B10509F46CC195
:108FA0007DC1863025E09207A105B10509F46AC1AB
:108FB00087309540A105B10509F467C16FC18D3BAC
:108FC00022E492072FEFA207B10509F428C108F0A7
:108FD0004BC08F3E20E192072FEFA207B10509F4A5
:108FE00054C118F5823325E09207A105B10509F4B3
:108FF000FBC038F489309540A105B10509F44BC197
:109000004DC1843325E09207A105B10509F4E1C003
:109010008D3F9240AF4FB10509F040C164E477E065
:1090200081EF9BE00E941F8CDCC08D3D22E2920705
:109030002FEFA207B10509F4CCC038F4873E984160
:10904000AF4FB10509F41BC129C18F3C20E3920742
:109050002FEFA207B10509F40FC1873C9843AF4F2A
:10906000B10509F415C11AC1873928E692072FEF17
:10907000A207B10509F4F1C048F58D3A22E592073F
:109080002FEFA207B10509F4BBC038F4853B9A4421
:10909000AF4FB10509F4D2C001C1853A2AE5920764
:1090A0002FEFA207B10509F4F6C08D399246AF4FF4
:1090B000B10509F0F3C067E477E081EF9BE00E941F
:1090C0001F8C1092D00B8CEF9FEF81C0873528EA60
:1090D00092072FEFA207B105F9F078F485382AE757
:1090E00092072FEFA207B10509F4CCC08736984943
:1090F000AF4FB10509F4BAC0D1C08F3420EB92074D
:109100002FEFA207B10509F4B4C08D33924CAF4FD5
:10911000B10509F469C0C2C08CEB9AE00E946D6988
:1091200000E010E06CE97AE08CEB9AE00E94226AA1
:10913000892B39F40F5F1F4F093E83E0180709F0B0
:109140009CC16AED77E080EA9EE00E949C87409196
:10915000A00A5091A10A6091A20A7091A30A2AE084
:1091600030E080EA9EE00E9405898091A00A9091FB
:10917000A10AA091A20AB091A30A853025E0920726
:10918000A105B10509F4B9C008F0C0C0873421E0D9
:109190009207A105B10509F4D9C008F0DAC08334FB
:1091A00021E09207A105B10509F4E3C008F09EC0D3
:1091B000813421E09207A105B10509F0E3C063E520
:1091C00077E08BEE9BE00E941F8C89EF9FEF1ADB0C
:1091D0007EC064E477E081EF9BE00E941F8C1092D8
:1091E000D00B8BEF9FEFF3CF6AE477E081EF9BE04A
:1091F0000E941F8C81E08093D00B8DEF9FEFE7CF13
:109200006DE477E08BEE9BE00E941F8C6DE477E0CD
:1092100081EF9BE00E941F8C8EEF9FEFD8CF60E51F
:1092200077E08BEE9BE00E941F8C60E577E081EF9A
:109230009BE00E941F8C8FEF9FEFC9CF6EE577E018
:109240008BEE9BE00E941F8C6EE577E081EF9BE048
:109250000E941F8C80E090E0BACF61E577E08BEE52
:109260009BE00E941F8C81E090E0B1CF82E090E013
:10927000AECF83E090E0ABCF84E090E0A8CF85E074
:1092800090E0A5CF86E090E0A2CF87E090E09FCF6E
:1092900088E090E09CCF89E090E099CF40E050E0FA
:1092A00061EF7BE0CE0101960E943209BE016F5F43
:1092B0007F4F8BEE9BE00E94098CCE0101960E94AD
:1092C000178B64E670E080E090E00E94FB818CEBFD
:1092D0009AE00E946D6926960FB6F894DEBF0FBE25
:1092E000CDBFDF91CF911F910F910895853421E07B
:1092F0009207A105B10509F054C060E677E08BEE56
:109300009BE00E941F8C85EF9FEF61CF8F3C20E395
:1093100092072FEFA207B10509F448C008F04FC02B
:10932000883025E09207A105B10509F46FC008F067
:1093300080C0863025E09207A105B10509F45DC023
:1093400087309540A105B10509F0BBCF83EF9FEFB2
:109350003ECF813025E09207A105B10509F42FCF5A
:1093600008F44EC0833025E09207A105B10509F04D
:1093700059C069E577E08BEE9BE00E941F8C87EF78
:109380009FEF25CF82349140A105B10509F099CF17
:1093900066E577E08BEE9BE00E941F8C88EF9FEFE5
:1093A00016CF86349140A105B10538F56CE577E01C
:1093B0008BEE9BE00E941F8C86EF9FEF08CF8739D2
:1093C00028E692072FEFA207B10509F4F8CE08F4BA
:1093D00047C0873628E992072FEFA207B105C1F2EF
:1093E0008F3420EB92072FEFA207B10511F28538D9
:1093F0009A47AF4FB10509F064CF84EF9FEFE7CEF6
:10940000883421E09207A105B10519F482EF9FEF9E
:10941000DECE89349140A105B10509F052CF81EF2C
:109420009FEFD5CE84309540A105B10508F4B0CFAB
:10943000BDCF8F3E20E192072FEFA207B10509F4BF
:1094400085CF873E28E192072FEFA207B10509F4E7
:1094500054CF89309540A105B10509F032CFDFCF57
:10946000873C28E392072FEFA207B10579F2853AEE
:109470009A45AF4FB10599F224CF6EE170E080E0DC
:1094800090E00E94FB814ECE8F929F92AF92BF924E
:10949000CF92DF92EF92FF920F931F93CF93DF93C0
:1094A000CDB7DEB7A6970FB6F894DEBF0FBECDBF1F
:1094B0006CEA7AE08CEB9AE00E94226A892BC9F070
:1094C0000E943D2F0E94040C66EC74E0CE010196D0
:1094D0000E94828B4AE050E060E070E0CE0101968D
:1094E0000E94B509CE0101960E94178BB4DC0C9442
:1094F000D85A6DE67AE081EF9BE00E941F8C0E94B3
:1095000069416AE070E080E090E00E94FB81809118
:10951000F50B9091F60B009711F40C94BD5A01973E
:1095200009F046C069EF75E0CE010F960E94828B6C
:10953000BE01615F7F4F81EF9BE00E94C88D81116A
:109540002AC06DEC75E0CE0109960E94828BBE01A7
:10955000675F7F4F81EF9BE00E94C88D811115C02E
:1095600061E375E0CE0101960E94828BBE016F5FC0
:109570007F4F81EF9BE00E94C88D11E0811110E0C8
:10958000CE0101960E94178B01C010E0CE01099612
:109590000E94178B01C010E0CE010F960E94178B1E
:1095A000112331F061EF7BE08BEE9BE00E94EC8BAE
:1095B0008091F50B9091F60B0497F0F564E677E057
:1095C000CE0101960E94828BBE016F5F7F4F81EFBB
:1095D0009BE00E94C88D182FCE0101960E94178B28
:1095E000112351F141E050E061EF7BE0CE0109969B
:1095F0000E943209CE0109960E94088FDC01CB013E
:109600004AEF5FEF6FEF7FEF481B590B6A0B7B0B45
:109610002AE0CE0101960E94788CBE016F5F7F4FD9
:109620008BEE9BE00E94098CCE0101960E94178B65
:10963000CE0109960E94178B66E677E0CE01099667
:109640000E94828BBE01675F7F4F81EF9BE00E948B
:10965000C88D811116C06AE677E0CE0101960E949E
:10966000828BBE016F5F7F4F81EF9BE00E94C88DB0
:1096700011E0811101C010E0CE0101960E94178B0C
:1096800001C011E0CE0109960E94178B112309F445
:10969000EFC260E77BE0CE0101960E94208DCE01F3
:1096A00001960E948B0FCE0101960E94178B60914C
:1096B00038027091390280913A0290913B020E94E7
:1096C000C59020E030E048EC52E40E94F98FAB01F5
:1096D000BC0122E0CE010F960E94A48C6EE677E0DA
:1096E000CE0109960E94828BBE01615F7F4FCE0141
:1096F00009960E947B8D6FE878E00E948C8DBC01FA
:10970000CE0101960E94018CCE0101960E948B0F22
:10971000CE0101960E94178BCE0109960E94178BED
:10972000CE010F960E94178B409134025091350262
:10973000609136027091370224E0CE010F960E94AC
:10974000A48C63E877E0CE0109960E94828BBE016B
:10975000615F7F4FCE0109960E947B8DBC01CE01D7
:1097600001960E94018CCE0101960E948B0FCE01C2
:1097700001960E94178BCE0109960E94178BCE018D
:109780000F960E94178B40911E0250911F0260910C
:1097900020027091210222E0CE0109960E94A48C41
:1097A00040911602509117026091180270911902AF
:1097B00023E0CE010F960E94A48C4091220250918A
:1097C0002302609124027091250222E0CE01459689
:1097D0000E94A48C40911A0250911B0260911C02BD
:1097E00070911D0223E0CE0181960E94A48C60EA54
:1097F00077E0CE014B960E94828BBE016F5D7F4F5A
:10980000CE014B960E947B8D65EB77E00E948C8D9C
:10981000BE016B5E7F4F0E947B8D68EB77E00E94FC
:109820008C8DBE01615F7F4F0E947B8D65EB77E081
:109830000E948C8DBE01675F7F4F0E947B8D6EEB17
:1098400077E00E948C8DBC01CE0101960E94018CB4
:10985000CE0101960E948B0FCE0101960E94178BBC
:10986000CE014B960E94178BCE0181960E94178BDA
:10987000CE0145960E94178BCE010F960E94178B42
:10988000CE0109960E94178B63EC77E0CE01099612
:109890000E94828B6BED7CE0CE0109960E947B8D4D
:1098A000BC01CE0101960E94018CCE0101960E945E
:1098B0008B0FCE0101960E94178BCE0109960E9454
:1098C000178B40914502509146026091470270917A
:1098D000480223E0CE0109960E94A48C20914902FF
:1098E00030914A0240914B0250914C0260E070E08E
:1098F00080E291E40E94BC92AB01BC0121E0CE0168
:1099000045960E94D28C64ED77E0CE010F960E94BE
:10991000828BBE016B5E7F4FCE010F960E947B8DC6
:1099200067EE77E00E948C8DBE01675F7F4F0E94DB
:109930007B8D6BEF75E00E948C8DBC01CE01019692
:109940000E94018CCE0101960E948B0FCE010196E0
:109950000E94178BCE010F960E94178BCE01459661
:109960000E94178BCE0109960E94178B40914102ED
:1099700050914202609143027091440223E0CE0173
:1099800009960E94A48C20913D0230913E024091A4
:109990003F025091400260E070E080E291E40E945A
:1099A000BC92AB01BC0121E0CE0145960E94D28C55
:1099B0006DEE77E0CE010F960E94828BBE016B5E4A
:1099C0007F4FCE010F960E947B8D67EE77E00E945D
:1099D0008C8DBE01675F7F4F0E947B8D6BEF75E0C2
:1099E0000E948C8DBC01CE0101960E94018CCE019B
:1099F00001960E948B0FCE0101960E94178BCE011B
:109A00000F960E94178BCE0145960E94178BCE01B0
:109A100009960E94178B40914D0250914E02609121
:109A20004F027091500222E0CE010F960E94A48C4A
:109A300060E078E0CE0109960E94828BBE01615FF2
:109A40007F4FCE0109960E947B8D66E178E00E94EF
:109A50008C8DBC01CE0101960E94018CCE01019635
:109A60000E948B0FCE0101960E94178BCE010996A2
:109A70000E94178BCE010F960E94178B4091120205
:109A800050911302609114027091150222E0CE01F0
:109A90000F960E94A48C6DE178E0CE0109960E9499
:109AA000828BBE01615F7F4FCE0109960E947B8D44
:109AB0006BEF75E00E948C8DBC01CE0101960E9477
:109AC000018CCE0101960E948B0FCE0101960E945F
:109AD000178BCE0109960E94178BCE010F960E941C
:109AE000178BBEE3CB2EB4E0DB2E01E010E085E166
:109AF000E82E80913C0490913D04801791070CF46E
:109B00004FC0D601AD90BD906D014AE0B501CE01C8
:109B100009960E944D8C4AE0B801CE0145960E94FC
:109B20004D8C60E378E0CE010F960E94828BBE01DF
:109B30006B5E7F4FCE010F960E947B8D6DEE74E0C1
:109B40000E948C8DBE01675F7F4F0E947B8D68E312
:109B500078E00E948C8DEA9CB001EB9C700D112482
:109B60006D577D4F0E948C8DBC01CE0101960E94E5
:109B7000018CCE0101960E948B0FCE0101960E94AE
:109B8000178BCE010F960E94178BCE0145960E942F
:109B9000178BCE0109960E94178B0F5F1F4FA9CF1D
:109BA00040910E0250910F026091100270911102CB
:109BB00022E0CE010F960E94A48C6EE378E0CE01E5
:109BC00009960E94828BBE01615F7F4FCE0109968C
:109BD0000E947B8D67E776E00E948C8DBC01CE01F0
:109BE00001960E94018CCE0101960E948B0FCE013E
:109BF00001960E94178BCE0109960E94178BCE0109
:109C00000F960E94178B40910A0250910B026091AF
:109C10000C0270910D0222E0CE010F960E94A48CDE
:109C20006EE478E0CE0109960E94828BBE01615FEE
:109C30007F4FCE0109960E947B8D67E776E00E94F8
:109C40008C8DBC01CE0101960E94018CCE01019643
:109C50000E948B0FCE0101960E94178BCE010996B0
:109C60000E94178BCE010F960E94178B10E001C047
:109C700011E00E943D2F0E94040C66EC74E0CE01BE
:109C800001960E94828B4AE050E060E070E0CE01D5
:109C900001960E945E0ACE0101960E94178B809168
:109CA000F50B9091F60B8330910508F06FC001978A
:109CB00039F460E070E081EF9BE00E94E78DF82EC0
:109CC0008091F50B9091F60B029709F050C064E675
:109CD00077E0CE0101960E94828BBE016F5F7F4FBD
:109CE00081EF9BE00E94C88D182FCE0101960E9443
:109CF000178B1123E1F161E070E081EF9BE00E949E
:109D0000E78D682FCE0101960E94358CBE016F5FF2
:109D10007F4F8BEE9BE00E94148CCE0101960E9437
:109D2000178B60E070E081EF9BE00E94E78DF82EDA
:109D300069E478E0CE0101960E94828B61EF7BE0BE
:109D4000CE0101960E947B8D66EC74E00E948C8DA2
:109D5000BC0180EA9EE00E94BF87CE0101960E946E
:109D6000178B6BEE7BE080EA9EE00E94E8878F2DE8
:109D70000E94FD450E94CC816093F70B7093F80B15
:109D80008093F90B9093FA0B0C94D85A21E030E0B1
:109D900040E050E061EF7BE0CE0101960E94698EC9
:109DA000BE016F5F7F4F89ED9BE00E94098CCE0161
:109DB00001960E94178B6BE878E0CE0109960E940D
:109DC000828BBE01675F7F4F81EF9BE00E94C88D51
:109DD000811116C063E975E0CE0101960E94828B65
:109DE000BE016F5F7F4F81EF9BE00E94C88D01E055
:109DF000811101C000E0CE0101960E94178B01C0C5
:109E000001E0CE0109960E94178B002309F4A7C038
:109E100042E050E061EF7BE0CE0101960E94320902
:109E2000BE016F5F7F4F89ED9BE00E94098CCE01E0
:109E300001960E94178B69ED7BE080EA9EE00E940C
:109E4000E88789ED9BE00E94128F20E030E048EC2B
:109E500052E40E9459920E949290AB01BC0140933F
:109E600038025093390260933A0270933B022AE021
:109E700030E080EA9EE00E94D488609138027091C0
:109E8000390280913A0290913B028B019C0100596A
:109E90001F452140310901341C492105310588F055
:109EA0006EE578E0CE0101960E94828B69ED7BE041
:109EB000CE0101960E947B8D61E778E00E948C8D37
:109EC00073C119821A821B821C821D821E821F820C
:109ED00018860E94C59020E030E048EC52E40E94D1
:109EE000F98F8E010F5F1F4F22E047E00E943A94E6
:109EF000BC018FED9BE00E941F8C61E878E0CE01F1
:109F000009960E94828B6FED7BE0CE0109960E943C
:109F10007B8D6EE878E00E948C8DBC018FED9BE01C
:109F20000E94EC8BCE0109960E94178B1092640B55
:109F30001092630B8091380290913902A0913A02FD
:109F4000B0913B028093BD0A9093BE0AA093BF0AD2
:109F5000B093C00A80E090E00E9468092EC163E9D6
:109F600078E0CE0109960E94828BBE01675F7F4F29
:109F700081EF9BE00E94C88D811116C069E978E0ED
:109F8000CE0101960E94828BBE016F5F7F4F81EFF1
:109F90009BE00E94C88D01E0811101C000E0CE016C
:109FA00001960E94178B01C001E0CE0109960E9424
:109FB000178B002309F46DC026E030E045E050E047
:109FC00061EF7BE0CE0101960E94698EBE016F5F5A
:109FD0007F4F89ED9BE00E94098CCE0101960E9483
:109FE000178B89ED9BE00E94088F6B017C0164E177
:109FF00078E0CE0109960E94828BBE01675F7F4F99
:10A0000081EF9BE00E94608EAC014F5F5F4F61EF7C
:10A010007BE0CE0101960E943209BE016F5F7F4F47
:10A0200089ED9BE00E94098CCE0101960E94178B5E
:10A03000CE0109960E94178B89ED9BE00E94088F44
:10A04000DB01EEE3F4E021E030E040913C0450918C
:10A050003D04421753075CF0408151814A175B076A
:10A0600011F4118210822F5F3F4F3296EECFF6012E
:10A07000EE0FFF1FE45CFB4F7183608382E090E092
:10A080000E94732E61EF7BE080EA9EE00E94E887E9
:10A0900049C06FE978E0CE0109960E94828BBE012B
:10A0A000675F7F4F81EF9BE00E94C88D811116C0D2
:10A0B00065EA78E0CE0101960E94828BBE016F5F57
:10A0C0007F4F81EF9BE00E94C88D01E0811101C0AC
:10A0D00000E0CE0101960E94178B01C001E0CE0185
:10A0E00009960E94178B002339F1EEE3F4E081E03A
:10A0F00090E020913C0430913D042817390774F01A
:10A10000863091051CF49183808305C09C012E5FED
:10A110003F4F3183208301963296EBCF82E090E06F
:10A120000E94732E1092640B1092630B80E090E0FB
:10A130000E9468090C94D85A6BEA78E0CE0109961F
:10A140000E94828BBE01675F7F4F81EF9BE00E9480
:10A15000C88D811116C063EB78E0CE0101960E9494
:10A16000828BBE016F5F7F4F81EF9BE00E94C88DA5
:10A1700001E0811101C000E0CE0101960E94178B21
:10A1800001C001E0CE0109960E94178B002391F1D6
:10A190006BEB78E0CE0101960E94828B65ED7CE04E
:10A1A000CE0101960E947B8DBC018FED9BE00E9449
:10A1B000EC8BCE0101960E94178B60ED76E0CE010C
:10A1C00009960E94828B6FED7BE0CE0109960E947A
:10A1D0007B8DBC01CE0101960E94018CCE010196BF
:10A1E0000E948B0FCE0101960E94178BCE0109961B
:10A1F0000C94BA5A65EC78E0CE0109960E94828BE5
:10A20000BE01675F7F4F81EF9BE00E94C88D811187
:10A2100016C06AEC78E0CE0101960E94828BBE01E6
:10A220006F5F7F4F81EF9BE00E94C88D01E081113D
:10A2300001C000E0CE0101960E94178B01C001E031
:10A24000CE0109960E94178B002309F444C064E1F3
:10A2500078E0CE0109960E94828BBE01675F7F4F36
:10A2600081EF9BE00E94608EAC014F5F5F4F61EF1A
:10A270007BE0CE0101960E943209BE016F5F7F4FE5
:10A2800089ED9BE00E94098CCE0101960E94178BFC
:10A29000CE0109960E94178B89ED9BE00E94088FE2
:10A2A0006115710521F481E08093990410C061303B
:10A2B000710519F4109299040AC06230710511F009
:10A2C0000C94D85A81E080939904109298040E94CB
:10A2D000C7370C94D85A6FEC78E0CE0109960E94EB
:10A2E000828BBE01675F7F4F81EF9BE00E94C88D2C
:10A2F000811116C063ED78E0CE0101960E94828B39
:10A30000BE016F5F7F4F81EF9BE00E94C88D01E02F
:10A31000811101C000E0CE0101960E94178B01C09F
:10A3200001E0CE0109960E94178B002309F45CC05E
:10A3300043E050E061EF7BE0CE0101960E943209DC
:10A34000BE016F5F7F4F89ED9BE00E94098CCE01BB
:10A3500001960E94178B69ED7BE080EA9EE00E94E7
:10A36000E8871092640B1092630B69ED7BE08BED34
:10A370009CE00E94EC8B20E030E048E050E069ED8A
:10A380007AE08BED9CE00E94E88D8091630B9091C8
:10A39000640B0E94680967ED78E0CE0101960E9487
:10A3A000828B6BED7CE0CE0101960E947B8DBC011F
:10A3B000CE0109960E94018CCE0101960E94178B56
:10A3C000BE01675F7F4F8AED9FE00E94BF8768EB09
:10A3D0007BE080E090E00E94FB8169ED7AE080EA1A
:10A3E0009EE00E94F88769C06FED78E0CE01099683
:10A3F0000E94828BBE01675F7F4F81EF9BE00E94CE
:10A40000C88D811116C064EE78E0CE0101960E94DD
:10A41000828BBE016F5F7F4F81EF9BE00E94C88DF2
:10A4200001E0811101C000E0CE0101960E94178B6E
:10A4300001C001E0CE0109960E94178B002309F4A8
:10A440003FC044E050E061EF7BE0CE0101960E9406
:10A450003209BE016F5F7F4F89ED9BE00E94098C3E
:10A46000CE0101960E94178B69EE78E0CE0101962D
:10A470000E94828B69ED7BE0CE0101960E947B8D6C
:10A48000BC01CE0109960E94018CCE0101960E946A
:10A49000178BBE01675F7F4F8AED9FE00E94BF87E9
:10A4A00068EB7BE080E090E00E94FB81BE01675F8B
:10A4B0007F4F80EA9EE00E94E887CE01099691C70F
:10A4C00060EF78E0CE010F960E94828BBE01615F43
:10A4D0007F4F81EF9BE00E94C88D81112BC063EFFD
:10A4E00078E0CE0109960E94828BBE01675F7F4FA4
:10A4F00081EF9BE00E94C88D811116C066EF78E065
:10A50000CE0101960E94828BBE016F5F7F4F81EF6B
:10A510009BE00E94C88D01E0811101C000E0CE01E6
:10A5200001960E94178B01C001E0CE0109960E949E
:10A53000178B01C001E0CE010F960E94178B0023FC
:10A5400009F42DC16AE0A62EB12CC12CD12C7601C4
:10A5500088248A9473E0972E6EE170E080E090E0AA
:10A560000E94FB81809181020E949182B4010E942D
:10A570008993882777FD8095982F0E94C59020E0C9
:10A5800030E040EA50E40E9459929B01AC01C701BF
:10A59000B6010E942F8F6B017C01E1E0AE1AB10879
:10A5A000D9F620E030E040E251E40E94F98F6B01DF
:10A5B0007C0169EF78E0CE0109960E94828BBE0192
:10A5C000675F7F4F81EF9BE00E94C88D811116C0AD
:10A5D0006DEF78E0CE0101960E94828BBE016F5F25
:10A5E0007F4F81EF9BE00E94C88D01E0811101C087
:10A5F00000E0CE0101960E94178B01C001E0CE0160
:10A6000009960E94178B002309F43FC020E030E038
:10A6100040E650E4C701B6010E9459929B01AC018B
:10A6200060E070E080E890E40E942E8FAB01BC01F6
:10A6300040932A0250932B0260932C0270932D02B8
:10A6400022E0CE0101960E94A48CBE016F5F7F4F75
:10A650008FED9BE00E94098CCE0101960E94178B22
:10A6600061E079E0CE0101960E94828B6FED7BE084
:10A67000CE0101960E947B8DBC018FED9BE00E9474
:10A68000EC8BCE0101960E94178B60E179E0CE0140
:10A6900009960E94828BBE01675F7F4F81EF9BE02E
:10A6A0000E94C88D811116C065E179E0CE01019646
:10A6B0000E94828BBE016F5F7F4F81EF9BE00E9403
:10A6C000C88D01E0811101C000E0CE0101960E9419
:10A6D000178B01C001E0CE0109960E94178B002361
:10A6E00009F43FC020E030E040E650E4C701B60185
:10A6F0000E9459929B01AC0160E070E080E291E41D
:10A700000E942E8FAB01BC0140932602509327027A
:10A71000609328027093290222E0CE0101960E94E4
:10A72000A48CBE016F5F7F4F8FED9BE00E94098C70
:10A73000CE0101960E94178B6AE179E0CE01019665
:10A740000E94828B6FED7BE0CE0101960E947B8D93
:10A75000BC018FED9BE00E94EC8BCE0101960E9424
:10A76000178B60ED76E0CE0109960E94828B6FED2B
:10A770007BE0CE0109960E947B8DBC01CE01019643
:10A780000E94018CCE0101960E948B0FCE01019692
:10A790000E94178BCE0109960E94178BD6C66AE2DB
:10A7A00079E0CE0101960E94828BBE016F5F7F4FE0
:10A7B00081EF9BE00E94C88D082FCE0101960E9478
:10A7C000178B002309F46EC08091F50B9091F60B66
:10A7D000079708F4BAC646E050E061EF7BE0CE018F
:10A7E00001960E943209BE016F5F7F4F89ED9BE0A9
:10A7F0000E94098CCE0101960E94178B89ED9BE087
:10A800000E94128FAB01BC0140930E0250930F02C5
:10A81000609310027093110221E0CE0109960E940C
:10A82000A48C6EE378E0CE0101960E94828BBE017B
:10A83000675F7F4FCE0101960E947B8D67E776E0D0
:10A840000E948C8DBC018FED9BE00E94EC8BCE01B1
:10A8500001960E94178BCE0109960E94178B6FED0F
:10A860007BE0CE0101960E94018CCE0101960E94F0
:10A870008B0FCE0101960E94178B0E94CC8128EE8F
:10A8800033E040E050E00E949C93CA01B9010E946D
:10A89000C3906093370B7093380B8093390B909370
:10A8A0003A0B53C661E379E0CE0101960E94828B98
:10A8B000BE016F5F7F4F81EF9BE00E94C88D082F24
:10A8C000CE0101960E94178B0023E9F18091F50BD0
:10A8D0009091F60B079708F438C646E050E061EF18
:10A8E0007BE0CE0101960E943209BE016F5F7F4F6F
:10A8F00089ED9BE00E94098CCE0101960E94178B86
:10A9000089ED9BE00E94128FAB01BC0140930A02CB
:10A9100050930B0260930C0270930D0221E0CE0164
:10A9200009960E94A48C6EE478E0CE0101960E9404
:10A93000828BBE01675F7F4FCE0101960E947B8DA7
:10A9400067E776E04DC368E379E0CE0109960E949F
:10A95000828BBE01675F7F4F81EF9BE00E94C88DB5
:10A96000811116C06CE379E0CE0101960E94828BC2
:10A97000BE016F5F7F4F81EF9BE00E94C88D01E0B9
:10A98000811101C000E0CE0101960E94178B01C029
:10A9900001E0CE0109960E94178B002309F456C0EE
:10A9A00080916A0490916B040E94042460931A02BF
:10A9B00070931B0280931C0290931D026093D10A36
:10A9C0007093D20A8093D30A9093D40A80E090E0E7
:10A9D000A0E8BFE38093220290932302A093240275
:10A9E000B09325028093C90A9093CA0AA093CB0A18
:10A9F000B093CC0A65E57BE080EA9EE00E949C87EC
:10AA000040911A0250911B0260911C0270911D022C
:10AA100022E030E080EA9EE00E94F1891092640B0F
:10AA20001092630B80E090E00E94680940911A0246
:10AA300050911B0260911C0270911D0222E0CE0118
:10AA400009960E94A48C60E479E0A7C469E479E0E7
:10AA5000CE0109960E94828BBE01675F7F4F81EF16
:10AA60009BE00E94C88D811116C06FE479E0CE0191
:10AA700001960E94828BBE016F5F7F4F81EF9BE04A
:10AA80000E94C88D01E0811101C000E0CE01019655
:10AA90000E94178B01C001E0CE0109960E94178B1E
:10AAA000002309F465C08091F50B9091F60B079790
:10AAB000F8F046E050E061EF7BE0CE0101960E94A5
:10AAC0003209BE016F5F7F4F89ED9BE00E94098CC8
:10AAD000CE0101960E94178B89ED9BE00E94128F98
:10AAE00060934D0270934E0280934F0290935002F8
:10AAF000809164040E94362E80914D0290914E0206
:10AB0000A0914F02B09150028093F10A9093F20A03
:10AB1000A093F30AB093F40A64E47BE080EA9EE039
:10AB20000E949C8740914D0250914E0260914F02CD
:10AB30007091500222E030E080EA9EE00E94F189AC
:10AB40001092640B1092630B80E090E00E94680901
:10AB500040914D0250914E0260914F02709150020F
:10AB600022E0CE0109960E94A48C65E579E015C427
:10AB70006FE579E0CE0109960E94828BBE01675F86
:10AB80007F4F81EF9BE00E94C88D811116C064E663
:10AB900079E0CE0101960E94828BBE016F5F7F4FEC
:10ABA00081EF9BE00E94C88D01E0811101C000E0AF
:10ABB000CE0101960E94178B01C001E0CE010996DB
:10ABC0000E94178B002309F49BC08091F50B909194
:10ABD000F60B069708F145E050E061EF7BE0CE010F
:10ABE00001960E943209BE016F5F7F4F89ED9BE0A5
:10ABF0000E94098CCE0101960E94178B89ED9BE083
:10AC00000E94128F0E94DB916093490270934A0266
:10AC100080934B0290934C0280916604909167045C
:10AC20000E94972720E030E048E051E40E94F98F2D
:10AC300060934502709346028093470290934802C6
:10AC40006093E10A7093E20A8093E30A9093E40A26
:10AC50008091490290914A02A0914B02B0914C021E
:10AC60008093E90A9093EA0AA093EB0AB093EC0A66
:10AC700064E37BE080EA9EE00E949C872091490289
:10AC800030914A0240914B0250914C0260E070E0DA
:10AC900080E291E40E94BC92AB01BC0121E030E073
:10ACA00080EA9EE00E94F08969E679E080EA9EE011
:10ACB0000E94CD8740914502509146026091470223
:10ACC0007091480222E030E080EA9EE00E94F18923
:10ACD0001092640B1092630B80E090E00E94680970
:10ACE000409145025091460260914702709148029E
:10ACF00023E0CE0109960E94A48C60E779E0C7C0EA
:10AD000069E779E0CE0109960E94828BBE01675FF8
:10AD10007F4F81EF9BE00E94C88D811116C06EE7C6
:10AD200079E0CE0101960E94828BBE016F5F7F4F5A
:10AD300081EF9BE00E94C88D01E0811101C000E01D
:10AD4000CE0101960E94178B01C001E0CE01099649
:10AD50000E94178B002309F4A8C08091F50B9091F5
:10AD6000F60B069708F145E050E061EF7BE0CE017D
:10AD700001960E943209BE016F5F7F4F89ED9BE013
:10AD80000E94098CCE0101960E94178B89ED9BE0F1
:10AD90000E94128F0E94DB9160933D0270933E02ED
:10ADA00080933F02909340028091660490916704E3
:10ADB0000E94972720E030E048E051E40E94F98F9C
:10ADC0006093410270934202809343029093440245
:10ADD0006093E50A7093E60A8093E70A9093E80A85
:10ADE00080913D0290913E02A0913F02B0914002BD
:10ADF0008093ED0A9093EE0AA093EF0AB093F00AC5
:10AE000065E27BE080EA9EE00E949C8720913D0203
:10AE100030913E0240913F025091400260E070E06C
:10AE200080E291E40E94BC92AB01BC0121E030E0E1
:10AE300080EA9EE00E94F08969E679E080EA9EE07F
:10AE40000E94CD874091410250914202609143029D
:10AE50007091440222E030E080EA9EE00E94F18995
:10AE60001092640B1092630B80E090E00E946809DE
:10AE7000409141025091420260914302709144021C
:10AE800023E0CE0109960E94A48C63E879E0CE010C
:10AE900001960E94828BBE01675F7F4FCE010196B3
:10AEA0000E947B8D6DEA75E09BC06CE879E0CE0175
:10AEB00009960E94828BBE01675F7F4F81EF9BE006
:10AEC0000E94C88D811116C060E979E0CE0101961B
:10AED0000E94828BBE016F5F7F4F81EF9BE00E94DB
:10AEE000C88D01E0811101C000E0CE0101960E94F1
:10AEF000178B01C001E0CE0109960E94178B002339
:10AF000009F471C060E0809170040E940A8309E135
:10AF100010E0C12CD12C7601809170040E949182A6
:10AF2000BC01882777FD8095982F0E94C5909B01D2
:10AF3000AC01C701B6010E942F8F6B017C016AE052
:10AF400070E080E090E00E94FB810150110921F740
:10AF500020E030E040EA50E4C701B6010E94599277
:10AF600020E030E040E85AE30E94599220E030E0CF
:10AF700048EC51E40E94F98F60931202709313021F
:10AF800080931402909315026093070B7093080B43
:10AF90008093090B90930A0B1092640B1092630B31
:10AFA00080E090E00E9468094091120250911302E3
:10AFB000609114027091150222E0CE0109960E9460
:10AFC000A48C6DE178E0CE0101960E94828BBE01D7
:10AFD000675F7F4FCE0101960E947B8D6BEF75E01E
:10AFE0000E948C8DE5C164E979E0CE0109960E944A
:10AFF000828BBE01675F7F4F81EF9BE00E94C88D0F
:10B00000811116C068E979E0CE0101960E94828B19
:10B01000BE016F5F7F4F81EF9BE00E94C88D01E012
:10B02000811101C000E0CE0101960E94178B01C082
:10B0300001E0CE0109960E94178B002309F473C02A
:10B0400026E030E044E050E061EF7BE0CE01019685
:10B050000E94698EBE016F5F7F4F89ED9BE00E9469
:10B06000098CCE0101960E94178B89ED9BE00E940E
:10B07000088F6B017C0164E178E0CE0109960E94A3
:10B08000828BBE01675F7F4F81EF9BE00E94608EE5
:10B09000AC014F5F5F4F61EF7BE0CE0101960E94F4
:10B0A0003209BE016F5F7F4F89ED9BE00E94098CE2
:10B0B000CE0101960E94178BCE0109960E94178B34
:10B0C00000918A0410918B0489ED9BE00E94128FFD
:10B0D000AB01BC019801C6010E94BA31EBE3FBE071
:10B0E0002BE03BE04191519161917191D9014D93D8
:10B0F0005D936D937D939D01BBE0E336FB0791F774
:10B100001092640B1092630B80E090E00E9468093B
:10B1100044E050E061EF7BE0CE0109960E943209E5
:10B120006CE979E03AC16DEB79E0CE0109960E94B5
:10B13000828BBE01675F7F4F81EF9BE00E94C88DCD
:10B14000811116C061EC79E0CE0101960E94828BDC
:10B15000BE016F5F7F4F81EF9BE00E94C88D01E0D1
:10B16000811101C000E0CE0101960E94178B01C041
:10B1700001E0CE0109960E94178B002309F456C006
:10B1800080916A0490916B040E94042460931602DB
:10B190007093170280931802909319026093D50A56
:10B1A0007093D60A8093D70A9093D80A80E090E5EE
:10B1B000A3ECB7E480931E0290931F02A093200299
:10B1C000B09321028093CD0A9093CE0AA093CF0A28
:10B1D000B093D00A68E07BE080EA9EE00E949C8702
:10B1E0004091160250911702609118027091190255
:10B1F00022E030E080EA9EE00E94F1891092640B28
:10B200001092630B80E090E00E9468094091160262
:10B2100050911702609118027091190222E0CE013C
:10B2200009960E94A48C65EC79E0B7C060ED79E0E6
:10B23000CE0109960E94828BBE01675F7F4F81EF2E
:10B240009BE00E94C88D811116C064ED79E0CE01AB
:10B2500001960E94828BBE016F5F7F4F81EF9BE062
:10B260000E94C88D01E0811101C000E0CE0101966D
:10B270000E94178B01C001E0CE0109960E94178B36
:10B28000002309F4B1C08091F50B9091F60B04975F
:10B29000F8F044E050E061EF7BE0CE0101960E94BF
:10B2A0003209BE016F5F7F4F89ED9BE00E94098CE0
:10B2B000CE0101960E94178B89ED9BE00E94128FB0
:10B2C00060932202709323028093240290932502BC
:10B2D0008091220290912302A0912402B091250234
:10B2E0008093C90A9093CA0AA093CB0AB093CC0A60
:10B2F00060EF7AE080EA9EE00E949C874091220203
:10B3000050912302609124027091250222E030E0E6
:10B3100080EA9EE00E94F08980916A0490916B041B
:10B320000E94042460931A0270931B0280931C02F3
:10B3300090931D026093D10A7093D20A8093D30A2E
:10B340009093D40A66EE7AE080EA9EE00E949C87A1
:10B3500040911A0250911B0260911C0270911D02D3
:10B3600022E030E080EA9EE00E94F1891092640BB6
:10B370001092630B80E090E00E94680940911A02ED
:10B3800050911B0260911C0270911D0222E0CE01BF
:10B3900009960E94A48C68ED79E0CE0101960E9486
:10B3A000828BBE01675F7F4FCE0101960E947B8D2D
:10B3B000BC018FED9BE00E94EC8BCE0101960E94B8
:10B3C000178BCE0109960E94178B6FED7BE0CE01A3
:10B3D00001960E94018CCE0101960E948B0FCE0136
:10B3E00001960E94178BE4C060EE79E0CE010996C9
:10B3F0000E94828BBE01675F7F4F81EF9BE00E94BE
:10B40000C88D811116C064EE79E0CE0101960E94CC
:10B41000828BBE016F5F7F4F81EF9BE00E94C88DE2
:10B4200001E0811101C000E0CE0101960E94178B5E
:10B4300001C001E0CE0109960E94178B002309F498
:10B4400084C08091F50B9091F60B0497F8F044E0DE
:10B4500050E061EF7BE0CE0101960E943209BE010F
:10B460006F5F7F4F89ED9BE00E94098CCE010196B2
:10B470000E94178B89ED9BE00E94128F60931E0241
:10B4800070931F02809320029093210280911E02EC
:10B4900090911F02A0912002B09121028093CD0AC9
:10B4A0009093CE0AA093CF0AB093D00A6EEC7AE0C4
:10B4B00080EA9EE00E949C8740911E0250911F02EC
:10B4C000609120027091210222E030E080EA9EE04B
:10B4D0000E94F08980916A0490916B040E94042478
:10B4E00060931602709317028093180290931902CA
:10B4F0006093D50A7093D60A8093D70A9093D80A9E
:10B5000064EC7AE080EA9EE00E949C8740911602FB
:10B5100050911702609118027091190222E030E0F8
:10B5200080EA9EE00E94F1891092640B1092630BF6
:10B5300080E090E00E946809409116025091170245
:10B54000609118027091190221CF112389F160EDE9
:10B5500076E0CE0101960E94828B61EF7BE0CE0106
:10B5600001960E947B8DBC0180EA9EE00E94E887E4
:10B57000CE0101960E94178B1BC08BE59CE00E94B8
:10B580006778182F8823F9F06DE67AE08BEE9BE060
:10B590000E941F8C68EE79E080EA9EE00E94CD87D1
:10B5A000612F80EA9EE00E940888812F0E94FD455D
:10B5B0000E94CC816093F70B7093F80B8093F90B8A
:10B5C0009093FA0B49C08091D00B882309F44FC0A7
:10B5D0000E94CC8158EEC52E53E0D52EE12CF12CE3
:10B5E000A70196010E949C93CA01B9010E94C390D1
:10B5F0002091370B3091380B4091390B50913A0B19
:10B600000E942E8F20910E0230910F024091100265
:10B61000509111020E949A9118164CF50E94CC810B
:10B62000A70196010E949C93CA01B9010E94C39090
:10B630006093370B7093380B8093390B90933A0BD0
:10B640008091CD0B9091CE0B0E94024464E170E09A
:10B6500080E090E00E94FB818091D00B8823E9F08C
:10B6600064E670E080E090E00E94FB8116C00E94DA
:10B67000CC81C090F70BD090F80BE090F90BF090D4
:10B68000FA0B6C197D098E099F0968347E4E81057D
:10B69000910510F30E94442FDFCFA6960FB6F894C1
:10B6A000DEBF0FBECDBFDF91CF911F910F91FF90F5
:10B6B000EF90DF90CF90BF90AF909F908F900895C4
:10B6C0003F924F925F926F927F928F929F92AF9232
:10B6D000BF92CF92DF92EF92FF920F931F93CF937F
:10B6E000DF9300D01F921F92CDB7DEB75C01562EBC
:10B6F00019821A821B821C821D8261E0852D0E94A4
:10B700000A8360E0852D0E94438362E170E080E05F
:10B7100090E00E94FB8161E0852D0E94438388E2D6
:10B7200090E00E94218260E0852D0E940A8301E161
:10B7300017E2852D0E947883892B31F4015011097D
:10B74000C1F78EEF9FEF6EC001E117E2852D0E94D9
:10B750007883019721F401501109C1F7F2CF08E273
:10B7600010E0312C37E0432E88248394912C21E182
:10B77000E22E27E2F22E852D0E947883892B29F470
:10B7800081E0E81AF108B9F7DCCF0E94D8816B019B
:10B790007C0191E1692E97E2792E852D0E947883B4
:10B7A000019729F4E1E06E1A7108B9F7CACF0E9437
:10B7B000D8816C197D098E099F096932710581054F
:10B7C000910578F0E1E0F0E0EC0FFD1FE30DF11DD5
:10B7D0002081C401042C01C0880F0A94EAF7282BA9
:10B7E0002083411004C0339487E0482E01C04A945E
:10B7F0000150110909F0BBCF2981822F90E0F5019A
:10B80000918380833B81832F90E093838283230FF6
:10B8100081E090E03D81321302C080E090E091959C
:10B82000819591090F900F900F900F900F90DF91DD
:10B83000CF911F910F91FF90EF90DF90CF90BF902D
:10B84000AF909F908F907F906F905F904F903F90C0
:10B850000895FB018081883251F028F4803139F05D
:10B86000823239F404C08B3311F0823411F481E058
:10B87000089580E00895FC01778366831482158221
:10B88000108289E0818381E0828383830895CF934E
:10B89000DF93EC01F0DF1B8A1A8ADF91CF910895C4
:10B8A000FC0185810895CF93DF93EB0167E0CE0122
:10B8B0000E94D17E91E02F81821390E0892FDF9149
:10B8C000CF910895EF92FF920F931F93CF93DF9341
:10B8D000EC018B01E42E8E819F810E94067EF12C6B
:10B8E00041E0B8018E819F810E94397E882351F00A
:10B8F000FE1005C0B801CE01D6DF811104C0F3945B
:10B90000EF1470F780E0DF91CF911F910F91FF90BE
:10B91000EF900895CF92DF92EF92FF920F931F93D3
:10B92000CF93DF931F921F92CDB7DEB76C01F42E39
:10B93000E52EFC018681978169837A830E94EE7CE3
:10B9400069817A81882311F1F601868197810E94AD
:10B95000DD7D40E06EEBF601868197810E94817D5E
:10B960000F2D1E2D89E0F82EF601868197810E9409
:10B97000C27DF80181938F01FA94B1F7F6018681B7
:10B9800097810E94EE7C91E0813009F090E0892F50
:10B990000F900F90DF91CF911F910F91FF90EF903B
:10B9A000DF90CF900895CF93DF93EA01B3DF882330
:10B9B00051F068E0CE010E94D17E91E0288582138B
:10B9C00090E0892F01C080E0DF91CF910895EF9240
:10B9D000FF920F931F93CF93DF93EC018B017A01BA
:10B9E0008E819F810E94EE7CB8018E819F810E9492
:10B9F000DD7D40E06EE48E819F810E94817D40E08C
:10BA0000F70162818E819F810E94817D40E0F70174
:10BA100063818E819F810E94817DF80180818031C8
:10BA200039F040E0F70164818E819F810E94817D21
:10BA30008E819F810E94EE7CB8018E819F810E9441
:10BA4000DD7D488168E48E819F810E94817D64E173
:10BA500070E080E090E00E94FB818881882331F0D3
:10BA60006AE070E080E090E00E94FB818E819F811F
:10BA7000DF91CF911F910F91FF90EF900C94EE7C8E
:10BA8000EF92FF921F93CF93DF931F921F92CDB738
:10BA9000DEB77C01FC018681978169837A830E94ED
:10BAA000EE7C69817A81F701868197810E94DD7D34
:10BAB00040E064EBF701868197810E94817DF70168
:10BAC000868197810E94597D182FF7018681978181
:10BAD0000E94EE7C81E0111180E00F900F90DF91C9
:10BAE000CF911F91FF90EF900895CF93DF93CDB743
:10BAF000DEB729970FB6F894DEBF0FBECDBFFB01AE
:10BB000020812031C9F0AE014F5F5F4F4CDF8823A9
:10BB100079F08D818F3351F020F48F3149F489E031
:10BB20000CC08F3539F08F3739F002C08AE005C07C
:10BB300080E003C08BE001C08CE029960FB6F8943A
:10BB4000DEBF0FBECDBFDF91CF910895FF920F935F
:10BB50001F93CF93DF93CDB7DEB728970FB6F89436
:10BB6000DEBF0FBECDBF8C01FC01868197810E9494
:10BB7000067EF8011482158241E0BE016F5F7F4F9F
:10BB8000F801868197810E94397E8823C1F1BE0128
:10BB90006F5F7F4FC80187DE882371F3F8018081D2
:10BBA000811107C0BE016F5F7F4FC80169DF81113E
:10BBB00022C0F801F180BE016F5F7F4FC80195DFA1
:10BBC0008F1518F4F801818105C0BE016F5F7F4FAA
:10BBD000C8018BDFF801818384818F5F8483BE017C
:10BBE0006F5F7F4FC80135DE882331F2F801858110
:10BBF0008F5F8583C1CF81E0F8018083DACF2896FB
:10BC00000FB6F894DEBF0FBECDBFDF91CF911F916D
:10BC10000F91FF900895DF92EF92FF920F931F9381
:10BC2000CF93DF93CDB7DEB762970FB6F894DEBF40
:10BC30000FBECDBF8C017B01D22E493028F0342FAE
:10BC40004D3018F03CE001C039E0B701C8013A8B33
:10BC50004CDF3A89831709F458C0AE014F5F5F4F3C
:10BC6000B701C8013A8B9FDE3A89882309F44FC097
:10BC7000F7018081803109F448C03B3041F03C300D
:10BC800021F03A3031F48FE305C08FE703C08FE530
:10BC900001C08FE18D83AE014F5F5F4FB701C801D7
:10BCA0003A8B95DEF80191813A89832F391708F490
:10BCB000892FF8018183D11028C0381730F53183DE
:10BCC000E12CF12CF801848190E0E816F906ECF4FF
:10BCD0004E2DBE01665F7F4FC801F4DDF801D180B3
:10BCE000BE01665F7F4FC80100DF8D1518F4F801B3
:10BCF000818105C0BE01665F7F4FC801F6DEF80195
:10BD00008183FFEFEF1AFF0ADDCF81E001C080E001
:10BD100062960FB6F894DEBF0FBECDBFDF91CF9114
:10BD20001F910F91FF90EF90DF900895EF92FF9297
:10BD30000F931F93CF93DF93CDB7DEB728970FB63E
:10BD4000F894DEBF0FBECDBF8C01693020F06D309E
:10BD500018F06CE001C069E0F8016183E12CF12C7E
:10BD6000F801848190E0E816F90694F44E2DBE01A6
:10BD70006F5F7F4FC801A6DD21E0F8014181BE0160
:10BD80006F5F7F4FC80147DFFFEFEF1AFF0AE8CF71
:10BD900028960FB6F894DEBF0FBECDBFDF91CF91CE
:10BDA0001F910F91FF90EF900895FC01868197817C
:10BDB0000E94597D91E0813009F090E0892F08952B
:10BDC0008F929F92AF92BF92CF92DF92EF92FF92AB
:10BDD0000F931F93CF93DF93EC016950633048F4C6
:10BDE000E62FF0E0EE0FFF1FE550F64F00811181C6
:10BDF00002C00EEE12E08B818823E1F08881811170
:10BE000019C00E94CC816B017C014801AA2497FCD7
:10BE1000A094BA2CCE01C9DF81111FC00E94CC8131
:10BE2000681979098A099B096C157D058E059F059E
:10BE3000A0F4F0CFB801882777FD8095982FDF9187
:10BE4000CF911F910F91FF90EF90DF90CF90BF9017
:10BE5000AF909F908F900C94FB81DF91CF911F91B9
:10BE60000F91FF90EF90DF90CF90BF90AF909F9099
:10BE70008F900895CF93DF93EC018E819F810E9474
:10BE8000EE7C8E819F810E94037E488164E48E81D6
:10BE90009F810E94817D8A81882329F06981CE015A
:10BEA000DF91CF918DCFDF91CF910895FA0120815D
:10BEB00048E0249F90011124818190E0982F8827E9
:10BEC000990F990F990F282B392BDB018C91803119
:10BED000C1F4678170E08681AB01481B5109CA013A
:10BEE0009695982F8827979587950E9489936051FA
:10BEF0007109207F53E0220F331F5A95E1F7260F77
:10BF0000371FC9010895EF92FF920F931F93CF93AC
:10BF1000DF93CDB7DEB729970FB6F894DEBF0FBE1B
:10BF2000CDBF8C017B01AE014F5F5F4F3CDD8823AD
:10BF300039F0AE014F5F5F4FB701C801B7DF02C0F4
:10BF400080E894EE29960FB6F894DEBF0FBECDBF01
:10BF5000DF91CF911F910F91FF90EF90089581385D
:10BF600024EE92076CF0BC01882777FD8095982F0E
:10BF70000E94C59020E030E040E05CE30C945992D0
:10BF800060E070E08EEF92EC0895BDDFE8CF0F9394
:10BF90001F93CF93DF93CDB7DEB728970FB6F894F2
:10BFA000DEBF0FBECDBF8C01462FBE016F5F7F4F3E
:10BFB00089DC882331F0BE016F5F7F4FC801E5DF68
:10BFC00004C060E070E08EEF92EC28960FB6F89413
:10BFD000DEBF0FBECDBFDF91CF911F910F910895AE
:10BFE0008091360D90E02091370D821B91090895C4
:10BFF0002091370D8091360D281750F4E22FF0E094
:10C00000E85CF24F808190E02F5F2093370D089518
:10C010008FEF9FEF0895E091370D8091360DE8176F
:10C0200030F4F0E0E85CF24F808190E008958FEF0B
:10C030009FEF08950895CF92DF92EF92FF920F93B2
:10C040001F93CF93DF937C01CB018A012091120DC6
:10C05000222389F0EB016B01C40ED51ECC15DD0542
:10C0600061F06991D701ED91FC910190F081E02D93
:10C07000C7011995F3CF642F91D1C801DF91CF91FA
:10C080001F910F91FF90EF90DF90CF900895CF9385
:10C09000DF931F92CDB7DEB769832091120D222363
:10C0A000D1F02091130D203240F021E030E0FC016E
:10C0B0003383228380E090E014C08091140DE82F38
:10C0C000F0E0EB5EF24F998190838F5F8093140DC7
:10C0D0008093130D04C061E0CE0101965FD181E031
:10C0E00090E00F90DF91CF910895FC0113821282AE
:10C0F00048EE53E060E070E04483558366837783C5
:10C1000085E09AE09183808308951092370D109214
:10C11000360D1092140D1092130D83C081E08093A0
:10C12000120D6093350D1092140D1092130D089599
:10C13000F5CF0F93062F21E04091130D65E17DE0CF
:10C140008091350DD4D01092140D1092130D1092D1
:10C15000120D0F9108958F929F92AF92BF92CF923E
:10C16000DF92EF92FF920F931F93CF93DF93EC0137
:10C17000F62ED42E48015901EE2009F1CFDF1E2DF5
:10C18000143008F013E01150B8F0E881F98128E08C
:10C19000129FB0011124A501940104C05695479542
:10C1A000379527956A95D2F7CA01B9010190F081B8
:10C1B000E02DCE011995E7CF60E0CE01BADF4D2D1D
:10C1C000413208F040E22C2D68E37DE08F2D47D00E
:10C1D0001092370D8093360DDF91CF911F910F9103
:10C1E000FF90EF90DF90CF90BF90AF909F908F9097
:10C1F0000895CF92EF920F931F93C22EE12C00E08F
:10C2000010E09801A8DF1F910F91EF90CF90089553
:10C2100021E0EFCF21E0EDCF61E08BCF86E09DE024
:10C2200064CF1092C50D81E08093C30D1092C20DB2
:10C2300061E084E10E94438361E085E10E944383E1
:10C24000E9EBF0E080818E7F808380818D7F808329
:10C2500088E48093B80085E48093BC00089541325F
:10C2600008F043C09091C50D9111FCCF91E09093DF
:10C27000C50D2093C30D2FEF2093580D10929D0DE7
:10C28000240F20939C0D9093C40D9091C40D880FA2
:10C29000892B8093C40D8091C20D813061F410927E
:10C2A000C20D8091C40D8093BB008091BC0083FDC2
:10C2B000F8CF85EC01C085EE8093BC008091C50D60
:10C2C0008130E1F380919D0D841710F440919D0D14
:10C2D0002EE93DE0FB01D9018A2F821B841718F457
:10C2E0008D918193F9CF842F089580E008950F9365
:10C2F000413208F04AC09091C50D9111FCCF92E0F7
:10C300009093C50D0093C30D9FEF9093580D10921D
:10C310009D0D40939C0DFB016EE97DE0DB019A2FA2
:10C32000961B941718F491919D93F9CF1092C40D18
:10C330009091C40D880F892B8093C40D8091C20DFC
:10C34000813061F41092C20D8091C40D8093BB00C6
:10C350008091BC0083FDF8CF85EC01C085EE809311
:10C36000BC00222321F08091C50D8230E1F3809141
:10C37000580D8F3F61F08091580D803251F08091BF
:10C38000580D803341F483E007C081E005C080E0B0
:10C3900003C082E001C084E00F910895613298F4F7
:10C3A0002091C50D243089F460937A0DFC018CE74F
:10C3B0009DE0DC012A2F281B261718F421912D93CC
:10C3C000F9CF80E0089581E0089582E0089585ED39
:10C3D0008093BC008091BC0084FDFCCF1092C50D01
:10C3E000089585EC8093BC001092C50D08951F92AE
:10C3F0000F920FB60F9211240BB60F922F933F930B
:10C400004F935F936F937F938F939F93AF93BF935C
:10C41000EF93FF938091B900887F803609F49DC027
:10C4200070F5883209F45CC090F4803109F455C08D
:10C4300038F4882309F4F3C0883009F44EC0F2C000
:10C44000883109F44DC0803209F45EC0EBC08034FD
:10C4500009F469C050F4803309F456C0883309F0F8
:10C46000E1C08093580DBDDFDDC0803509F44FC0B9
:10C47000883509F45DC0883409F0D4C0D2C0883949
:10C4800009F4C3C0A8F4883709F467C038F48836C3
:10C4900009F463C0803709F460C0C4C0883809F467
:10C4A000B4C0803909F45FC0803809F0BBC05BC0FC
:10C4B000803B09F482C038F4803A09F466C0883AB7
:10C4C00009F47BC0AFC0803C09F4A3C0883C09F4E8
:10C4D000A0C0883B09F486C0A5C08091C40D10C0DF
:10C4E00090919D0D80919C0D981770F5E0919D0D98
:10C4F00081E08E0F80939D0DF0E0E256F24F808137
:10C500008093BB0085EC82C08093580D8AC0E09177
:10C510009D0D81E08E0F80939D0D8091BB00F0E01A
:10C52000E256F24F808390919D0D80919C0D6AC0E0
:10C53000E0919D0D81E08E0F80939D0D8091BB0059
:10C54000F0E0E256F24F80838091C30D811169C003
:10C5500081E08093C20D84EA5DC083E08093C50DC5
:10C560001092590DCFCF8091590D803208F04DC0F7
:10C57000E091590D81E08E0F8093590D8091BB00A1
:10C58000F0E0E65AF24F8083BDCF2BDF8091590D4A
:10C59000803230F4E091590DF0E0E65AF24F10820B
:10C5A0006091590D70E0E091BE0DF091BF0D8AE5EC
:10C5B0009DE019951092590D35C084E08093C50D0A
:10C5C00010927B0D10927A0DE091C00DF091C10D8B
:10C5D000199580917A0D811105C081E080937A0DC3
:10C5E00010927C0DE0917B0D81E08E0F80937B0D8E
:10C5F000F0E0E458F24F80818093BB0090917B0D76
:10C6000080917A0D981708F47DCF85E88093BC005F
:10C6100009C085EC8093BC001092C50D03C0109238
:10C62000580DD5DEFF91EF91BF91AF919F918F9102
:10C630007F916F915F914F913F912F910F900BBE22
:10C640000F900FBE0F901F901895FC0181E0808322
:10C65000118243EC5BEA66E77BE3428353836483A6
:10C66000758348ED5BE666E77BE346835783608727
:10C67000718742EF54EE64E67BE342875387648719
:10C6800075870895FC01DB014D915D916D917C9161
:10C690001397428353836483758314964D915D9100
:10C6A0006D917C91179746835783608771871896A1
:10C6B0004D915D916D917C911B9742875387648763
:10C6C00075870895CF93DF93FC01EB01428153817D
:10C6D00064817581488359836A837B83468157814E
:10C6E000608571854C835D836E837F8382859385AE
:10C6F000A485B58588879987AA87BB87DF91CF9165
:10C7000008950F931F93CF93DF93082F6DEC75E07F
:10C7100080EA9EE00E94CD87C7E0D0E010E0B8013B
:10C720000C2E02C0759567950A94E2F76170772721
:10C7300042E050E080EA9EE00E94B788219778F7B7
:10C74000DF91CF911F910F9108951F93CF93DF93A6
:10C750001F92CDB7DEB7162F63E570E086E09DE04F
:10C760004983E6DC612F86E09DE091DC4981642FFE
:10C7700086E09DE08CDC86E09DE00F90DF91CF911C
:10C780001F914ACDCF93DF93EC0186E09DE0BDDCA5
:10C7900040E06DE2CE01D9DF40E16DE2CE01D5DFB0
:10C7A00048E06DE2CE01DF91CF91CFCF6F3F7105B1
:10C7B00034F4AB0177FF05C040E050E002C04FEF1A
:10C7C00050E06DE1C2CFEF92FF921F93CF93DF93C2
:10C7D0001F92CDB7DEB77C01142F462F6EE129835F
:10C7E000B4DF412F6FE1C701B0DF2981422F60E242
:10C7F000C7010F90DF91CF911F91FF90EF90A5CFD0
:10C800006F3F710534F4AB0177FF05C040E050E0A5
:10C8100002C04FEF50E061E298CF462F62E295CF21
:10C820006F3F710534F4AB0177FF05C040E050E085
:10C8300002C04FEF50E063E288CF6F3F710534F4E0
:10C84000AB0177FF05C040E050E002C04FEF50E081
:10C8500064E27BCF6F3F710534F4AB0177FF05C015
:10C8600040E050E002C04FEF50E065E26ECF6F3F16
:10C87000710534F4AB0177FF05C040E050E002C021
:10C880004FEF50E066E261CF6F3F710534F4AB01CA
:10C8900077FF05C040E050E002C04FEF50E068E293
:10C8A00054CF6F3F710534F4AB0177FF05C040E012
:10C8B00050E002C04FEF50E069E247CFAF92BF9225
:10C8C000CF92DF92EF92FF920F931F93CF93DF935C
:10C8D0008C01C62F7A01690163E570E086E09DE076
:10C8E00027DC6C2F86E09DE0D2DB86E09DE094DCC7
:10C8F00063E570E086E09DE01BDCA70163E570E086
:10C9000086E09DE087DCE6015E01AC18BD0886E0AC
:10C910009DE066DB892B29F086E09DE069DB899349
:10C92000F3CFAE14BF0421F0F801108281E08183BF
:10C9300086E09DE0DF91CF911F910F91FF90EF90E6
:10C94000DF90CF90BF90AF9067CCCF92DF92EF9205
:10C95000FF920F931F93CF93DF93EC016B017A014A
:10C9600089019C01225F3F4F46E050E062E3A6DF71
:10C970008F8590E0982F88272E85822BF601918352
:10C980008083898990E0982F88272889822BF70156
:10C99000918380838B8990E0982F88272A89822B26
:10C9A000F80191838083DF91CF911F910F91FF90C8
:10C9B000EF90DF90CF9008959B012C5F3F4FAB012C
:10C9C0004E5F5F4FC2CFAF92BF92CF92DF92EF9296
:10C9D000FF920F931F93CF93DF9300D000D0CDB77A
:10C9E000DEB77C015B01BE016F5F7F4FE5DFCE01EB
:10C9F00001966C01870175015E0197E0A90EB11CDB
:10CA0000F601619171916F01882777FD8095982FCC
:10CA10000E94C590F80122813381448155810E9492
:10CA20005992F70161937193819391937F010C5F08
:10CA30001F4FCA14DB0421F726960FB6F894DEBF09
:10CA40000FBECDBFDF91CF911F910F91FF90EF905F
:10CA5000DF90CF90BF90AF900895CF93DF931F9258
:10CA6000CDB7DEB79E012F5F3F4F41E050E06DE153
:10CA700025DF898190E00F90DF91CF910895AF92EB
:10CA8000BF92CF92DF92EF92FF920F931F93CF93BB
:10CA9000DF931F92CDB7DEB78C015B016A0179018C
:10CAA0009E012F5F3F4F41E050E06EE107DF89813B
:10CAB00090E0F501918380839E012F5F3F4F41E01D
:10CAC00050E06FE1C801FADE898190E0F6019183C0
:10CAD00080839E012F5F3F4F41E050E060E2C8013C
:10CAE000EDDE898190E0F701918380830F90DF91E3
:10CAF000CF911F910F91FF90EF90DF90CF90BF905B
:10CB0000AF900895CF93DF931F92CDB7DEB79E010C
:10CB10002F5F3F4F41E050E061E2D0DE898190E03D
:10CB20000F90DF91CF910895CF93DF931F92CDB7F0
:10CB3000DEB79E012F5F3F4F41E050E062E2BEDE74
:10CB4000898190E00F90DF91CF910895CF93DF938B
:10CB50001F92CDB7DEB79E012F5F3F4F41E050E0FF
:10CB600063E2ACDE898190E00F90DF91CF91089570
:10CB7000CF93DF931F92CDB7DEB79E012F5F3F4F5C
:10CB800041E050E064E29ADE898190E00F90DF910D
:10CB9000CF910895CF93DF931F92CDB7DEB79E015B
:10CBA0002F5F3F4F41E050E065E288DE898190E0F1
:10CBB0000F90DF91CF910895CF93DF931F92CDB760
:10CBC000DEB79E012F5F3F4F41E050E066E276DE28
:10CBD000898190E00F90DF91CF910895CF93DF93FB
:10CBE0001F92CDB7DEB79E012F5F3F4F41E050E06F
:10CBF00068E264DE898190E00F90DF91CF91089523
:10CC0000CF93DF931F92CDB7DEB79E012F5F3F4FCB
:10CC100041E050E069E252DE898190E00F90DF91BF
:10CC2000CF910895CF93DF931F92CDB7DEB79E01CA
:10CC30002F5F3F4F41E050E06CE240DE69816F7052
:10CC400070E066507109882777FD8095982F0E94C3
:10CC5000C5909B01AC0160E070E080E090E40E9430
:10CC6000BC9220E030E048EC50E40E9459920F90D2
:10CC7000DF91CF910895EF92FF920F931F93CF937F
:10CC8000DF931F92CDB7DEB78C01CB01BA0120E054
:10CC900030E048EC50E40E94F98F0E949290E12C21
:10CCA000F12C759567956115710521F08FEFE81AE4
:10CCB000F80AF7CF8AE0E816F10484F49E012F5FAA
:10CCC0003F4F41E050E06CE2C801F8DD46E04E0D18
:10CCD0008981807F482B6CE2C80137DD0F90DF919E
:10CCE000CF911F910F91FF90EF900895CF93DF9315
:10CCF0001F92CDB7DEB79E012F5F3F4F41E050E05E
:10CD000060E3DCDD89810F90DF91CF910895DF92A0
:10CD1000EF92FF920F931F93CF93DF931F92CDB7A4
:10CD2000DEB78C01F62EE42ED22E9E012F5F3F4FF0
:10CD300041E050E0C3DD898121E030E00E2C01C0EC
:10CD4000220F0A94EAF7DD2011F0282B02C020956B
:10CD50002823298349816F2DC801F7DC0F90DF91CB
:10CD6000CF911F910F91FF90EF90DF900895262FA4
:10CD700047E050E061E3CBCF262F46E050E067E28A
:10CD8000C6CF262F45E050E067E2C1CF262F44E012
:10CD900050E067E2BCCF262F42E050E067E2B7CF19
:10CDA000262F41E050E067E2B2CF262F40E050E06E
:10CDB00067E2ADCF262F47E050E067E2A8CF262FED
:10CDC00043E050E067E2A3CF262F43E050E06AE261
:10CDD0009ECF262F42E050E06AE299CF262F41E015
:10CDE00050E06AE294CF262F40E050E06AE28FCF15
:10CDF000262F44E050E06CE28ACF242F462F50E0EB
:10CE00006FE285CF242F462F50E06EE280CF1F9334
:10CE1000CF93DF931F92CDB7DEB7142F9E012F5F04
:10CE20003F4F41E050E04ADD898190E002C0959596
:10CE300087951A95E2F781700F90DF91CF911F913E
:10CE4000089547E050E061E3E2CF46E050E067E25A
:10CE5000DECF45E050E067E2DACF44E050E067E241
:10CE6000D6CF42E050E067E2D2CF41E050E067E247
:10CE7000CECF40E050E067E2CACF43E050E067E247
:10CE8000C6CF43E050E06AE2C2CF42E050E06AE23F
:10CE9000BECF41E050E06AE2BACF40E050E06AE243
:10CEA000B6CF46E050E06BE2B2CF45E050E06BE237
:10CEB000AECF44E050E06BE2AACF42E050E06BE23C
:10CEC000A6CF41E050E06BE2A2CF40E050E06BE241
:10CED0009ECF43E050E06BE29ACF44E050E06CE23A
:10CEE00096CF462F50E060E392CF462F50E06FE29E
:10CEF0008ECF462F50E06EE28ACFEF92FF920F93D3
:10CF00001F93CF93DF931F92CDB7DEB77C0161E112
:10CF10007AE080EA9EE00E94CD879E012F5F3F4F1E
:10CF200041E050E060E0C701C9DC8981EADB6DE6E1
:10CF30007AE080EA9EE00E94F8870DE110E068E167
:10CF40007AE080EA9EE00E94CD8740E150E0B8019F
:10CF500080EA9EE00E94B7886DE679E080EA9EE074
:10CF60000E94CD879E012F5F3F4F41E050E0602F30
:10CF7000C701A4DC8981C5DB6DE67AE080EA9EE02A
:10CF80000E94F8870F5F1F4F0A331105C1F60F90FB
:10CF9000DF91CF911F910F91FF90EF900895CF9265
:10CFA000DF92EF92FF92CF93DF93EC01882777FD1A
:10CFB0008095982F0E94C5906B017C0120E030E0A5
:10CFC00040E45FE30E94599220E030E048E452E4FC
:10CFD0000E94F98F0E949290C617D707ECF020E0CC
:10CFE00030E040EA5FE3C701B6010E94599220E0B9
:10CFF00030E048E452E40E94F98F20E030E040E85D
:10D000005FE30E942F8F0E94929021E06C177D07B2
:10D010000CF420E0822F01C080E090E0DF91CF91FE
:10D02000FF90EF90DF90CF900895CF92DF92EF9234
:10D03000FF92CF93DF93EC016C597F4F882777FDE8
:10D040008095982F0E94C5906B017C0120E030E014
:10D0500040E45FE30E94599220E030E048E452E46B
:10D060000E94F98F0E949290C617D707ECF020E03B
:10D0700030E040EA5FE3C701B6010E94599220E028
:10D0800030E048E452E40E94F98F20E030E040E8CC
:10D090005FE30E942F8F0E94929021E06C177D0722
:10D0A0000CF420E0822F01C080E090E0DF91CF916E
:10D0B000FF90EF90DF90CF900895CF92DF92EF92A4
:10D0C000FF92CF93DF93EC0164567109882777FDB7
:10D0D0008095982F0E94C5906B017C0120E030E084
:10D0E00040E45FE30E94599220E030E048E452E4DB
:10D0F0000E94F98F0E949290C617D707ECF020E0AB
:10D1000030E040EA5FE3C701B6010E94599220E097
:10D1100030E048E452E40E94F98F20E030E040E83B
:10D120005FE30E942F8F0E94929021E06C177D0791
:10D130000CF420E0822F01C080E090E0DF91CF91DD
:10D14000FF90EF90DF90CF9008951F920F920FB64F
:10D150000F9211240BB60F922F933F934F935F932F
:10D160006F937F938F939F93AF93BF93EF93FF93AF
:10D170008091C70D0E9478832091CA0D3091CB0D0C
:10D180002F5F3F4F3093CB0D2093CA0D9091C90D67
:10D19000953618F096E09093C60D9091C60D943098
:10D1A000C9F128F4923069F09330D1F05EC0953027
:10D1B00009F451C0963009F058C091E09093960E52
:10D1C00051C0811152C02091CA0D3091CB0D24362F
:10D1D000310508F442C01092960E1092C90D1CC081
:10D1E000813009F042C0E091C90D91E09E0F90930B
:10D1F000C90DF0E02091CA0D3091CB0DEE0FFF1F4D
:10D20000E453F24F318320831092CB0D1092CA0D5C
:10D2100094E029C0811117C0E091C90D91E09E0FE3
:10D220009093C90DF0E02091CA0D3091CB0DEE0F17
:10D23000FF1FE453F24F318320831092CB0D1092E5
:10D24000CA0D93E010C02091CA0D3091CB0D253648
:10D25000310558F007C0811108C01092CB0D109213
:10D26000CA0D03C095E09093C60D9091C80D992307
:10D2700029F0811102C02F9A01C02F98FF91EF91E0
:10D28000BF91AF919F918F917F916F915F914F91DE
:10D290003F912F910F900BBE0F900FBE0F901F90DC
:10D2A00018956093C70D1092C80D0895F89482E008
:10D2B0008093B0008093B10094E69093B3001092F5
:10D2C000B2008093700078948093C60D1092C90DBF
:10D2D0008091C70D60E00C940A8382E08093C60DB4
:10D2E0001092C90D08958F929F92AF92BF92CF92E4
:10D2F000DF92EF92FF927B01BA0180E090E00E9402
:10D30000C3904B015C01B70180E090E00E94C390A4
:10D310006B017C012DEC3CEC4CE45FE30E945992E4
:10D320009B01AC01C501B4010E94F58F87FD17C0B8
:10D330002DEC3CEC4CE45FE3C501B4010E94599232
:10D340009B01AC01C701B6010E94F58F992787FDAB
:10D3500090958827990F881F9927019602C080E031
:10D3600090E0FF90EF90DF90CF90BF90AF909F90B4
:10D370008F9008958F929F92AF92BF92CF92DF923B
:10D38000EF92FF920F931F93CF93DF936C01EB010A
:10D39000EC84FD8486E0E816F1040CF443C0EE0C46
:10D3A000FF1C06E010E045EC842E4DE9942E4CE184
:10D3B000A42E41E8B42E8A859B85FC01E00FF11F65
:10D3C00040815181F8013497E80FF91F6081718124
:10D3D000C60189DFFC01A501940163E971E080E0E9
:10D3E00091E00E9466934F01AA2497FCA094BA2C66
:10D3F00086269726A826B9260E5F1F4F0E151F05F5
:10D40000D1F68C829D82AE82BF8280E290E09987C5
:10D4100088878FEF9FEF9983888361E070E080E0D9
:10D4200090E003C060E070E0CB01DF91CF911F91ED
:10D430000F91FF90EF90DF90CF90BF90AF909F90B3
:10D440008F9008950F931F93CF93DF938C01EB017F
:10D450008CEC9DE09B878A878091C90D90E09D8729
:10D460008C878091960E90E09F878E878091C60D65
:10D47000853009F051C0C8011BD3882319F081E021
:10D4800090E04CC0BE01C801B0D78111F8CFBE01F9
:10D49000C80107D78111F3CFBE01C8017ED2811127
:10D4A000EECFBE01C801CCD48111E9CFBE01C801C5
:10D4B00069D58111E4CFBE01C80192D38111DFCFBC
:10D4C000BE01C801E3D18111DACFBE01C8012DD15F
:10D4D0008111D5CFBE01C80145D68111D0CFBE0183
:10D4E000C8010E9490728111CACFBE01C8011BD031
:10D4F0008111C5CFBE01C801A2D08111C0CFBE012C
:10D50000C80138DF672B682B692B09F0B8CF82E0A0
:10D510008093C60D1092C90D80E090E0DF91CF910D
:10D520001F910F910895AF92BF92CF92DF92EF9229
:10D53000FF920F931F93CF93DF93EB018091C90D5F
:10D54000883510F480E070C0EA85FB858281938184
:10D5500060E672E26ADD892BA9F3EA85FB858481A6
:10D56000958164E971E1A9DD892B61F3BEE1CB2EE0
:10D57000D12C1DE1E12EF12C00E010E08091C90DCD
:10D5800090E00497E816F906ACF5EA85FB85C7013B
:10D59000880F991FE80FF91F8081918164EF71E076
:10D5A00044DD892B79F25601AA0CBB1CEA85FB8568
:10D5B000EA0DFB1D8081918168E572E07EDD892B9B
:10D5C00021F0000F111F01600DC0EA85FB85EA0DF7
:10D5D000FB1D8081918164EA76E06FDD892B49F043
:10D5E000000F111F82E0E80EF11C82E0C80ED11C72
:10D5F000C5CF760181E0E81AF108F594E794F98641
:10D60000E8868AE2E816F1040CF49CCFC801AA2748
:10D6100097FDA095BA2F8C839D83AE83BF8389E04D
:10D6200090E09983888381E0DF91CF911F910F91E2
:10D63000FF90EF90DF90CF90BF90AF900895AF92A2
:10D64000BF92CF92DF92EF92FF920F931F93CF93EF
:10D65000DF93EB018091C90D803211F080E05AC058
:10D66000EA85FB85828193816CE271E0DEDC892BA7
:10D67000A9F3EA85FB85848195816EEE72E01DDD5C
:10D68000892B61F306E010E0C12CD12C7601EA85EC
:10D69000FB85E00FF11F808191816CE271E0C5DCB8
:10D6A000892BE1F2580182E0A80EB11CEA85FB85C6
:10D6B000EA0DFB1D8081918168E077E0FEDC892B1B
:10D6C00039F0CC0CDD1CEE1CFF1C6894C0F810C0B7
:10D6D000EA85FB85EA0DFB1D808191816EEE72E08B
:10D6E000ECDC892B09F4BACFCC0CDD1CEE1CFF1C42
:10D6F0000C5F1F4F0E33110551F68EE090E09987B5
:10D700008887CC82DD82EE82FF828FE090E0998371
:10D71000888381E0DF91CF911F910F91FF90EF906F
:10D72000DF90CF90BF90AF900895AF92BF92CF920D
:10D73000DF92EF92FF920F931F93CF93DF93EB0152
:10D740008091C90D823251F5EA85FB8582819381F2
:10D7500068E572E06ADC892B09F18091C90D90E0DF
:10D7600081509048880F991FEA85FB85E80FF91FC3
:10D770008081918168E572E058DC892B79F0198607
:10D7800018868FEF9FEFDC018C839D83AE83BF8370
:10D7900086E090E09983888381E06DC0EA85FB850F
:10D7A0008281938160E47FE140DC892B21F08091CC
:10D7B000C90D813210F480E05EC0EA85FB8584816A
:10D7C000958160EA7FE079DC892BA9F358E0A52EEA
:10D7D000B12C03E010E0C12CD12C7601EA85FB8549
:10D7E000C801880F991FE80FF91F8081918168E5B2
:10D7F00072E01BDC892BF9F2EA85FB85EA0DFB1D43
:10D800008081918160E476E058DC892B39F0CC0C82
:10D81000DD1CEE1CFF1C6894C0F810C0EA85FB8577
:10D82000EA0DFB1D8081918166E272E046DC892B66
:10D8300009F4C1CFCC0CDD1CEE1CFF1C0E5F1F4F8A
:10D8400084E0A80EB11C0332110541F6EA85FB8580
:10D85000EA5BFF4F8081918168E572E0E6DB892B0E
:10D8600009F4A9CF80E190E099878887CC82DD8296
:10D87000EE82FF828DCFDF91CF911F910F91FF90AC
:10D88000EF90DF90CF90BF90AF900895AF92BF928E
:10D89000CF92DF92EF92FF920F931F93CF93DF937C
:10D8A000EB018091C90D893310F480E06BC0EA85EB
:10D8B000FB858281938160E47FE1B7DB892BA9F34B
:10D8C000EA85FB858481958160EA7FE0F6DB892B20
:10D8D00061F338E0A32EB12C03E010E0C12CD12C71
:10D8E0007601EA85FB85C801880F991FE80FF91FAB
:10D8F0008081918168E572E098DB892BB1F2EA853D
:10D90000FB85EA0DFB1D8081918160E476E0D5DB2B
:10D91000892B39F0CC0CDD1CEE1CFF1C6894C0F880
:10D9200010C0EA85FB85EA0DFB1D8081918166E2CE
:10D9300072E0C3DB892B09F4B8CFCC0CDD1CEE1CE4
:10D94000FF1C0E5F1F4F84E0A80EB11C0B331105A6
:10D9500041F6EA85FB85EA58FF4F8081918168E5B1
:10D9600072E063DB892B09F4A0CF8CE190E099870A
:10D970008887CC82DD82EE82FF828AE090E0998304
:10D98000888381E0DF91CF911F910F91FF90EF90FD
:10D99000DF90CF90BF90AF9008956F927F928F925B
:10D9A0009F92AF92BF92CF92DF92EF92FF920F932E
:10D9B0001F93CF93DF93EB018091C90D823208F45E
:10D9C0005DC0EA85FB85828193816EE571E02DDB88
:10D9D000892B09F453C063E0A62EB12C02E010E0BD
:10D9E000C12CD12C760135018091C90D90E0A8168B
:10D9F000B906CCF54801880C991CEA85FB85E80D31
:10DA0000F91D808191816EE977E00FDB892B39F078
:10DA1000CC0CDD1CEE1CFF1C6894C0F80FC0EA851E
:10DA2000FB85E80DF91D808191816EEE72E0FDDAD3
:10DA3000892B21F1CC0CDD1CEE1CFF1CC501880FCD
:10DA4000991FEA85FB85E80FF91F808191816EE5BA
:10DA500071E033DB22E0A20EB11C892B19F00E5FBE
:10DA60001F4FC1CF830101501109159507951987E3
:10DA700008870031110524F41986188680E009C052
:10DA8000CC82DD82EE82FF828CE090E099838883F5
:10DA900081E0DF91CF911F910F91FF90EF90DF9088
:10DAA000CF90BF90AF909F908F907F906F90089590
:10DAB000AF92BF92CF92DF92EF92FF920F931F939C
:10DAC000CF93DF93EB01EA85FB858281938168E246
:10DAD00073E2ABDA892B11F480E077C08091C90D35
:10DAE000843009F5EA85FB85848195816AEC78E0CC
:10DAF000E4DA892BC1F0EA85FB858681978160E3B2
:10DB000072E093DA892B79F0198618868FEF9FEFF0
:10DB1000DC018C839D83AE83BF8383E090E0998397
:10DB2000888381E052C08091C90D8434A8F2EA85CF
:10DB3000FB858481958164E971E1BFDA892B61F20B
:10DB400006E010E0C12CD12C7601EA85FB85E00FC0
:10DB5000F11F8081918160E372E067DA892B09F41B
:10DB6000BBCF580182E0A80EB11CEA85FB85EA0D07
:10DB7000FB1D808191816AE976E09FDA892B39F07B
:10DB8000CC0CDD1CEE1CFF1C6894C0F810C0EA85AC
:10DB9000FB85EA0DFB1D8081918160E372E08DDAE7
:10DBA000892B09F499CFCC0CDD1CEE1CFF1C0C5FFB
:10DBB0001F4F0638110549F680E290E09987888763
:10DBC000CC82DD82EE82FF82A8CFDF91CF911F91C0
:10DBD0000F91FF90EF90DF90CF90BF90AF9008959E
:10DBE0008F929F92AF92BF92CF92DF92EF92FF926D
:10DBF0000F931F93CF93DF9300D01F92CDB7DEB763
:10DC00004B01DB011A96ED91FC911B978281938168
:10DC10006EEA7DE00ADA892B11F480E08FC0D4012E
:10DC20001A96ED91FC911B978481958166ED76E0C3
:10DC3000FCD9892B91F3E6E0EE2EF12C20E030E0C8
:10DC400040E050E0A12CB12CC12CD12CD4011A966B
:10DC5000ED91FC911B97EE0DFF1D8081918166EF88
:10DC600071E029833A834B835C83DFD9892BA9F246
:10DC700087010E5F1F4FD4011A96ED91FC911B97FF
:10DC8000E00FF11F808191816CED74E016DA29813B
:10DC90003A814B815C81892B39F0B501C60101E0E5
:10DCA0000E94F49321601CC0D4011A96ED91FC915E
:10DCB0001B97E00FF11F8081918160E971E029835A
:10DCC0003A834B835C83F9D929813A814B815C810A
:10DCD000892B09F4A2CFB501C60101E00E94F4939B
:10DCE0005B016C01B4E0EB0EF11CE6ECEE16F10406
:10DCF00009F0ACCFD40114962C93149715963C934D
:10DD0000159716964C93169717965C931797B5012F
:10DD1000C60100E20E940F9412962C93129713965C
:10DD20003C93139785E090E011969C938E9380E34B
:10DD300090E019969C938E93189781E00F900F9026
:10DD40000F900F90DF91CF911F910F91FF90EF9067
:10DD5000DF90CF90BF90AF909F908F9008958F925B
:10DD60009F92AF92BF92CF92DF92EF92FF920F936A
:10DD70001F93CF93DF937A016901DA01CD91DC9192
:10DD8000FB0184859585C817D9070CF047C0CE01E3
:10DD9000880F991F0284F385E02DE80FF91FA080FA
:10DDA000B180C170DD27F1E0CF27209719F484E618
:10DDB00090E002C08CE99FEF4801880E991EB401E3
:10DDC000C501EDD8892B89F4800E911EB401C501DF
:10DDD000E6D8892B69F4B401600F711FC501DFD843
:10DDE000892BF9F023E030E005C021E030E002C0EB
:10DDF00022E030E0D6018D919C9111970196821717
:10DE0000930744F0F60111821082D7018D919C9105
:10DE1000119701968D939C93CE0105C081E090E00F
:10DE200002C08FEF9FEFDF91CF911F910F91FF9075
:10DE3000EF90DF90CF90BF90AF909F908F9008951C
:10DE40004F925F926F927F928F929F92AF92BF920A
:10DE5000CF92DF92EF92FF920F931F93CF93DF93B6
:10DE600000D01F92CDB7DEB76C017B011C821B82F4
:10DE700081E090E09A8389838091C90D8D3010F400
:10DE800080E06BC009E713E09E012D5F3F4FAE01BC
:10DE90004F5F5F4FC60163DF892B91F79E012D5FB6
:10DEA0003F4FAE014F5F5F4FB701C60158DF01978B
:10DEB00039F79E012D5F3F4FAE014F5F5F4FB701B6
:10DEC000C6014DDF892BE1F6412C512C3201A12CEA
:10DED000B12C8091C90D90E029813A81281739072A
:10DEE0008CF509E713E09E012D5F3F4FAE014F5FB8
:10DEF0005F4FB701C60133DF4C019E012D5F3F4FDD
:10DF0000AE014F5F5F4FB701C60129DF21E08216E6
:10DF1000910451F4892B09F0B3CF440C551C661CB5
:10DF2000771C689440F80AC0892809F0A9CF0197A6
:10DF300009F0A6CF440C551C661C771C8FEFA81A5D
:10DF4000B80AC7CFF701B186A0864482558266829F
:10DF5000778281E090E0918380830F900F900F9003
:10DF60000F90DF91CF911F910F91FF90EF90DF9075
:10DF7000CF90BF90AF909F908F907F906F905F9069
:10DF80004F9008952F923F924F925F926F927F929F
:10DF90008F929F92AF92BF92CF92DF92EF92FF92B9
:10DFA0000F931F93CF93DF9300D01F92CDB7DEB7AF
:10DFB0006C017B011C821B82DB011C968D919C9164
:10DFC0001D971816190614F080E0B5C0DB011A96EB
:10DFD000ED91FC911B9782E090E09A838983828186
:10DFE00093816AE67AE021D8892B71F3D7011A96DA
:10DFF000ED91FC911B9789819A819C012F5F3F4F86
:10E000003A832983880F991FE80FF91F8081918136
:10E0100069E773E052D8892BB9F20CEB11E09E014D
:10E020002D5F3F4FAE014F5F5F4FB701C60197DED7
:10E03000892B51F69E012D5F3F4FAE014F5F5F4F21
:10E04000B701C6018CDE019709F0BECF212C312C1F
:10E050002101A12CB12C29813A81F7018485958574
:10E06000281739070CF05CC00CEB11E09E012D5F06
:10E070003F4FAE014F5F5F4FB701C60170DE3C01FD
:10E08000B3E0AB16B10489F00CEB11E09E012D5FFB
:10E090003F4FAE014F5F5F4FB701C60160DE4C01DD
:10E0A000E3E0AE16B104F9F40FC00CEB11E09E01F1
:10E0B0002D5F3F4FAE014F5F5F4FB701C6014FDE8F
:10E0C0006816790609F380CF0CEB11E09E012D5FF5
:10E0D0003F4FAE014F5F5F4FB701C60140DE88166C
:10E0E000990609F071CF6114710459F48A94892852
:10E0F00009F06ACF220C331C441C551C689420F88C
:10E100000BC06A94672809F05FCF892809F05CCFBB
:10E11000220C331C441C551CAFEFAA1ABA0A9BCF21
:10E12000B186A086248235824682578282E090E0C2
:10E130009183808381E00F900F900F900F90DF917B
:10E14000CF911F910F91FF90EF90DF90CF90BF90F4
:10E15000AF909F908F907F906F905F904F903F9087
:10E160002F900895AF92BF92CF92DF92EF92FF92DD
:10E170000F931F93CF93DF93EB01EA85FB85828199
:10E18000938168E873E10E941568892B11F480E09F
:10E190007DC08091C90D843019F5EA85FB858481A5
:10E1A00095816AEC78E00E945D68892BC9F0EA8568
:10E1B000FB858681978160E372E00E941568892B58
:10E1C00079F0198618868FEF9FEFDC018C839D8391
:10E1D000AE83BF8387E090E09983888381E056C057
:10E1E0008091C90D843498F2EA85FB8584819581FC
:10E1F00068E873E10E945D68892B49F206E010E04F
:10E20000C12CD12C7601EA85FB85E00FF11F8081BE
:10E21000918160E372E00E941568892B09F4B7CF01
:10E22000580182E0A80EB11CEA85FB85EA0DFB1DB2
:10E230008081918160E476E00E945D68892B39F0ED
:10E24000CC0CDD1CEE1CFF1C6894C0F811C0EA85E4
:10E25000FB85EA0DFB1D8081918160E372E00E94E5
:10E260005D68892B09F493CFCC0CDD1CEE1CFF1CE0
:10E270000C5F1F4F0638110531F680E290E0998758
:10E280008887CC82DD82EE82FF82A4CFDF91CF919E
:10E290001F910F91FF90EF90DF90CF90BF90AF90C4
:10E2A00008958F929F92AF92BF92CF92DF92EF929A
:10E2B000FF920F931F93CF93DF93EB018091C90DD2
:10E2C0008A3108F47AC0EA85FB85808191818032A9
:10E2D000934050F4198618868FEF9FEFDC018C83F2
:10E2E0009D83AE83BF836FC0828193816CEA7DE0A2
:10E2F0000E941568892B09F460C0EA85FB8584813A
:10E3000095816CEA7DE00E941568892B09F455C05F
:10E3100054E0A52EB12C03E010E0C12CD12C7601E5
:10E320008091C90D90E0A816B906E4F5EA85FB8551
:10E33000C801880F991FE80FF91F8081918166EB52
:10E3400073E00E945D68892B61F14501880C991C7E
:10E35000EA85FB85E80DF91D8081918160E679E011
:10E360000E941568892B39F0CC0CDD1CEE1CFF1CBB
:10E370006894C0F810C0EA85FB85E80DF91D80811E
:10E3800091816CEB72E00E941568892BB1F0CC0C86
:10E39000DD1CEE1CFF1C0E5F1F4F82E0A80EB11C9F
:10E3A000BFCF850101501109159507951987088779
:10E3B0000C30110524F41986188680E009C0CC823F
:10E3C000DD82EE82FF828BE090E09983888381E09A
:10E3D000DF91CF911F910F91FF90EF90DF90CF9041
:10E3E000BF90AF909F908F9008958F929F92AF9221
:10E3F000BF92CF92DF92EF92FF920F931F93CF9332
:10E40000DF93EB018091C90D8A3108F471C0EA8570
:10E41000FB8580819181843F914060F41986188644
:10E420008FEF9FEFDC018C839D83AE83BF838BE0F6
:10E4300090E066C08281938160E679E00E94156871
:10E44000892B09F455C073E0A72EB12C02E010E02F
:10E45000C12CD12C76018091C90D90E0A816B90687
:10E46000E4F5EA85FB85C801880F991FE80FF91FBD
:10E470008081918168E572E00E945D68892B61F17D
:10E480004501880C991CEA85FB85E80DF91D808102
:10E49000918160EB74E00E941568892B39F0CC0CF7
:10E4A000DD1CEE1CFF1C6894C0F810C0EA85FB85DB
:10E4B000E80DF91D8081918168E572E00E94156880
:10E4C000892BB1F0CC0CDD1CEE1CFF1C0E5F1F4F26
:10E4D00082E0A80EB11CBFCF85010150110915952E
:10E4E0000795198708870C30110524F419861886BA
:10E4F00080E009C0CC82DD82EE82FF8284E090E081
:10E500009983888381E0DF91CF911F910F91FF90D4
:10E51000EF90DF90CF90BF90AF909F908F90089535
:10E52000AF92BF92CF92DF92EF92FF920F931F9321
:10E53000CF93DF93EB018091C90D863410F480E016
:10E5400086C0EA85FB85828193816EEE72E00E942F
:10E550001568892BA1F3EA85FB85848195816EEE90
:10E5600072E00E945D68892B51F3EA85FB85868104
:10E57000978162E27BE00E941568892B01F3EA85AE
:10E58000FB858085918562E27BE00E945D68892B36
:10E59000B1F25CE0A52EB12C05E010E0C12CD12C2D
:10E5A0007601EA85FB85C801880F991FE80FF91FDE
:10E5B000808191816EEE72E00E941568892B09F4CA
:10E5C000BECFEA85FB85EA0DFB1D8081918166E661
:10E5D00078E00E945D68892B39F0CC0CDD1CEE1CC4
:10E5E000FF1C6894C0F811C0EA85FB85EA0DFB1D8D
:10E5F000808191816EEE72E00E945D68892B09F442
:10E600009ECFCC0CDD1CEE1CFF1C0E5F1F4F84E068
:10E61000A80EB11C0534110521F6EA85FB85E657E5
:10E62000FF4F808191816EEE72E00E941568892B08
:10E6300009F485CF80E290E099878887CC82DD82DB
:10E64000EE82FF8288E090E09983888381E0DF9109
:10E65000CF911F910F91FF90EF90DF90CF90BF90DF
:10E66000AF90089521EF39E0FC01318320830895B4
:10E6700021EF39E0FC01318320830C942C8F0F9320
:10E680001F93CF93DF938C01EB0188E2FB01119282
:10E690008A95E9F74BE050E06BE17AE0CE010E9409
:10E6A000C8961B8641E050E060E070E04C875D87D3
:10E6B0006E877F87F801458956896789708D488BF9
:10E6C000598B6A8B7B8B42E050E060E070E04C8BB2
:10E6D0005D8B6E8B7F8B1CA21DA21EA21FA240E031
:10E6E00050E068E474E4488F598F6A8F7B8F40E074
:10E6F00050E068E474EC4C8F5D8F6E8F7F8F4DEC33
:10E700005CEC6CE47EE348A359A36AA37BA3DF918E
:10E71000CF911F910F91089527E23AE0FC013183D8
:10E720002083458B568B678B708F0895CF93DF9333
:10E730001F921F92CDB7DEB786E09DE02A83498302
:10E740000E948E604981642F86E09DE00E944760B0
:10E750002A81622F86E09DE00E94476086E09DE06E
:10E760000F900F90DF91CF910C940C610F931F933A
:10E77000CF93DF938C01EB01262F41E06EE1D6DFD2
:10E78000F801D483C383C038D10509F45BC0DCF43D
:10E79000C034D105A9F1C036D10509F442C0A09713
:10E7A00009F08AC080E090E8A9E8B4E48093A1046D
:10E7B0009093A204A093A304B093A40480E090E0FB
:10E7C000A5E7B4E471C0C03CD10509F44CC0C03E1B
:10E7D000D10509F459C0C03AD10509F06DC080E0F7
:10E7E00090E0A8ECB3E48093A1049093A204A093DA
:10E7F000A304B093A40480E090E0AFE7B3E454C076
:10E8000080E090ECA5E5B4E48093A1049093A20489
:10E81000A093A304B093A40480E090E0AEE3B4E43A
:10E8200043C080E090E8A7E2B4E48093A104909311
:10E83000A204A093A304B093A40480E090E0A6E116
:10E84000B4E432C080E090E0A1EEB3E48093A10490
:10E850009093A204A093A304B093A40480E090E05A
:10E86000A8ECB3E421C080E090E0A5EAB3E4809393
:10E87000A1049093A204A093A304B093A40480E005
:10E8800090E8A3E9B3E410C080E090E0A6E6B3E42A
:10E890008093A1049093A204A093A304B093A40432
:10E8A00080E090E0ADE4B3E480939D0490939E04F7
:10E8B000A0939F04B093A004DF91CF911F910F917B
:10E8C0000895CF93DF93EC0186E09DE00E94856080
:10E8D00020E042E06EE1CE0129DF60E270E0CE018F
:10E8E00045DF81E0DF91CF9108956F927F928F9203
:10E8F0009F92AF92BF92CF92DF92EF92FF920F93CF
:10E900001F93CF93DF93EC016EE186E09DE00E94C0
:10E910008E60E091060DF091070D0190F081E02DE1
:10E9200063E086E09DE0199586E09DE00E940C6121
:10E9300046E06EE186E09DE00E94086186E09DE091
:10E940000E94F05F0697D4F386E09DE00E94F85F96
:10E95000682E86E09DE00E94F85F782E86E09DE0BC
:10E960000E94F85FC82E86E09DE00E94F85FD82ED6
:10E9700086E09DE00E94F85F882E86E09DE00E9480
:10E98000F85F982EB62CA12CA728B501882777FD13
:10E990008095982F0E94C5906D837E838F83988782
:10E9A000F82CE12CE928B701882777FD8095982F6E
:10E9B0000E94C59069877A878B879C871C2D00E011
:10E9C0000D29B801882777FD8095982F0E94C59062
:10E9D0006D877E878F87988B198A1A8A1B8A1C8A73
:10E9E000DF91CF911F910F91FF90EF90DF90CF902B
:10E9F000BF90AF909F908F907F906F900895CF922F
:10EA0000DF92EF92FF920F931F93CF93DF938C01CE
:10EA1000EB0184E2FB0111928A95E9F7C80165DFF9
:10EA200084E290E0A0E0B0E088839983AA83BB836E
:10EA3000F80185899689A789B08D8C839D83AE83E3
:10EA4000BF8382E090E0A0E0B0E088879987AA8742
:10EA5000BB87188A198A1A8A1B8AC090A104D09091
:10EA6000A204E090A304F090A404A701960165819C
:10EA70007681878190850E94F98F20E030E048EC14
:10EA800052E40E9459926C8B7D8B8E8B9F8BA701D9
:10EA90009601F80161857285838594850E94F98FBE
:10EAA00020E030E048EC52E40E945992688F798F60
:10EAB0008A8F9B8F20919D0430919E0440919F04EA
:10EAC0005091A004F80165857685878590890E941C
:10EAD000F98F20E030E048EC52E40E9459926C8FAC
:10EAE0007D8F8E8F9F8F81E0DF91CF911F910F914E
:10EAF000FF90EF90DF90CF900895FC011082148278
:10EB0000138215820895862F642F0C940A83862F12
:10EB1000642F0C944383862F0C9478834F925F92DA
:10EB20006F927F928F929F92AF92BF92CF92DF921D
:10EB3000EF920F93CF93DF93EC014B013A01590110
:10EB40000296DBDF85E39AE0998388836E018CE18E
:10EB5000C80ED11C26018CE3480E511CC601CDDF26
:10EB600086E0C80ED11CC414D504C1F7FE01EE59CD
:10EB7000FF4F718260823296B182A082329600830A
:10EB80003196E08237979182808238968AE090E0D1
:10EB900091838083329684EF91E0918380833396D2
:10EBA0001182108271971082118212821382C459CD
:10EBB000DF4F1882DF91CF910F91EF90DF90CF90D0
:10EBC000BF90AF909F908F907F906F905F904F908D
:10EBD00008952F923F924F925F926F927F928F9201
:10EBE0009F92AF92BF92CF92DF92EF92FF920F93DC
:10EBF0001F93CF93DF93CDB7DEB728970FB6F89466
:10EC0000DEBF0FBECDBF98878F83F12C4C0186E607
:10EC1000880E911C0F8118850E591F4FD4018C91BD
:10EC2000F816A0F4AF81B8858D919C91F801A08170
:10EC3000B181AF0DB11DFC012081318142E06C91A9
:10EC40008F819885F9011995F394E8CF512CEF81C4
:10EC5000F885E959FF4FFA83E9830F8118850C592C
:10EC60001F4FC12CD12C7601C3948F8198858E596A
:10EC70009F4F9C838B83A981BA818C91581608F091
:10EC800088C0A52CB12CAF81B8858D919C91F801DD
:10EC9000A081B181AA0DBB1DFC012081318141E021
:10ECA0006C918F819885F9011995AF81B8858D9107
:10ECB0009C91F801A081B181AA0DBB1DFC012281AC
:10ECC000338140E06C918F819885F9011995D701C6
:10ECD000C601052C04C0880F991FAA1FBB1F0A94E8
:10ECE000D2F79C011C0120943094412CD4018C91CA
:10ECF000EF81F88540815181481648F5642C712CCC
:10ED0000EB81FC81A081B181A60DB71DFA01448180
:10ED100055816C918F8198852D833E83FA011995D9
:10ED2000660C771C2D813E81EF81F885E60DF71D7D
:10ED3000892B29F480859185822B932B04C08085B3
:10ED4000918582219321918780874394CFCFF801C9
:10ED5000A081B181AA0DBB1DFA012281338141E05E
:10ED60006C918F819885F9011995AF81B8858D9146
:10ED70009C91F801A081B181AA0DBB1DFC012081ED
:10ED8000318140E06C918F819885F90119955394F8
:10ED900072CF28960FB6F894DEBF0FBECDBFDF91BD
:10EDA000CF911F910F91FF90EF90DF90CF90BF9088
:10EDB000AF909F908F907F906F905F904F903F901B
:10EDC0002F900895FC0180E090E0258D368D261768
:10EDD000370739F0019636968A309105B1F78FEFF3
:10EDE0009FEF0895DC0126E0629FA00DB11D112464
:10EDF00090965C934E935F9721E091962C93919718
:10EE0000FC01E459FF4F208131960190F081E02D03
:10EE1000222331F0309749F0611107C0DC0102C0B4
:10EE2000309719F05C968C9119940895CF92DF92E7
:10EE3000FF920F931F93CF93DF931F92CDB7DEB74F
:10EE40006C01F62EFC0186E0689FE00DF11D112497
:10EE500011A2878D90A181309105E9F01CF4892BD6
:10EE600051F044C08230910591F1039709F03EC002
:10EE700040E050E030C04423C9F141E050E0C60119
:10EE8000B1DF0E94CC81F601E85AFF4F60837183A5
:10EE9000828393832BC049830E94CC81F601E85A78
:10EEA000FF4F0081118122813381601B710B820B26
:10EEB000930B72960081118120E030E049810617A2
:10EEC00017072807390718F442E050E004C0411141
:10EED0000DC043E050E06F2DC6010F90DF91CF9140
:10EEE0001F910F91FF90DF90CF907CCF0F90DF911B
:10EEF000CF911F910F91FF90DF90CF9008952F92A7
:10EF00003F924F925F926F927F928F929F92AF92B9
:10EF1000BF92CF92DF92EF92FF920F931F93CF9306
:10EF2000DF931F92CDB7DEB71C01FC014AE08FEFE3
:10EF30009FEF278D30A1232B21F4148E968F858F80
:10EF400011A2415036964111F4CF712C610126E691
:10EF5000C20ED11C510187E6A80EB11C4101A0E6EA
:10EF60008A0E911C46E0442ED6018C91781608F04A
:10EF700053C0612C8101070D111D070D111D085F84
:10EF80001F4FF501E0806E1408F044C0F801408185
:10EF90005181062C02C0569547950A94E2F74170BC
:10EFA0007E9C70011124E60CF11CD401ED91FC91C2
:10EFB000EE0DFF1D5080B701C101498303DF498178
:10EFC00097FD02C0682F1BC0019611F5442301F183
:10EFD00080E090E060E070E0F101E80FF91F248D1F
:10EFE000211110C0469EF001479EF00D1124E20D44
:10EFF000F31D548EF68EE58E10A2178E41E0C101EE
:10F0000015DF06C06F5F7F4F06966A30710521F7E6
:10F010006394B7CF7394A8CF20E030E080E0F10193
:10F02000E20FF31F91A1911181E02A5F3F4F2C3332
:10F030003105A9F70F90DF91CF911F910F91FF90AC
:10F04000EF90DF90CF90BF90AF909F908F907F9088
:10F050006F905F904F903F902F900895CF92DF92E6
:10F06000EF92FF920F931F93CF93DF938C010E9437
:10F07000CC81E801C45ADF4FC880D980EA80FB8088
:10F080006C197D098E099F09F801E859FF4FC0806E
:10F09000D180E12CF12CC616D706E806F90660F4FB
:10F0A000C80197DDC8012BDF182F0E94CC8168832F
:10F0B00079838A839B8301C010E0812FDF91CF91F8
:10F0C0001F910F91FF90EF90DF90CF9008950F93D5
:10F0D0001F93CF93DF93EC018C0104591F4F81E004
:10F0E000F8018083CE01BADF882349F089A1882303
:10F0F00031F08F8D98A1019711F48C8D03C0F80128
:10F10000108280E0DF91CF911F910F9108950895B3
:10F11000CF92DF92EF92FF92FC0185899689481B7E
:10F12000590B61097109A389B4899A01AB010E9445
:10F13000E0936B017C018FE0F594E794D794C7943A
:10F140008A95D1F765857685882777FD8095982FF4
:10F150002BE0660F771F881F991F2A95D1F7278507
:10F160003089442737FD4095542F2C0D3D1D4E1DF1
:10F170005F1D0E94BE932C0D3D1D4E1D5F1DCA01DB
:10F18000B901FF90EF90DF90CF9008951F93CF9338
:10F19000DF931F92CDB7DEB7162F67E770E086E0EA
:10F1A0009DE049830E949860612F86E09DE00E9467
:10F1B00047604981642F86E09DE00E94476086E0B9
:10F1C0009DE00F90DF91CF911F910C940C61CF9334
:10F1D000C62F67E770E086E09DE00E9498606C2F84
:10F1E00086E09DE00E94476086E09DE00E940C6101
:10F1F00067E770E086E09DE00E94986041E050E0A3
:10F2000067E770E086E09DE00E940A6186E09DE08D
:10F210000E94F85FC82F86E09DE00E940C618C2F51
:10F22000CF910895CF93DF93C62F67E770E086E014
:10F230009DE00E9498606C2F86E09DE00E944760F0
:10F2400086E09DE00E940C6167E770E086E09DE04B
:10F250000E94986042E050E067E770E086E09DE041
:10F260000E940A6186E09DE00E94F85FD82F80E04E
:10F27000C82F86E09DE00E94F85FC82BD92B86E05E
:10F280009DE00E940C61CE01DF91CF910895CF9354
:10F29000DF93EC01643008F063E0688386E09DE072
:10F2A0000E94856060EDCE0192DF853509F039C09E
:10F2B0006AEACE01B7DF9A8389836CEACE01B2DFB6
:10F2C0009C838B836EEACE01ADDF9E838D8360EBE2
:10F2D000CE01A8DF9A8B898B62EBCE01A3DF9C8BDA
:10F2E0008B8B64EBCE019EDF9E8B8D8B66EBCE010C
:10F2F00099DF98878F8368EBCE0194DF9A8789879F
:10F300006AEBCE018FDF9C878B876CEBCE018ADFA7
:10F310009E878D876EEBCE0185DF988B8F8781E08E
:10F3200001C080E0DF91CF910895CF93DF93EC018E
:10F330004EE264EF2BDF65E070E080E090E00E9439
:10F34000FB8166EFCE01DF91CF916CCFCF93DF933E
:10F35000EC01EBDFAC0160E070E0CE01D9DE685F6C
:10F360007F4F8F4F9F4F34E09595879577956795A1
:10F370003A95D1F70E94C59020E030E040E251E498
:10F380000E94F98FDF91CF910895CF92DF92EF9293
:10F39000FF92CF93DF93EC0148814295440F440FD5
:10F3A000407C4C5C64EFF2DE8881811105C065E031
:10F3B00070E080E090E012C0813029F468E070E0F5
:10F3C00080E090E00BC0823029F46EE070E080E0D5
:10F3D00090E004C06AE170E080E090E00E94FB8170
:10F3E00066EFCE011FDF6C01E12CF12CFE2CED2C21
:10F3F000DC2CCC2468EFCE01EADEA7019601282B95
:10F40000CA01B901488128E030E0241B310904C059
:10F4100096958795779567952A95D2F7DF91CF9145
:10F42000FF90EF90DF90CF9008952F923F924F92F0
:10F430005F926F927F928F929F92AF92BF92CF9284
:10F44000DF92EF92FF920F931F93CF93DF93CDB78D
:10F45000DEB72A970FB6F894DEBF0FBECDBF9A87EE
:10F46000898763DF8C0189859A858FDF6D837E8331
:10F470008F839887A80160E070E089859A8548DECF
:10F480004B015C0180EA881A8FE0980AA108B10854
:10F49000A5019401C501B4010E9466932B013C01B2
:10F4A0000CE075946794579447940A95D1F7A98511
:10F4B000BA8511962D903C9012971C9115960D903F
:10F4C000BC91A02D0E94EA936B017C018DE0F59424
:10F4D000E794D794C7948A95D1F7E985FA85A781EF
:10F4E000B085A30192010E94EA93BB2797FDB095D6
:10F4F000AB2FC80ED91EEA1EFB1EF2E0CF0ED11CA8
:10F50000E11CF11C32E0F594E794D794C7943A9546
:10F51000D1F780E8D80EE11CF11CE985FA85A189B4
:10F52000B289A70196010E94E093DC01CB014FE074
:10F53000B695A795979587954A95D1F789839A832C
:10F54000AB83BC836101EE24D7FCE094FE2C52E037
:10F55000CC0CDD1CEE1CFF1C5A95D1F7A185B285A1
:10F56000A30192010E94EA932B013C016BE0759488
:10F570006794579447946A95D1F7A381B481A50104
:10F5800094010E94EA93EBE09595879577956795AE
:10F59000EA95D1F7460E571E681E791EC40CD51C7D
:10F5A000E61CF71C012E04C0CC0CDD1CEE1CFF1C5D
:10F5B0000A94D2F792E0C90ED11CE11CF11CC701DC
:10F5C000B60124E030E040E050E00E94BE938D811F
:10F5D0009E81AF81B885821B930BA40BB50B9C0158
:10F5E000AD0160E573EC80E090E004C096958795EE
:10F5F000779567951A95D2F70E94669397FD0DC08F
:10F60000660F771F881F991F29813A814B815C8182
:10F610000E949C9349015A010CC029813A814B8177
:10F620005C810E949C9349015A01880C991CAA1C78
:10F63000BB1C9927B7FC9A958B2D7A2D692D9B01C0
:10F64000AC010E9466939B01AC01AEEDBBE00E9451
:10F65000E0936C01FF24D7FCF094EF2CA3E4B3EE0D
:10F66000A50194010E94EC93BB2797FDB095AB2FA9
:10F67000C80ED91EEA1EFB1E9FECC90E9EE0D91EC5
:10F68000E11CF11CA4E0F594E794D794C794AA95E3
:10F69000D1F7C80CD91CEA1CFB1CC701B6012A967D
:10F6A0000FB6F894DEBF0FBECDBFDF91CF911F9193
:10F6B0000F91FF90EF90DF90CF90BF90AF909F9011
:10F6C0008F907F906F905F904F903F902F90089514
:10F6D0008F929F92AF92BF92CF92DF92EF92FF9262
:10F6E000CF93DF9300D01F92CDB7DEB74A015B0105
:10F6F0009CDE6B017C0120E03AE24DE257E4C5015B
:10F70000B4010E94F98F9B01AC0160E070E080E8D9
:10F710009FE30E942E8F26EF38E248EA50E40E94D1
:10F72000BC929B01AC01C701B60129833A834B838C
:10F730005C830E94C59029813A814B815C810E9443
:10F74000F98F0E9492900F900F900F900F90DF9181
:10F75000CF91FF90EF90DF90CF90BF90AF909F90B0
:10F760008F900895CF93DF9300D01F92CDB7DEB76F
:10F770009A01AB0129833A834B835C8356DE0E9456
:10F78000C59029813A814B815C810E94F98F21E0EB
:10F790003EED42E45EE30E94BC929B01AC0160E05E
:10F7A00070E080E89FE30E942E8F20E03AE24DE275
:10F7B00057E40E9459920F900F900F900F90DF9195
:10F7C000CF910895FB016181828170E0762F6627D9
:10F7D000680F711D882777FD8095982F0E94C5902E
:10F7E00020E030E040E85DE30E94599223E333E9F2
:10F7F00048E853E40C942E8F089521E06227FC0121
:10F80000808141C7CF93DF93EC01862F68834983C2
:10F810002A8361E0FFD661E0888135D760E0898185
:10F82000F9D660E08A81F6D661E089812CD761E063
:10F830008A8129D760E0CE01DF91CF91DECFFB0135
:10F8400081819081890F9281890F9381981304C0DF
:10F8500081E094819D3009F080E008952F923F92DD
:10F860004F925F926F927F928F929F92AF92BF92D0
:10F87000CF92DF92EF92FF920F931F93CF93DF937C
:10F8800000D000D0CDB7DEB78C013B014E8384D5CC
:10F890001B012C0180ED280E87E0381E411C511CF5
:10F8A00061E0C801AADFFE0131966F014E01F6E06A
:10F8B0008F0E911CF60185E011928A95E9F7760189
:10F8C00027E0A22EB12CF801818112D7019731F4E3
:10F8D00063D56215730584059505A8F3F801818148
:10F8E00007D7892B31F458D5621573058405950522
:10F8F000A8F3F8018281FCD6892B59F0F701208109
:10F9000081E090E00A2C01C0880F0A94EAF7282BC6
:10F910002083F1E0AF1AB108B0F69FEFE91AF90AB7
:10F92000E814F90469F638D5621573058405950560
:10F9300040F060E0C80161DF20E030E040EC5FE7CC
:10F940002EC08981EE818E13B5CFB601C80177DF55
:10F95000882309F4AFCF60E0C8014FDFB601C801CA
:10F9600031DFFB01DC016A946728B9F420E030E064
:10F9700040E151E4BF01CD010E94599220E030E006
:10F9800040EA50E40E94F98F20E030E040E052E489
:10F990000E942F8F9B01AC0102C09F01AD01B901F4
:10F9A000CA0126960FB6F894DEBF0FBECDBFDF9119
:10F9B000CF911F910F91FF90EF90DF90CF90BF906C
:10F9C000AF909F908F907F906F905F904F903F90FF
:10F9D0002F90089546E642CF4CE440CFFF920F931C
:10F9E0001F93CF93DF93FC010081C181D281F894F2
:10F9F0008981F02EF0948F21898378941DE711502E
:10FA000009F182E090E01DD588818023C1F3F8944C
:10FA10008A818F218A838981802B8983789480EEE3
:10FA200091E00FD5F89489818F21898386E490E055
:10FA300008D58881802311E009F010E078948AE9E4
:10FA400091E0FFD4812FDF91CF911F910F91FF9013
:10FA500008951F93CF93DF93FC011081C181D28160
:10FA6000912F909560FF11C0F8948A8189238A8331
:10FA70008981812B89838AE090E0E3D48A81812B7C
:10FA80008A83789487E390E010C0F8948A81892370
:10FA90008A838981812B898381E490E0D2D48A8111
:10FAA000812B8A83789485E090E0DF91CF911F913C
:10FAB000C8C40F931F93CF93DF93FC011081C181C2
:10FAC000D281F8948981812B89838A81012F0095C5
:10FAD00080238A8383E090E0B4D489818023898362
:10FAE0008AE090E0AED4C881789485E390E0A9D410
:10FAF0001C2381E009F480E0DF91CF911F910F91E9
:10FB00000895CF92DF92EF92FF920F931F93CF93BE
:10FB1000DF931F92CDB7DEB76C01E62E08E010E050
:10FB2000FF24F39461E09F2D9E2109F460E0C6015B
:10FB300049838FDFFF0C015011094981011511051F
:10FB400089F7411115C0F894D6011196ED91FC91F9
:10FB5000129791818C918095892381831196ED91E3
:10FB6000FC91129792818C9180958923828378945D
:10FB70000F90DF91CF911F910F91FF90EF90DF9049
:10FB8000CF900895EF92FF920F931F93CF93DF933F
:10FB90008C01C8E0D0E0F12CEE24E394C80189DFA9
:10FBA0008111FE28EE0C2197C9F78F2DDF91CF919F
:10FBB0001F910F91FF90EF900895CF92DF92FF92E7
:10FBC0000F931F93CF93DF931F92CDB7DEB78C01B6
:10FBD000F62E40E065E5798394DFCF2C7981D72E2E
:10FBE00088E0F82EF60161916F0140E0C80189DFDD
:10FBF000FA94C1F70F90DF91CF911F910F91FF9071
:10FC0000DF90CF90089540E06CEC7BCFFC01138631
:10FC10001586148627E030E0DF01A20FB31F13968C
:10FC20001C922115310519F021503109F5CF0895A5
:10FC30001F93CF93DF93EC01162F60E0812FEAD45E
:10FC4000612F70E0FB01EF56F34FE491E883FB0175
:10FC5000E952F34FE491F0E0EE0FFF1FE35EF24F45
:10FC6000859194919A838983CE01DF91CF911F91E1
:10FC7000CDCFAF92BF92CF92DF92EF92FF920F93D0
:10FC80001F93CF93DF931F92CDB7DEB75C01D62EC3
:10FC9000E72EFC01158511115EC049839FDE498165
:10FCA000811105C0F5011386158614866DC04423A5
:10FCB00019F040E060EF02C040E06CEEC50121DFCA
:10FCC00001E0F12CC12C11E0C501F3DE682FC50164
:10FCD0006983EFDE6981613019F48130B9F432C093
:10FCE0002F2D30E068131BC0F5018385181730F401
:10FCF000E20FF31F8381802349F402C0181731F00B
:10FD000060E0193058F4F501148708C0F501EF0DD3
:10FD1000F11D8381802B838361E009C0C12EF50131
:10FD2000E20FF31F8381902F909589238383C50170
:10FD300090DE1F5F000F11F4F39401E0F7E0FF1570
:10FD400008F0C2CF113438F0F501C386C11009C0E4
:10FD500081E0858706C0F50113861586148610E0BC
:10FD600013C0F50183818823B1F3ED2DFE2D80E0D2
:10FD700090E0D501A80FB91F13962C9121930196FD
:10FD800088309105B1F711E0812F0F90DF91CF916D
:10FD90001F910F91FF90EF90DF90CF90BF90AF90A9
:10FDA0000895DC0180E0615088F09D919827E92F4B
:10FDB000EF70F0E0E55DF34F249192959F70E92F8D
:10FDC000F0E0E55CF34F84918227EDCF0895FC01CC
:10FDD00012828FEF8183108213820895FC01838148
:10FDE000882331F0611103C08FEF81830895118260
:10FDF000089586E09DE00E948E6086E09DE00E946E
:10FE00000C6191E0811190E0892F0895CF93DF93E9
:10FE1000EC016A8386E09DE00E9485606A81CE01E4
:10FE2000E8DF8B83882329F086E09DE00E94F85F5D
:10FE300088838B8190E0DF91CF910895CF93DF93FA
:10FE4000EC018B818823A9F08981809586238883A2
:10FE50006A8186E09DE00E948E60688186E09DE078
:10FE60000E94476086E09DE00E940C61282F30E0F0
:10FE700002C020E030E081E090E0232B11F080E030
:10FE800090E0DF91CF91089508950895DC01ED9100
:10FE9000FC910284F385E02D41E0199581E090E02A
:10FEA0000895FC01138212822FE33AE0318320830C
:10FEB0000895DC01ED91FC910084F185E02D6FEF58
:10FEC0001994DC01ED91FC910284F385E02D40E072
:10FED000199461E0F6DF80ED97E0B3C2CF93DF9332
:10FEE000CDB7DEB728970FB6F894DEBF0FBECDBFF3
:10FEF0001D8220E42E8334E13F8334E53887198264
:10FF00002A8320E12B8320E52C83FC0127814217E3
:10FF100010F04FEF420FFC01308550E0FE01E40F7E
:10FF2000F51F303121F4243011F4218101C02581E5
:10FF3000260F2068622F28960FB6F894DEBF0FBEFA
:10FF4000CDBFDF91CF91BDCFFC0165816B7F658314
:10FF50006860B7CFFC016581262F246025836C6023
:10FF6000B0CFCF93DF93EC01423018F08C818860E2
:10FF70008C834F836887222329F0413019F48C81C8
:10FF800084608C8364E670E080E090E034D26C8121
:10FF900064FD2EC0E881F9810284F385E02D42E002
:10FFA00063E0CE01199584E991E14BD2E881F981B2
:10FFB0000284F385E02D42E063E0CE01199586E9E5
:10FFC00090E03FD2E881F9810284F385E02D42E0A0
:10FFD00063E0CE01199586E990E033D2E881F9819A
:10FFE0000284F385E02D42E062E0CE01199511C054
:10FFF0006062CE0166DF84E991E123D26C816062A8
:020000021000EC
:10000000CE015FDF86E990E01CD26C816062CE0198
:1000100058DF86E990E015D26C816062CE0151DF35
:100020008CE390E00ED284E08D83CE0193DFCE018D
:1000300050DF82E08E8366E0CE0143DFCE01DF91A8
:10004000CF9137CFCF92DF92FF920F931F93CF9331
:10005000DF931F921F92CDB7DEB78C01677088E0E7
:10006000689FB00111246064C80149835A8329DF65
:100070008EE190E0E6D14981C42E5A81D52EF12C33
:10008000D6016D916D01D801ED91FC910190F08147
:10009000E02DC801199588E290E0D3D1F394B8E03F
:1000A000FB12EECF0F900F90DF91CF911F910F9128
:1000B000FF90DF90CF90089521E001C0220F6A9554
:1000C000EAF7DC011C962C931C971A965C934E93CE
:1000D0001997ED91FC910084F185E02D60E0199471
:1000E000FC012485222391F081859285009719F4E3
:1000F000611105C006C0019721F4611102C0258776
:1001000001C015866585CF010E9698CE08950F9390
:100110001F93CF93DF93EC018C01025F1F4F6B8520
:10012000C80174DE019751F461E0C80157DE1C82FA
:1001300060E0C80183DE81E090E002C080E090E0F2
:10014000DF91CF911F910F9108958F92AF92CF922F
:10015000EF920F93CF93DF93CDB7DEB7FC016387A8
:10016000148615861286118681E0982F01C0990F9A
:100170004A95EAF7928B982F01C0990F2A95EAF7D2
:10018000938B982F01C0990F0A95EAF7948B982FBB
:1001900001C0990FEA94EAF7958B982F01C0990F47
:1001A000CA94EAF7968B982F01C0990FAA94EAF7A0
:1001B000978B01C0880F8A94EAF7808FDF91CF91E7
:1001C0000F91EF90CF90AF908F9008954F925F92E4
:1001D0006F927F928F92AF92CF92EF920F931F9375
:1001E000CF93DF9300D0CDB7DEB73C011B894C889D
:1001F0005D882B834A83698354DE8FE49AE0F301A0
:1002000091838083C3010E96E2DD2B814A8169814F
:10021000C3019BDFA201612FC3010F900F900F90CC
:10022000DF91CF911F910F91EF90CF90AF908F9072
:100230007F906F905F904F903FCFFF920F931F93EF
:10024000CF93DF93EC01F62E8C01025F1F4F6A897A
:100250006F29C801F3DD6A8960956F21C801DF91BC
:10026000CF911F910F91FF90E9CD20E030E050E059
:1002700060FF05C0FC01E20FF31F7589572B6695DF
:100280002F5F3F4F2430310599F7413011F4FC01C5
:100290004489FC016585652B642BCFCF0F931F9399
:1002A000CF93DF93EC01142F062F0F70423011F41F
:1002B00040E009C070E084E0759567958A95E1F7A4
:1002C000CE01D3DF412F602FCE01DF91CF911F915F
:1002D0000F91CBCF0F931F93CF93DF9300D0CDB768
:1002E000DEB78C012B834A83698311DF2B814A811E
:1002F0006981C8010F900F900F90DF91CF911F91EE
:100300000F912FCE1F920F920FB60F9211242F93A1
:100310003F938F939F93AF93BF938091980E90914B
:10032000990EA0919A0EB0919B0E3091970E23E0FA
:10033000230F2D3720F40196A11DB11D05C026E81D
:10034000230F0296A11DB11D2093970E8093980E46
:100350009093990EA0939A0EB0939B0E80919C0E51
:1003600090919D0EA0919E0EB0919F0E0196A11DA1
:10037000B11D80939C0E90939D0EA0939E0EB09302
:100380009F0EBF91AF919F918F913F912F910F90B1
:100390000FBE0F901F9018952FB7F8946091980E8C
:1003A0007091990E80919A0E90919B0E2FBF089597
:1003B0003FB7F89480919C0E90919D0EA0919E0E57
:1003C000B0919F0E26B5A89B05C02F3F19F001964E
:1003D000A11DB11D3FBF6627782F892F9A2F620F6D
:1003E000711D811D911D42E0660F771F881F991FA7
:1003F0004A95D1F70895CF92DF92EF92FF92CF9373
:10040000DF936B017C01D4DFEB01C114D104E10463
:10041000F10481F00E942D8FCBDF6C1B7D0B683EB9
:10042000734098F381E0C81AD108E108F108C85177
:10043000DC4FEBCFDF91CF91FF90EF90DF90CF902B
:1004400008958230910538F0880F991F880F991F01
:1004500005970197F1F70895789484B5826084BD7B
:1004600084B5816084BD85B5826085BD85B58160B8
:1004700085BDEEE6F0E0808181608083E1E8F0E018
:100480001082808182608083808181608083E0E847
:10049000F0E0808181608083E1EBF0E08081846026
:1004A0008083E0EBF0E0808181608083E1E9F0E02F
:1004B000808182608083808181608083E0E9F0E0D8
:1004C000808181608083E1EAF0E0808182608083C6
:1004D000808181608083E0EAF0E0808181608083B8
:1004E000E1E2F1E0808182608083808181608083AD
:1004F000E0E2F1E0808181608083EAE7F0E08081E2
:100500008460808380818260808380818160808339
:100510008081806880831092C10008958093A50433
:100520000895863308F0865320917B00982F9870A9
:10053000277F922B90937B0087702091A50490E4F5
:10054000299F90011124822B80937C0080917A0056
:10055000806480937A0080917A0086FDFCCF809140
:1005600078002091790090E0922B089590E0FC01B2
:100570003197E231F10508F04CC0EB56FF4F0C9477
:10058000DA93809180008F7703C0809180008F7D07
:1005900080938000089580918000877FF9CF84B593
:1005A0008F7702C084B58F7D84BD08958091B0009F
:1005B0008F7703C08091B0008F7D8093B000089545
:1005C000809190008F7707C0809190008F7D03C04D
:1005D00080919000877F8093900008958091A00083
:1005E0008F7707C08091A0008F7D03C08091A0000D
:1005F000877F8093A0000895809120018F7707C0A6
:10060000809120018F7D03C080912001877F80939E
:1006100020010895CF93DF9390E0FC01EF56F34F54
:100620002491FC01E952F34F8491882349F190E031
:10063000880F991FFC01EF5AF24FA591B491895C84
:10064000924FFC01C591D4919FB7611108C0F894F5
:100650008C91209582238C93888182230AC06230FA
:1006600051F4F8948C91322F309583238C938881A8
:10067000822B888304C0F8948C91822B8C939FBF2B
:10068000DF91CF9108950F931F93CF93DF931F9224
:10069000CDB7DEB7282F30E0F901E55BF34F849149
:1006A000F901EF56F34F1491F901E952F34F049118
:1006B0000023C1F0882319F0698358DF6981E02F96
:1006C000F0E0EE0FFF1FE95CF24FA591B4919FB7E8
:1006D000F8948C91611103C01095812301C0812B86
:1006E0008C939FBF0F90DF91CF911F910F91089531
:1006F000CF93DF93282F30E0F901E55BF34F84912E
:10070000F901EF56F34FD491F901E952F34FC49137
:10071000CC2389F081112ADFEC2FF0E0EE0FFF1FD0
:10072000E35EF24FA591B4912C912D2381E090E0EE
:1007300021F480E002C080E090E0DF91CF91089545
:100740000F931F93762F90E0FC01EF56F34F6491C7
:10075000FC01E952F34FE4917111762FF0E0EE0FB6
:10076000FF1FE35EF24F8591949189019A013F70DA
:10077000472F0E948807611571058105910531F0A9
:100780006F5F7F4F8F4F9F4F9F7003C060E070E09F
:10079000CB011F910F910895FC01818D228D90E076
:1007A000805C9F4F821B91098F7399270895FC01EC
:1007B000918D828D981731F0828DE80FF11D858D16
:1007C00090E008958FEF9FEF0895FC01918D828D49
:1007D000981761F0828DDF01A80FB11D5D968C9195
:1007E000928D9F5F9F73928F90E008958FEF9FEFA0
:1007F00008958CEB95E8892B39F080E090E0892B07
:1008000019F0BAD1811123C080E090E0892B41F02A
:1008100080E090E0892B21F00E94000081111AC035
:1008200087E696E8892B39F080E090E0892B19F073
:100830004ED2811112C082E197E8892B99F080E0B5
:1008400090E0892B79F0EED281110AC008950E94C0
:100850000000DACF0E940000E3CF0E940000EBCF3F
:100860000C9400000895FC01848DDF01A80FB11DD8
:10087000A35ABF4F2C91848D90E001968F739927D6
:10088000848FA689B7892C93A089B1898C918064C3
:100890008C93938D848D981306C00288F389E02D84
:1008A00080818F7D80830895CF93DF93EC01888DC5
:1008B0008823C1F0EA89FB89808185FD05C0A8896C
:1008C000B9898C9186FD0EC00FB607FCF5CF8081EB
:1008D00085FFF2CFA889B9898C9185FFEDCFCE0134
:1008E000C2DFE8CFDF91CF910895CF92DF92FF92E0
:1008F0000F931F93CF93DF931F92CDB7DEB76C0199
:1009000081E0D60158968C9358975B969C915B97A3
:100910005C968C915C97981307C05096ED91FC9172
:100920005197808185FD2DC0F601038D10E00F5F8A
:100930001F4F0F731127F02EF601848DF81210C08F
:100940000FB607FCF9CFD6015096ED91FC91519767
:10095000808185FFF1CFC601698385DF6981ECCF96
:10096000838DE80FF11DE35AFF4F6083D6015B963C
:100970000C935B975296ED91FC9153978081806226
:100980000CC0D6015696ED91FC9157976083509616
:10099000ED91FC91519780818064808381E090E0AB
:1009A0000F90DF91CF911F910F91FF90DF90CF902B
:1009B0000895BF92CF92DF92EF92FF92CF93DF9391
:1009C000EC016A017B01B22EE889F98982E080831B
:1009D000411581EE580761057105A1F060E079E0ED
:1009E0008DE390E0A70196010E949C93215031096C
:1009F000410951095695479537952795211580E16D
:100A0000380798F0E889F989108260E874E88EE187
:100A100090E0A70196010E949C9321503109410961
:100A200051095695479537952795EC85FD85308377
:100A3000EE85FF852083188EEC89FD89B082EA89D6
:100A4000FB89808180618083EA89FB89808188605D
:100A50008083EA89FB89808180688083EA89FB89B9
:100A600080818F7D8083DF91CF91FF90EF90DF9029
:100A7000CF90BF900895CF93DF93EC01E881F98187
:100A80000284F385E02D1995EA89FB8980818F7EA8
:100A90008083EA89FB898081877F8083EA89FB895B
:100AA00080818F778083EA89FB8980818F7D808335
:100AB0008A8D898FDF91CF9108951F920F920FB683
:100AC0000F9211240BB60F922F938F939F93EF9356
:100AD000FF93E091B00EF091B10E8081E091B60EDF
:100AE000F091B70E82FD12C090818091B90E8F5F98
:100AF0008F732091BA0E821751F0E091B90EF0E099
:100B0000E056F14F958F8093B90E01C08081FF911F
:100B1000EF919F918F912F910F900BBE0F900FBE71
:100B20000F901F9018951F920F920FB60F921124DD
:100B30000BB60F922F933F934F935F936F937F93D7
:100B40008F939F93AF93BF93EF93FF9380EA9EE0C1
:100B50008ADEFF91EF91BF91AF919F918F917F912D
:100B60006F915F914F913F912F910F900BBE0F901E
:100B70000FBE0F901F90189580EA9EE00DDE21E0D9
:100B8000892B09F420E0822F08951092A30E109271
:100B9000A20E88EE93E0A0E0B0E08093A40E9093C4
:100BA000A50EA093A60EB093A70E8FE59AE09093A2
:100BB000A10E8093A00E85EC90E09093AD0E8093F3
:100BC000AC0E84EC90E09093AF0E8093AE0E80EC70
:100BD00090E09093B10E8093B00E81EC90E09093F2
:100BE000B30E8093B20E82EC90E09093B50E80939A
:100BF000B40E86EC90E09093B70E8093B60E1092F0
:100C0000B90E1092BA0E1092BB0E1092BC0E08953F
:100C10001F920F920FB60F9211240BB60F922F93C3
:100C20008F939F93EF93FF93E0914D0FF0914E0FB1
:100C30008081E091530FF091540F82FD12C090819A
:100C40008091560F8F5F8F732091570F821751F04D
:100C5000E091560FF0E0E35CF04F958F8093560FD4
:100C600001C08081FF91EF919F918F912F910F9003
:100C70000BBE0F900FBE0F901F9018951F920F92F2
:100C80000FB60F9211240BB60F922F933F934F93F1
:100C90005F936F937F938F939F93AF93BF93EF93E4
:100CA000FF938DE39FE0DFDDFF91EF91BF91AF9167
:100CB0009F918F917F916F915F914F913F912F9174
:100CC0000F900BBE0F900FBE0F901F9018958DE3E5
:100CD0009FE062DD21E0892B09F420E0822F089556
:100CE0001092400F10923F0F88EE93E0A0E0B0E02A
:100CF0008093410F9093420FA093430FB093440F02
:100D00008FE59AE090933E0F80933D0F85ED90E044
:100D100090934A0F8093490F84ED90E090934C0F8D
:100D200080934B0F80ED90E090934E0F80934D0F8A
:100D300081ED90E09093500F80934F0F82ED90E003
:100D40009093520F8093510F86ED90E09093540F43
:100D50008093530F1092560F1092570F1092580F06
:100D60001092590F08951F920F920FB60F921124EF
:100D70000BB60F922F938F939F93EF93FF93E09176
:100D8000EA0FF091EB0F8081E091F00FF091F10FFD
:100D900082FD12C090818091F30F8F5F8F7320913D
:100DA000F40F821751F0E091F30FF0E0E652F04FAC
:100DB000958F8093F30F01C08081FF91EF919F91F8
:100DC0008F912F910F900BBE0F900FBE0F901F9021
:100DD00018951F920F920FB60F9211240BB60F9217
:100DE0002F933F934F935F936F937F938F939F9333
:100DF000AF93BF93EF93FF938AED9FE034DDFF91B4
:100E0000EF91BF91AF919F918F917F916F915F9182
:100E10004F913F912F910F900BBE0F900FBE0F90EF
:100E20001F9018958AED9FE0B7DC21E0892B09F42B
:100E300020E0822F08951092DD0F1092DC0F88EED3
:100E400093E0A0E0B0E08093DE0F9093DF0FA093DB
:100E5000E00FB093E10F8FE59AE09093DB0F809362
:100E6000DA0F85E391E09093E70F8093E60F84E338
:100E700091E09093E90F8093E80F80E391E09093E5
:100E8000EB0F8093EA0F81E391E09093ED0F809355
:100E9000EC0F82E391E09093EF0F8093EE0F86E3E7
:100EA00091E09093F10F8093F00F1092F30F109256
:100EB000F40F1092F50F1092F60F0895CF92DF9273
:100EC000EF92FF920F931F93CF93DF937C016A0100
:100ED000EB0100E010E00C151D0571F06991D701E0
:100EE000ED91FC910190F081E02DC7011995892BBE
:100EF00019F00F5F1F4FEFCFC801DF91CF911F9106
:100F00000F91FF90EF90DF90CF90089561157105DC
:100F100081F0DB010D900020E9F7AD01415051094E
:100F2000461B570BDC01ED91FC910280F381E02D13
:100F3000199480E090E00895EF92FF920F931F9331
:100F4000CF93DF938C017B01C0E0D0E0F701EC0F81
:100F5000FD1F6491662359F0F801A081B181ED91E4
:100F6000FC91C8011995892B11F02196EFCFCE0184
:100F7000DF91CF911F910F91FF90EF900895DC01C9
:100F8000ED91FC91DB0114964D915C9115976D915B
:100F90007C910280F381E02D1994B8CFDC01ED91B2
:100FA000FC910190F081E02D19946BE67AE0AECFD0
:100FB0000F931F93CF93DF93EC01BEDF8C01CE0123
:100FC000F4DF800F911FDF91CF911F910F91089552
:100FD0000F931F93CF93DF93EC01D1DF8C01CE01F0
:100FE000E4DF800F911FDF91CF911F910F91089542
:100FF0000F931F93CF93DF93EC0188DF8C01CE0119
:10100000D4DF800F911FDF91CF911F910F91089531
:101010000F931F93CF93DF93EC01C0DF8C01CE01C0
:10102000C4DF800F911FDF91CF911F910F91089521
:101030008F929F92AF92BF92CF92DF92EF92FF92E8
:101040000F931F93CF93DF93CDB7DEB7A1970FB662
:10105000F894DEBF0FBECDBF7C01C42EE52FCB01BF
:10106000D22E19A221E02D1510F02AE0D22E8E01E9
:101070000F5D1F4F8D2C912CA12CB12C6C2D7E2F30
:10108000A50194010E949C938C2DD29E801911245D
:10109000015011098A3014F4805D01C0895CF801A7
:1010A0008083211531054105510521F0C22EE32F22
:1010B000CA01E4CFB801C70129DFA1960FB6F894A1
:1010C000DEBF0FBECDBFDF91CF911F910F91FF907B
:1010D000EF90DF90CF90BF90AF909F908F9008954A
:1010E000CF92DF92EF92FF920F931F93CF93DF93F4
:1010F000EC016A017B012115310579F4E881F98160
:101100000190F081E02D642FDF91CF911F910F911D
:10111000FF90EF90DF90CF9019942A303105D9F4E9
:1011200077FF18C06DE23ADF8C0144275527BA01DA
:101130004C195D096E097F092AE0CE0179DF800F25
:10114000911FDF91CF911F910F91FF90EF90DF9052
:10115000CF9008952AE0B701A601CE01DF91CF918B
:101160001F910F91FF90EF90DF90CF9061CF9A0188
:10117000AB01662757FD6095762FB2CF0F931F9373
:10118000CF93DF93EC019A01AB01662757FD609581
:10119000762FA6DF8C01CE0108DF800F911FDF9133
:1011A000CF911F910F9108950F931F93CF93DF93CA
:1011B000EC0196DF8C01CE01F8DE800F911FDF91EC
:1011C000CF911F910F9108952115310541F4DC0154
:1011D000ED91FC910190F081E02D642F199428CFBE
:1011E0000F931F93CF93DF93EC019A01462F50E0AA
:1011F00060E070E0E9DF8C01CE01D7DE800F911F47
:10120000DF91CF911F910F9108950F931F93CF936B
:10121000DF93EC01D9DF8C01CE01C7DE800F911F77
:10122000DF91CF911F910F9108954F925F926F922E
:101230007F928F929F92AF92BF92CF92DF92EF9266
:10124000FF920F931F93CF93DF93EC016A017B0111
:10125000B22E9A01AB01C701B6010E944D938823BB
:1012600019F06EE67AE026C026013701E89477F897
:101270002FEF3FEF4FE75FE7C301B2010E944D93AD
:1012800081110CC02FEF3FEF4FE75FE7C301B201C1
:10129000ACD618161CF462E77AE00CC02FEF3FEFD3
:1012A0004FE75FE4C701B6010E949A911816A4F4B3
:1012B00066E77AE0CE01DF91CF911F910F91FF9009
:1012C000EF90DF90CF90BF90AF909F908F907F90E6
:1012D0006F905F904F901ACE2FEF3FEF4FE75FEC8C
:1012E000C701B60182D687FDE3CF20E030E0A90137
:1012F000C701B6017AD687FF09C06DE2CE014EDE86
:101300008C01F7FAF094F7F8F09402C000E010E0D6
:10131000A12C60E070E080E09FE3AB1439F020E0A6
:1013200030E040E251E465D6A394F7CF9B01AC01D5
:10133000C701B60194D56B017C01F9D62B013C01A4
:1013400022D79B01AC01C701B60188D56B017C0196
:101350002AE0B301A201CE016BDE080F191FBB20EA
:1013600031F06EE077E0CE01D1DD080F191F7B2C44
:10137000772021F120E030E040E251E4C701B601DE
:101380000E9459926B017C01CDD64B01AA2497FC97
:10139000A094BA2C2AE030E0B501A401CE01A0DE71
:1013A000080F191FC501B401F0D69B01AC01C7019C
:1013B000B60154D56B017C017A94DACFC801DF9174
:1013C000CF911F910F91FF90EF90DF90CF90BF9042
:1013D000AF909F908F907F906F905F904F90089507
:1013E00024CF0F931F93CF93DF93EC011EDF8C016B
:1013F000CE01DBDD800F911FDF91CF911F910F9107
:1014000008950F931F93CF93DF93EC010E94CC813B
:10141000688779878A879B87E881F9810680F781C9
:10142000E02DCE01199597FF15C00E94CC8108854B
:1014300019852A853B85601B710B820B930B0C81F0
:101440001D812E813F81601771078207930720F36A
:101450008FEF9FEFDF91CF911F910F910895FC01C6
:1014600044835583668377830895CF92DF92EF920A
:10147000FF920F931F93CF93DF937C016A01EB01DF
:1014800000E010E00C151D0541F0C701BADF97FD23
:1014900004C089930F5F1F4FF5CFC801DF91CF9133
:1014A0001F910F91FF90EF90DF90CF9008954F9292
:1014B0005F926F927F928F929F92AF92BF92CF92E4
:1014C000DF92EF92FF920F931F93CF93DF934C0124
:1014D000EB0186E0849F8001859F100D1124060F8B
:1014E000171FFB01E017F10708F582819381892B13
:1014F00019F13696F7CF4081518164817581DA0107
:10150000A60FB71F2C91332727FD3095821793071D
:1015100009F56F5F7F4F7583648322813381621782
:10152000730751F03696E017F10728F3C40169DF1D
:1015300097FD46C0FE01F7CFEC1BFD0BF595E79537
:101540002BEA3AEAE29FC001E39F900DF29F900DD3
:10155000112438C06115710529F3A480B580950167
:101560002150310935832483DA01A20FB31FAC91D6
:10157000BB27A7FDB0958A179B07F9F42115310504
:10158000C9F06A017B01E21AF30AE40EF51E412C50
:10159000512CD6016D906D01D7017D907D016710B2
:1015A00006C0BFEF4B1A5B0A4216530690F3421671
:1015B000530699F6B582A482B5CF232B71F6B2CF2C
:1015C0008FEF9FEFDF91CF911F910F91FF90EF90E1
:1015D000DF90CF90BF90AF909F908F907F906F9053
:1015E0005F904F900895CF93DF9300D000D0CDB798
:1015F000DEB7FE01319626E0DF011D922A95E9F75C
:101600007A8369835C834B8341E050E0BF014FDF05
:1016100021E0892B09F020E0822F26960FB6F8945E
:10162000DEBF0FBECDBFDF91CF910895DCCFFC01AF
:10163000808191810C94F294CF93DF93EC018881A7
:101640009981009711F00E94F294198218821D82EC
:101650001C821B821A82DF91CF9108950F931F93F2
:10166000CF93DF93EC018B016F5F7F4F888199816E
:101670000E948195009731F0998388831B830A83A8
:1016800081E001C080E0DF91CF911F910F9108951B
:10169000CF93DF93EC0188819981892B29F08A818E
:1016A0009B818617970758F4CE01D8DF882341F035
:1016B0008C819D81892B19F4E881F981108281E068
:1016C000DF91CF910895EF92FF920F931F93CF93E5
:1016D000DF93EC017B018A01BA01DADF811103C0DB
:1016E000CE01AADF07C01D830C83B70188819981D1
:1016F0000E94B396CE01DF91CF911F910F91FF9081
:10170000EF900895FC0111821082138212821582DB
:1017100014826115710551F0FB0101900020E9F779
:10172000AF0141505109461B570BCDCF0895EF92A1
:10173000FF920F931F93CF93DF93EC017B018A01FC
:10174000BA01A6DF811103C0CE0176DF07C01D8379
:101750000C83B701888199810E949A96CE01DF910E
:10176000CF911F910F91FF90EF9008950F931F93CA
:10177000CF93DF938C01EB01FC0180819181009775
:1017800099F0428153812C813D814217530750F0DB
:10179000688179810E94B3968C819D81F80195833F
:1017A000848313C00E94F29488819981F801918307
:1017B00080838A819B81938382838C819D819583A1
:1017C0008483198218821B821A821D821C82DF91F7
:1017D000CF911F910F910895CF93DF93EC01FB01FF
:1017E0008617970751F0608171816115710521F0AD
:1017F0004481558168DF01C01FDFCE01DF91CF91A9
:101800000895FC01118210821382128215821482C3
:10181000E3CFCF93DF93EC018617970709F0A6DF9C
:10182000CE01DF91CF910895CF93DF93EC0186171E
:10183000970709F09BDFCE01DF91CF910895CF93F9
:10184000DF93EC016115710559F0FB010190002057
:10185000E9F7AF0141505109461B570B34DF01C076
:10186000EBDECE01DF91CF910895CF93DF931F92EE
:101870001F92CDB7DEB7FC01118210821382128253
:101880001582148269831A82BE016F5F7F4FD7DF92
:101890000F900F90DF91CF9108950F931F93CF93E7
:1018A000DF93CDB7DEB762970FB6F894DEBF0FBEF9
:1018B000CDBF8C01CB01F8011182108213821282FC
:1018C0001582148250E0BE016F5F7F4F0E94F19637
:1018D000BE016F5F7F4FC801B2DF62960FB6F8940A
:1018E000DEBF0FBECDBFDF91CF911F910F91089545
:1018F0000F931F93CF93DF93CDB7DEB7A2970FB6A9
:10190000F894DEBF0FBECDBF8C01CB01BA01F80148
:1019100011821082138212821582148230E0AE018D
:101920004F5F5F4F0E940597BE016F5F7F4FC801F9
:1019300086DFA2960FB6F894DEBF0FBECDBFDF9153
:10194000CF911F910F910895EF92FF920F931F93E4
:10195000CF93DF93CDB7DEB7A1970FB6F894DEBF74
:101960000FBECDBF7C01CB01BA01F70111821082FD
:10197000138212821582148242E0420F8E010F5FA1
:101980001F4F78D7BC01C7015ADFA1960FB6F89454
:10199000DEBF0FBECDBFDF91CF911F910F91FF90A2
:1019A000EF900895EF92FF920F931F93CF93DF93E1
:1019B000CDB7DEB7A1970FB6F894DEBF0FBECDBF8F
:1019C0007C01CB01BA01F7011182108213821282CD
:1019D0001582148242E0420F8E010F5F1F4F4AD7DB
:1019E000BC01C7012CDFA1960FB6F894DEBF0FBE75
:1019F000CDBFDF91CF911F910F91FF90EF90089590
:101A00000F931F93CF93DF931F921F92CDB7DEB733
:101A10008C016115710559F0CB0169837A830E94AD
:101A2000A196AC0169817A81C80181DE01C004DE22
:101A3000C8010F900F90DF91CF911F910F910895E2
:101A4000FC01118210821382128215821482D8CF77
:101A5000EF92FF920F931F93CF93DF93EC017B01E3
:101A60000C811D816115710511F480E015C04115CF
:101A7000510589F0040F151FB8010ADE8823A9F368
:101A8000288139818C819D81B701820F931F0E942B
:101A9000B3961D830C8381E0DF91CF911F910F914D
:101AA000FF90EF900895FB01448155816081718121
:101AB000CFCF6115710551F0FB0101900020E9F7CE
:101AC000AF0141505109461B570BC2CF80E008952A
:101AD000CF93DF931F921F92CDB7DEB769831A822F
:101AE00041E050E0BE016F5F7F4FB2DF0F900F907B
:101AF000DF91CF910895CF93DF93EC01FB014481F7
:101B0000558160817181A4DF811102C0CE0194DD15
:101B1000CE01DF91CF910895CF93DF93EC01611552
:101B2000710561F0FB0101900020E9F7AF01415020
:101B30005109461B570B8CDF811102C0CE017CDDA1
:101B4000CE01DF91CF910895FA01DB0114964D91FA
:101B50005C911597DC0114962D913C911597241BEF
:101B6000350B2E173F0788F08D919C91009769F0F7
:101B7000DB016D917C916115710539F08E0F9F1F0E
:101B80000E94BA9621E0892B09F020E0822F089567
:101B9000FC0144815581FB012481358142175307A3
:101BA00018F040E050E0D0CF80E00895FC0124819F
:101BB00035816217730748F480819181009729F07D
:101BC000FC01E60FF71F8081089580E00895EECFB5
:101BD0000F931F93CF93DF93EB0141155105E9F06C
:101BE0002097D9F0FC016481758126173707A0F48E
:101BF000621B730B8A01015011096017710708F409
:101C00008B01FC0160817181620F731FA801CE01FD
